:020000040800F2
:10C000000000022075860108C5860108C586010862
:10C01000C5860108C5860108C58601080000000024
:10C02000000000000000000000000000C5860108BC
:10C03000C586010800000000C586010891040108BA
:10C04000C5860108C5860108C5860108C5860108A0
:10C05000C5860108C5860108C5860108C586010890
:10C06000C5860108C5860108C5860108C586010880
:10C07000C5860108C5860108C5860108C586010870
:10C08000C5860108C5860108C5860108C586010860
:10C09000C5860108C5860108C5860108C586010850
:10C0A000C5860108C5860108C5860108C586010840
:10C0B000C5860108C5860108C5860108C586010830
:10C0C000C5860108C5860108C5860108C586010820
:10C0D000C5860108C5860108C5860108C586010810
:10C0E000C5860108C5860108C5860108C586010800
:10C0F000C5860108C5860108C5860108C5860108F0
:10C10000C5860108C5860108C5860108C5860108DF
:10C11000C5860108C5860108C5860108C5860108CF
:10C12000C5860108C5860108C5860108C5860108BF
:10C13000C5860108C5860108C5860108C5860108AF
:10C14000C5860108C5860108C5860108C58601089F
:10C15000C5860108C5860108C58601087111010858
:10C16000C5860108C5860108C50A01083D09010800
:10C17000010A0108C586010800000000C586010803
:10C18000C5860108C5860108C5860108C58601085F
:10C19000C5860108C586010800000000C5860108A3
:10C1A000C5860108C58601080000000000000000E7
:10C1B000C58601080000000000000000C5860108D7
:10C1C000C5860108C5860108C5860108C58601081F
:08C1D000C5860108C5860108BF
:10C1D80010B5054C237833B9044B13B10448AFF3B9
:10C1E80000800123237010BDB8000020000000006B
:10C1F800CC8F01080C4B43B10C480D4910B5AFF377
:10C2080000800C48036823B910BD0A48036833B995
:10C218007047094B002BF7D0BDE810401847064B74
:10C22800002BF5D0184700BF00000000CC8F010894
:10C23800BC000020B400002000000000384B394842
:10C248001A68002142F0010210B41A6099601A6855
:10C2580022F0847222F480321A6058601A6883B01F
:10C2680022F480221A60D960009101911A6842F480
:10C2780080321A601A4603E0009BB3F5A04F09D03C
:10C28800136803F400330193009B01330093019B6F
:10C29800002BF1D0224B1B6813F4003318BF012385
:10C2A8000193019B012B05D01F4B204A9A6003B0D4
:10C2B80010BC70471A4B1E491A6C1E4C1E4842F09F
:10C2C80080521A640A6842F440420A609A689A6086
:10C2D8009A689A609A6842F480529A602268016863
:10C2E80042F0115242EA81125A601A6842F0807292
:10C2F8001A601A689201FCD51049094A40F2037085
:10C308000860996821F003019960996841F0020179
:10C318009960936803F00C03082BFAD1C4E700BFB7
:10C32800003802401030002400ED00E000C0000892
:10C33800007000402C00002028000020003C024033
:10C348001D4A936803F00C03082B20D00C2B09D04E
:10C358001A4B194A1A499268C2F303128A5CD340ED
:10C368000B617047506851685268144BC2F38812C9
:10C3780001F03F01B3FBF1F303FB02F30E4A5268ED
:10C38800C2F3027201325200B3FBF2F3E1E75068E4
:10C3980051685268094BC2F3881201F03F01B3FBA0
:10C3A800F1F303FB02F3044A5268C2F3014201327B
:10C3B8005200B3FBF2F3CCE7003802400024F4004B
:10C3C8000000002040F0BF60024B40F40030D8600D
:10C3D800704700BF00ED00E0C3785BB903781648EA
:10C3E8005A09203203F01F03012101FA03F340F830
:10C3F80022307047114A70B4D26843788678017841
:10C408000D48D243C2F30222C2F10405EDB20F2453
:10C41800AB4044FA02F23240DBB2134344181B012A
:10C4280001F01F0501224909DBB2AA4084F8003354
:10C4380070BC40F82120704700E100E000ED00E00A
:10C4480021F0604121F07F01014B01439960704761
:10C4580000ED00E029B9054A136923EA00001061DC
:10C468007047024B1A6910431861704700ED00E0ED
:10C47800044A136804280CBF43F0040323F00403A0
:10C488001360704710E000E00E4B0F481A68002157
:10C4980042F0010210B41A6099601A680B4C22F03D
:10C4A800A85222F410221A605C60C3F884001A684B
:10C4B80010BC22F480221A60D960C3F88C10C3F82B
:10C4C80094107047003802400030002010300024DB
:10C4D800024B00221A701870704700BF02380240E1
:10C4E80082B000230A4A019302E0B3F5A04F08D0B6
:10C4F800136813F4003F019B03F101030193019BAF
:10C50800F3D0034B1868C0F3404002B0704700BF37
:10C5180000380240034A136823F0F80343EAC000D6
:10C528001060704700380240014B1860704700BF28
:10C5380000004742064B002201281A701A7005D0E5
:10C54800042802D105221A70704770471870704786
:10C5580070380240014B1860704700BF800E474298
:10C5680070B4039C049E074D40EA046040EA0670DC
:10C578005B080843013B40EA821040EA03406860D8
:10C5880070BC704700380240014B1860704700BF0C
:10C598006000474230B4029C074D240744EA036414
:10C5A80052080443013A44EA811444EA0244C5F8B3
:10C5B800844030BC704700BF00380240014B18600F
:10C5C800704700BF68004742014B1860704700BFC2
:10C5D80070004742014B1860704700BF4C0047424B
:10C5E800034A936823F0EC63194301439160704751
:10C5F80000380240034A936823F078431943014303
:10C608009160704700380240034A936823F003039F
:10C6180018439060704700BF00380240024B98688A
:10C6280000F00C00704700BF00380240034A9368CE
:10C6380023F0F00318439060704700BF00380240B1
:10C64800034A936823F4E05318439060704700BF8F
:10C6580000380240034A936823F4604343EAC00069
:10C6680090607047003802402B4B9B6803F00C0326
:10C6780010B40C2B08D8DFE803F0070707070707F3
:10C688000707200707073700244B0360224A24497D
:10C698009468C4F303140C5DE34043609468C4F3E6
:10C6A80082240C5D23FA04F48460926810BCC2F3FF
:10C6B80042328A5CD340C36070471749174B4C68B5
:10C6C8004A68496802F03F02B3FBF2F3C1F38812EB
:10C6D80003FB02F3104A5268C2F3014201325200CE
:10C6E800B3FBF2F30360D1E70B490C4B4C684A6883
:10C6F800496802F03F02B3FBF2F3C1F3881203FB6F
:10C7080002F3054A5268C2F3027201325200B3FBC7
:10C71800F2F30360BAE700BF003802400024F400D7
:10C728001400002000F44073B3F5407F09D1084994
:10C738008A6820F0704322F4F81223F440731343FC
:10C748008B60034B1A6FC0F30B00104318677047D8
:10C7580000380240014B1860704700BF3C0E47424A
:10C76800014B1860704700BF400E47420C4BD3F88E
:10C778008C2050B122F0C052C3F88C20D3F88C2002
:10C7880042EA8101C3F88C10704722F0C062C3F8F6
:10C798008C20D3F88C201143C3F88C10704700BF4D
:10C7A80000380240044AD2F88C3023F4401318436E
:10C7B800C2F88C00704700BF00380240044AD2F823
:10C7C8008C3023F440031843C2F88C00704700BF34
:10C7D80000380240044AD2F88C30013823F01F0395
:10C7E8001843C2F88C00704700380240FFF7F2BFC8
:10C7F800054AD2F88C30013823F4F85343EA002371
:10C80800C2F88C30704700BF00380240FFF7F0BF15
:10C81800044AD2F88C3023F440331843C2F88C0011
:10C82800704700BF00380240044AD2F88C3023F029
:10C83800004343EAC070C2F88C00704700380240D9
:10C84800044AD2F88C3023F400431843C2F88C0011
:10C85800704700BF00380240FFF7F2BF014B186075
:10C86800704700BFE0114742044A136B19B923EA25
:10C878000000106370471843106370470038024087
:10C88800044A536B19B923EA0000506370471843F0
:10C898005063704700380240044A936B19B923EA81
:10C8A8000000906370471843906370470038024057
:10C8B800044A136C19B923EA00001064704718433E
:10C8C8001064704700380240044A536C19B923EACF
:10C8D80000005064704718435064704700380240A5
:10C8E800044A136919B923EA000010617047184314
:10C8F8001061704700380240044A536919B923EAA5
:10C90800000050617047184350617047003802407A
:10C91800044A936919B923EA0000906170471843E3
:10C928009061704700380240044A136A19B923EA33
:10C9380000001062704718431062704700380240C8
:10C94800044A536A19B923EA000050627047184331
:10C958005062704700380240044A136D19B923EA3F
:10C968000000106570471843106570470038024092
:10C97800044A536D19B923EA0000506570471843FB
:10C988005065704700380240044A936D19B923EA8C
:10C998000000906570471843906570470038024062
:10C9A800044A136E19B923EA000010667047184349
:10C9B8001066704700380240044A536E19B923EADA
:10C9C80000005066704718435066704700380240B0
:10C9D800044A136F01280CBF43F0080323F008032F
:10C9E8001367704700380240064BD3F8942022F0B2
:10C9F8004042C3F89420D3F894201043C3F894001D
:10CA0800704700BF00380240054AD2F89430012828
:10CA18000CBF43F0006323F00063C2F89430704702
:10CA280000380240054AD2F8943001280CBF43F080
:10CA3800805323F08053C2F8943070470038024086
:10CA4800064BD3F8942022F44002C3F89420D3F87C
:10CA580094201043C3F89400704700BF0038024088
:10CA6800044A137819B923EA000010707047184374
:10CA7800107070470D3802404309012B0BD0022B70
:10CA8800094B0CBF1B6F5B6F00F01F0023FA00F00F
:10CA980000F001007047044B1B6800F01F0023FAE8
:10CAA80000F000F00100704700380240024A536F5E
:10CAB80043F080735367704700380240034BDB68CC
:10CAC800184214BF01200020704700BF0038024000
:10CAD800014B1870704700BF0E38024008B54B4B29
:10CAE80098422AD04A4B984231D04A4B984238D083
:10CAF800494B98423FD0494B984246D0484B9842C0
:10CB08004DD0484B984254D0474B98425BD0474B46
:10CB1800984262D0464B98426BD0464B984200D020
:10CB280008BD01214FF48060FFF7DAFE00214FF4C1
:10CB38008060BDE80840FFF7D3BE01210846FFF733
:10CB4800CFFE00210120BDE80840FFF7C9BE012142
:10CB58000220FFF7C5FE00210220BDE80840FFF7CC
:10CB6800BFBE01210420FFF7BBFE00210420BDE861
:10CB78000840FFF7B5BE01210820FFF7B1FE0021EC
:10CB88000820BDE80840FFF7ABBE01211020FFF7E1
:10CB9800A7FE00211020BDE80840FFF7A1BE012133
:10CBA8002020FFF79DFE00212020BDE80840FFF768
:10CBB80097BE01214020FFF793FE00214020BDE8E9
:10CBC8000840FFF78DBE01218020FFF789FE002174
:10CBD8008020BDE80840FFF783BE01214FF4807034
:10CBE800FFF77EFE00214FF48070BDE80840FFF794
:10CBF80077BE01214FF40070FFF772FE00214FF459
:10CC08000070BDE80840FFF76BBE00BF000002409F
:10CC18000004024000080240000C024000100240DC
:10CC28000014024000180240001C0240002002408C
:10CC3800002402400028024000222DE9F047134654
:10CC4800D1F800E001274FF0030C04E00133102B6A
:10CC580002F1020229D007FA03F434EA0E05F5D1ED
:10CC6800D0F800800E790CFA02F5ED4308EA0508C1
:10CC7800C0F80080D0F800A006FA02F9013E49EA9F
:10CC88000A09012E0CFA02F8C0F800900FD9C568FD
:10CC9800CC7925EA0805C560C568944001332C4362
:10CCA800102BC46002F10202D5D1BDE8F087D0F89C
:10CCB80008904E7905EA09058560D0F808908D79C5
:10CCC800964046EA09068660466826EA04044460F7
:10CCD800466805FA03F4A4B234434460D7E700BFBA
:10CCE80000234FF6FF720260037143718371C371B1
:10CCF800704700BF82B04FF480330193019B0B4310
:10CD08000193019BC361C161019BC361C369019325
:10CD1800C369019302B070470369194214BF012027
:10CD280000207047006980B2704700BF436919420C
:10CD380014BF012000207047406980B2704700BFCF
:10CD480001837047418370470AB941837047018363
:10CD5800704700BF4161704743695940416170475E
:10CD6800CB0800EB830001F0070110B4036A8900C7
:10CD78000F248C4023EA04030362036A10BC02FAFE
:10CD880001F119430162704708B5154B98421AD052
:10CD9800144B98424FF001010AD04FF00060FFF7A2
:10CDA800C3FD00214FF00060BDE80840FFF7BCBD9F
:10CDB8004FF08060FFF7B8FD00214FF08060BDE8BC
:10CDC8000840FFF7B1BD01214FF00070FFF7ACFD3F
:10CDD80000214FF00070BDE80840FFF7A5BD00BF77
:10CDE8000064004000680040036823F00203036009
:10CDF800036843F0010303604368DB0707D44FF679
:10CE0800FF7301E0013B02D04268D207FAD54368BC
:10CE180013F001035AD08B790A88012B03680CBFE1
:10CE280043F0800323F0800370B40360CB79012BB7
:10CE380003680CBF43F0400323F0400303600B7A00
:10CE4800012B03680CBF43F0200323F02003036089
:10CE58004B7A012B03680CBF43F0100323F0100337
:10CE680003608B7A012B03680CBF43F0080323F09F
:10CE780008030360CB7A012B03680CBF43F004035B
:10CE880023F004030360CB788E780D794C791B0668
:10CE980043EA867343EA054343EA0453013A1343DA
:10CEA800C361036823F0010303604368D90707D50A
:10CEB8004FF6FF7301E0013B02D04268D207FAD473
:10CEC8004068C04300F0010070BC704718467047C6
:10CED800D0F800328A7A43F00103C0F80032012307
:10CEE8002DE9F0419340D0F81C42DD432C40C0F8B6
:10CEF8001C420C7B002C40D1D0F80C72B1F806C053
:10CF08004E88B1F804E00C8800EBC2022F4046EAD4
:10CF18000C4644EA0E44C0F80C72C2F84062C2F8EB
:10CF28004442CA7A1ABBD0F804222A40C0F8042224
:10CF38000A89A2B9D0F814222A40C0F814224A7BE0
:10CF4800012A04D1D0F81C221343C0F81C32D0F8AF
:10CF5800003223F00103C0F80032BDE8F081012A55
:10CF6800EDD1D0F814221A43C0F81422E7E7D0F81C
:10CF780004221A43C0F80422DAE7012CD1D1D0F8F0
:10CF88000CE2B1F800804F88B1F804C0CE8800EBFD
:10CF9800C20447EA084743EA0E0246EA0C46C0F8CC
:10CFA8000C22C4F84072C4F84462BAE7002310B4F3
:10CFB8000221032401220471417102808371C3712B
:10CFC800037243728372C3728370C37010BC70475C
:10CFD800D0F8003243F00103C0F80032D0F8003234
:10CFE80023F47C5323F00E03C0F80032D0F800324B
:10CFF80043EA0121C0F80012D0F8003223F00103FF
:10D00800C0F80032704700BF036819B923F48033B1
:10D018000360704743F48033036070470368A9B91D
:10D0280023F080030360D0F8843123F48073C0F8C0
:10D038008431D0F8943123F48073C0F89431D0F857
:10D04800A43123F48073C0F8A431704743F08003FF
:10D058000360D0F8843143F48073C0F88431D0F889
:10D06800943143F48073C0F89431D0F8A43143F478
:10D078008073C0F8A43170478368F0B4054658013E
:10D0880005D4AB681A0142D50122104601E00022FE
:10D0980010461201AB18D3F8804104F00104C3F81C
:10D0A80080410C7A4CB34E684F7A44EAC604D3F8F0
:10D0B80080613C433443C3F880418C7A04F00F0408
:10D0C8008C72D3F8846126F00F06C3F88461D3F814
:10D0D80084613443C3F884412A44D1F80B40C2F830
:10D0E8008841D1F80F10C2F88C11D3F8802142F092
:10D0F8000102C3F88021F0BC70470F684C7AD3F85E
:10D10800806144EA47543443C3F88041D5E7AB68AB
:10D11800DB0002D502221046BBE70420F0BC7047B2
:10D1280001291AD015D302290FD183680D4A13405B
:10D138000D4A934206D007D90C4A934202D0094AB5
:10D14800934204D1012070470BB902207047002098
:10D1580070478368044A1340EAE78268034B134028
:10D16800E6E700BF00000310030000040003000806
:10D1780001290DD007D3022904D1836843F40003A1
:10D18800836070477047836843F08003836070470B
:10D19800836843F400438360704700BF00EB0113CA
:10D1A80010B4D3F8B04104F004041472C4BBD3F82B
:10D1B800B041640D1460D3F8B04104F00204547215
:10D1C800D3F8B44104F00F049472D3F8B44100EBDF
:10D1D8000113240AD474D3F8B841D472D3F8B841EF
:10D1E800240A1473D3F8B841240C5473D3F8B84103
:10D1F800240E9473D3F8BC41D473D3F8BC41240AE9
:10D208001474D3F8BC41240C5474D3F8BC311B0EED
:10D21800937451B1036910BC43F020030361704754
:10D22800D3F8B041E4085460C5E7C36810BC43F0C4
:10D238002003C360704700BF21B1036943F0200396
:10D2480003617047C36843F02003C360704700BFA1
:10D2580031B1012906BF006900F0030000207047C2
:10D26800C06800F003007047E9B9036823F00303BE
:10D2780043F001030360436803F00303012B09D063
:10D288004FF6FF7201E0013A04D0436803F003034C
:10D29800012BF8D1406800F00300A0F10100B0FABA
:10D2A80080F040097047012903D0022917D00020D7
:10D2B8007047036823F0030303604368990707D0A6
:10D2C8004FF6FF7301E0013B02D042689207FAD1A2
:10D2D800436813F0030F0CBF012000207047036858
:10D2E80023F0030343F002030360436803F00303DE
:10D2F800022B09D04FF6FF7201E0013A04D04368CF
:10D3080003F00303022BF8D1406800F00300A0F1FA
:10D318000200B0FA80F04009704700BF036823F0AC
:10D32800030343F002030360406800F00300A0F128
:10D338000200B0FA80F04009704700BF036823F08C
:10D34800020303604368990707D54FF6FF7301E0AE
:10D35800013B02D042689207FAD4406880F002008C
:10D36800C0F34000704700BF806900F0700070474C
:10D378008069000E704700BF8069C0F3074070479E
:10D3880043691AB923EA01014161704719434161B0
:10D39800704700BF11F4700F07D08369C3F31303FC
:10D3A8000B4214BF012000207047CB0107D543680A
:10D3B800C3F313030B4214BF0120002070470A0176
:10D3C80007D58368C3F313030B4214BF0120002061
:10D3D80070478B014CBFC3680369C3F313030B4247
:10D3E80014BF0120002070470A4B99420CD08A01D3
:10D3F800C1F3130306D44A0109D40A014CBF836060
:10D4080043607047C36070470023836170470361BE
:10D41800704700BF7000F03043690B400FD04029BF
:10D4280065D00ED9B1F5006F5AD017D8B1F5007F85
:10D438004ED0B1F5806F3FD0B1F5807F25D0002068
:10D448007047042948D016D910292FD0202929D06F
:10D458000829F4D1C068C0F300107047B1F5803FC7
:10D4680032D0B1F5003F2BD0B1F5004FE7D140687D
:10D47800C0F38000704701290BD00229DFD1C068B2
:10D4880010F0030018BF01207047806900F0010008
:10D498007047806800F0013020F08070003018BFBD
:10D4A800012070470069C0F3C0007047006910F0A0
:10D4B800030018BF012070478069C0F380007047DF
:10D4C8004068C0F3001070474068C0F3C000704760
:10D4D8008069C0F340007047C068C0F3C00070475F
:10D4E800836913F0700F14BF012000207047006992
:10D4F800C0F30010704700BFB1F5807F1ED00DD972
:10D50800B1F5006F24D013D9B1F5803F25D0B1F51E
:10D51800003F2ED0B1F5004F1AD0704708291FD010
:10D528000FD9202922D0402927D110230361704721
:10D53800B1F5007F02D0B1F5806F1DD1042343609F
:10D54800704701290FD0042918D10823C3607047F8
:10D5580000220423826143607047082343607047B8
:10D568001023C3607047064B83607047082303612C
:10D57800704710234360704770477047704700BF7B
:10D588000101010008B52D4B98421BD02C4B984245
:10D5980024D02C4B98422DD02B4B984236D02B4B75
:10D5A80098423FD02A4B984200D008BD01214FF441
:10D5B8000010FFF7C5F900214FF40010BDE808403E
:10D5C800FFF7BEB901214FF48050FFF7B9F90021E8
:10D5D8004FF48050BDE80840FFF7B2B901214FF47D
:10D5E8008040FFF7A1F900214FF48040BDE80840D2
:10D5F800FFF79AB901214FF40040FFF795F9002190
:10D608004FF40040BDE80840FFF78EB901214FF400
:10D618000050FFF795F900214FF40050BDE808408D
:10D62800FFF78EB901214FF48010FFF789F9002127
:10D638004FF48010BDE80840FFF782B90030014080
:10D6480000380040003C00400034014000500140D8
:10D65800005401400A884B88F0B48F88CD880C8923
:10D668004E8913433B432B4323438D89CC8902883E
:10D67800098A33432B43234302F4415213439BB299
:10D688000380838B23F400631B041B0C8383F0BC8F
:10D6980001827047838B23F47B6323F00F031B0401
:10D6A80002221B0C2DE9F041D1F808E083830284A3
:10D6B800858B9645ADB26AD0374B8E889A68002E16
:10D6C8000CBF4FF0010C4FF0020C120203D59A6800
:10D6D80022F400029A60304FD7F88430D7F884409B
:10D6E8007A68D7F8048018F4800F02F03F07C3F374
:10D6F8008813C4F30274294A36D1B2FBF7F703FB47
:10D7080007F3CF88B3FBF4F4B7F5007F36D04FEAC0
:10D718004C12B4FBF2F202EB82025300B3FBFEF3AD
:10D7280005339BB21E4AA2FB0323DB084FEA530EC4
:10D73800AEF1020203F00103FD2A94BF4EEA03236F
:10D7480002234A881F4322F08003302B078409D123
:10D758000C888B89224342F4C0521A4315432E4346
:10D76800B6B28683BDE8F081B2FBF7F2CF88B7F591
:10D77800007F03FB02F2B2FBF4F4C8D1240A04EBE5
:10D7880084046400B4FBFEF305339BB2CAE7734616
:10D798008E88CF88D5E700BF003802400024F40007
:10D7A800CDCCCCCC00230722028203804380838027
:10D7B800C380038143818381C38170470023022290
:10D7C8008260038043808380C3808381704700BF69
:10D7D800038829B923F040031B041B0C03807047FE
:10D7E8009BB243F040030380704700BF838B29B985
:10D7F80023F480631B041B0C838370479BB243F4A0
:10D8080080638383704700BF038823F400631B048D
:10D818001B0C038003889BB219430180704700BF2B
:10D82800B1F5804F038805D023F480431B041B0CFB
:10D83800038070479BB243F480430380704700BF66
:10D848004FF6FF639942038804D09BB243F4807378
:10D858000380704723F480731B041B0C03807047FC
:10D86800838829B923F004031B041B0C83807047A9
:10D878009BB243F004038380704700BF838829B9B3
:10D8880023F010031B041B0C838070479BB243F0EA
:10D8980010038380704700BF828B4B8822F47B6221
:10D8A80022F00F0270B412048E880C888D89120C35
:10D8B8000221828333430184818B24F4007243F470
:10D8C800006392B22B43002A43EA01039BB20CBFC8
:10D8D8004FF4807200221343838370BC704700BFEB
:10D8E800808980B2704700BF81817047038829B959
:10D8F80023F400531B041B0C038070479BB243F4B2
:10D9080000530380704700BF03889BB243F48053E1
:10D9180003807047012914BF008B808A80B270474A
:10D92800008A80B2704700BF83889BB21AB923EA85
:10D9380001018180704719438180704701230909DB
:10D9480003FA01F1838889B29BB21AB923EA01016B
:10D958008180704719438180704700BF038919424D
:10D9680014BF012000207047C94389B20181704764
:10D9780010B48488008901F00F03012280B202FAF2
:10D9880003F3184006D00909A4B28A40144214BF10
:10D998000120002010BC704701F00F01012303FA99
:10D9A80001F1C94389B20181704700BF08B5604BD6
:10D9B800984235D0B0F1804F3CD05E4B984243D06E
:10D9C8005D4B98424AD05D4B984251D05C4B98428F
:10D9D80058D05C4B98425FD05B4B984266D05B4B0B
:10D9E80098426DD05A4B984276D05A4B98427FD085
:10D9F800594B984200F08880584B984200F08E802E
:10DA0800574B984200D008BD01214FF48070FEF7B3
:10DA18008BFF00214FF48070BDE80840FEF784BFFB
:10DA280001210846FEF78CFF00210120BDE80840CF
:10DA3800FEF786BF01210846FEF776FF0021012088
:10DA4800BDE80840FEF770BF01210220FEF76CFF19
:10DA580000210220BDE80840FEF766BF012104202E
:10DA6800FEF762FF00210420BDE80840FEF75CBF16
:10DA780001210820FEF758FF00210820BDE80840D2
:10DA8800FEF752BF01211020FEF74EFF00211020A3
:10DA9800BDE80840FEF748BF01212020FEF744FFFB
:10DAA80000212020BDE80840FEF73EBF01210220EA
:10DAB800FEF746FF00210220BDE80840FEF740BF00
:10DAC80001214FF48030FEF73BFF00214FF48030F6
:10DAD800BDE80840FEF734BF01214FF40030FEF7DF
:10DAE8002FFF00214FF40030BDE80840FEF728BFA3
:10DAF80001214FF48020FEF723FF00214FF48020FE
:10DB0800BDE80840FEF71CBF01214020FEF70CFFCE
:10DB180000214020BDE80840FEF706BF0121802013
:10DB2800FEF702FF00218020BDE80840FEF7FCBE9A
:10DB3800000001400004004000080040000C0040C4
:10DB48000010004000140040000401400040014063
:10DB5800004401400048014000180040001C0040FB
:10DB680000200040234A038890429BB212D002F55D
:10DB7800806290420ED0B0F1804F0BD0A2F5803277
:10DB8800904207D002F58062904203D002F580628D
:10DB9800904203D14A8823F070031343164A9042F7
:10DBA8001FD002F5806290421BD070B423F44073FA
:10DBB8000E894D680C8802F56C429BB23343904243
:10DBC8000380C562048506D00C4B984203D001231C
:10DBD800838270BC70478B7A03860123838270BC72
:10DBE800704703800B884A68C262038501238382D9
:10DBF800704700BF000001400010004000040140D1
:10DC080000234FF0FF324260038003814380837218
:10DC1800704700BF01858282704700BF038823F0E8
:10DC280070031B041B0C1943018070474162704745
:10DC3800C1627047406A7047008D80B2704700BF6C
:10DC4800038829B923F002031B041B0C03807047C7
:10DC58009BB243F002030380704700BF038829B9D1
:10DC680023F004031B041B0C038070479BB243F092
:10DC780004030380704700BF038829B923F0800399
:10DC88001B041B0C038070479BB243F08003038086
:10DC9800704700BF038823F008031B041B0C038094
:10DCA80003889BB219430180704700BF038823F49F
:10DCB80040731B041B0C038003889BB2194301802B
:10DCC800704700BF038829B923F001031B041B0C0C
:10DCD800038070479BB243F001030380704700BF85
:10DCE800F0B5048C8F89B1F802E00E88194D24F044
:10DCF80001042404240C0484038C8488028B23F0FC
:10DD080002031B0422F073021B0C47EA0E071204DD
:10DD18003B43120CA8429BB2A4B242EA060209D0C5
:10DD280005F58065A84205D089688480028341632F
:10DD38000384F0BDCE890D8A4F8A23F0080333434C
:10DD480024F440748E883D4323F004032C4333436A
:10DD5800A4B2E9E700000140F0B5048C8E89B1F85F
:10DD680002C0B1F800E01D4D24F010042404240C76
:10DD78000484038C8788028B23F0200322F4E64274
:10DD88001B04120446EA0C041B0C120C43EA04138D
:10DD980042EA0E22A8429BB2BCB292B209D005F563
:10DDA8008065A84205D089688480028381630384E2
:10DDB800F0BDCD890E8A4F8A23F0800343EA05130C
:10DDC8004FF6BF751D408B8824F440643E4345EAF6
:10DDD800031344EA86049BB2A4B2E4E700000140BE
:10DDE800F0B5048C8D89B1F802C00F881E4E24F45A
:10DDF80080742404240C0484038CB0F804E0828B1F
:10DE080023F400731B0422F073021B0C45EA0C0474
:10DE1800120443EA0423120CB0429BB21FFA8EFE8E
:10DE280042EA070209D0114CA04206D08968A0F83E
:10DE380004E08283C1630384F0BDCC890D8A4E8AD5
:10DE480023F4006343EA04234FF6FF341C408B8815
:10DE58002EF4405E354344EA03234EEA051E9BB286
:10DE68001FFA8EFEE2E700BF0000014000040140F7
:10DE7800F0B5048C8E89B1F802E00F88164D24F4B1
:10DE880080542404240C0484038C8488828B23F417
:10DE9800005322F4E6421B0412041B0C46EA0E0649
:10DEA800120C43EA063342EA0722A8429BB2A4B204
:10DEB80092B209D005F58065A84205D089688480AA
:10DEC800828301640384F0BD0D8A24F4804444EA0B
:10DED8008514A4B2F2E700BF0000014000230380CC
:10DEE8004380838083608381C38103824382704738
:10DEF800038C10B401248C409BB223EA040321F064
:10DF080008040384183074B10439C1F34E0148F68B
:10DF1800FF740B5823400B5012020B5810BC92B2DE
:10DF28001A430A50704749084FF68F740B5823401C
:10DF38000B500B5810BC1A430A5070474163704786
:10DF480081637047C163704701647047038B23F096
:10DF580070031B041B0C194301837047038B23F4C4
:10DF6800E0431B041B0C43EA012189B2018370477B
:10DF7800838B23F070031B041B0C194381837047A8
:10DF8800838B23F4E0431B041B0C43EA012189B271
:10DF980081837047038B23F008031B041B0C194370
:10DFA80001837047038B23F400631B041B0C43EAB3
:10DFB800012189B201837047838B23F008031B0476
:10DFC8001B0C194381837047838B23F400631B0464
:10DFD8001B0C43EA012189B281837047038B23F02C
:10DFE80004031B041B0C194301837047038B23F4A0
:10DFF80080631B041B0C43EA012189B2018370472B
:10E00800838B23F004031B041B0C19438183704783
:10E01800838B23F480631B041B0C43EA012189B220
:10E0280081837047038B23F080031B041B0C194367
:10E0380001837047038BC3F30E0343EA012189B2BE
:10E0480001837047838B23F080031B041B0C194347
:10E0580081837047838BC3F30E0343EA012189B29E
:10E0680081837047038C23F002031B041B0C1943A4
:10E0780001847047038C23F008031B041B0C19430D
:10E0880001847047038C23F020031B041B0C43EA14
:10E09800011189B201847047038C23F080031B04AB
:10E0A8001B0C43EA011189B201847047038C23F4E5
:10E0B80000731B041B0C43EA012189B201847047D9
:10E0C800038C23F400631B041B0C43EA012189B26F
:10E0D80001847047038C23F400531B041B0C43EA90
:10E0E800013189B201847047038C10B401248C403B
:10E0F8009BB223EA04030384038C10BC02FA01F1E7
:10E10800194389B201847047038C10B404248C40ED
:10E118009BB223EA04030384038C10BC02FA01F1C6
:10E12800194389B2018470470B88F0B5002B2FD0B2
:10E13800042B048C4D8851D0082B79D024F48054BA
:10E148002404240CB1F804E00E89C9880484878B60
:10E15800028C45F6FF731340340340F6FF4244EA4D
:10E168000E243A4043F48053224343EA053392B2E3
:10E178009BB282830384828B22F440621204120CC5
:10E188008283838B9BB243EA01239BB28383F0BDD6
:10E19800028C4C888B880E89C98822F001021204EF
:10E1A800120C0284058B028CADB225F0F30592B2F5
:10E1B8002B4322F00A0243EA061322439BB242F0A1
:10E1C800010203830284038B23F00C031B041B0C42
:10E1D8000383038B9BB219430183F0BD24F0100421
:10E1E8002404240C8E88B1F808E0C9880484078BBD
:10E1F800038C9BB2340223F0A00340F6FF4244EAAA
:10E208000E343A4043F01003224343EA051392B216
:10E218009BB202830384028B22F440621204120C24
:10E228000283038B9BB243EA01239BB20383F0BDB5
:10E2380024F480742404240C8A880E89C9880484F0
:10E24800848B038CA4B29BB224F0F30423F42063E0
:10E25800224343F4807342EA061243EA05239BB241
:10E2680092B282830384838B23F00C031B041B0C60
:10E278008383838B9BB219438183F0BD00230122E2
:10E28800828003804380C38003817047F0B54F8844
:10E298008E880B88002F0CBF02220022012E0CBF93
:10E2A80002240124002B4CD0038C0D89C98823F04B
:10E2B80010031B041B0C0384B0F818C0038C9BB21A
:10E2C800360240F6FF4E23F0A00346EA05360EEA72
:10E2D8000C0E43F010034EEA060643EA0713B6B2E3
:10E2E8009BB206830384038B23F440631B041B0C3B
:10E2F8000383038B9BB243EA01239BB20383038C02
:10E3080023F001031B041B0C0384038B068C9BB2B4
:10E3180023F0F303B6B243EA051326F00A059BB2CD
:10E3280045F0010523432A4303830284038B23F02A
:10E338000C031B041B0C0383038B9BB2194301833F
:10E34800F0BD038CB1F808E0CD8823F001031B046D
:10E358001B0C0384018B038C89B221F0F3019BB25F
:10E368000E4323F00A0346EA0E163B43B6B243F0C7
:10E37800010306830384038B23F00C031B041B0C8B
:10E388000383038B9BB22B430383038C23F010037B
:10E398001B041B0C0384068B018C40F6FF4333409F
:10E3A80089B243EA0E3E21F0A0011FFA8EFE41F029
:10E3B80010014EEA042441EA021204830284038B0A
:10E3C80023F440631B041B0C0383038B9BB243EAB7
:10E3D8000525ADB20583F0BD406B7047806B704773
:10E3E800C06B7047006C7047038B23F00C031B0451
:10E3F8001B0C0383038B9BB219430183704700BF37
:10E40800038B23F440631B041B0C0383038B9BB215
:10E4180043EA012189B20183704700BF838B23F04F
:10E428000C031B041B0C8383838B9BB219438183CE
:10E43800704700BF838B23F440631B041B0C83834A
:10E44800838B9BB243EA012189B28183704700BF65
:10E45800F0B40A884F888B88CE880D894C898989C1
:10E468003A43134333432B4323430B439BB2A0F854
:10E478004430F0BC704700BF002303804380838092
:10E48800C380038143818381704700BFB0F8443063
:10E4980021B9C3F30E03A0F8443070476FEA434331
:10E4A8006FEA53439BB2A0F844307047838829B978
:10E4B80023F004031B041B0C838070479BB243F0BA
:10E4C80004038380704700BF838829B923F00103C0
:10E4D8001B041B0C838070479BB243F001038380AD
:10E4E800704700BF81827047038A194214BF012018
:10E4F80000207047C94389B201827047038A828924
:10E5080011EA030092B203D0114214BF0120002087
:10E51800704700BFC94389B2018270470A43A0F817
:10E528004820704783899BB21AB923EA0101818187
:10E538007047194381817047FFF7F4BF838829B971
:10E5480023F008031B041B0C838070479BB243F025
:10E5580008038380704700BF038923F007031B0467
:10E568001B0C0381704700BF038923F070031B0451
:10E578001B0C1943018103899BB243F007030381F4
:10E58800704700BF602970B427D0068C26F00106BA
:10E598003604360C0684058B068C25F0F304240417
:10E5A800240C26F00A0544EA03142D0442F0010263
:10E5B80044F001042D0CA4B2154304830584038997
:10E5C80023F070031B041B0C1943018103899BB2C0
:10E5D80043F00703038170BC7047048C24F01004D7
:10E5E8002404240C0484068B058C25F0A00540F631
:10E5F800FF442D0434402D0C44EA033345EA02124B
:10E6080043F4807342F010029BB292B203830284F7
:10E61800D5E700BF10B4048942EA03231943E4B2E2
:10E62800214389B20181038910BC23F077031B04BD
:10E638001B0C43F077030381704700BF10B40489B3
:10E6480042EA03231943E4B2214389B201810389D1
:10E6580010BC9BB243F4804303817047038923F0C5
:10E6680070031B041B0C194301817047838823F036
:10E6780070031B041B0C838083889BB21943818021
:10E68800704700BF038923F007031B041B0C038199
:10E6980003899BB219430181704700BF038923F0A6
:10E6A80080031B041B0C038103899BB2194301815E
:10E6B800704700BF10B404890A43E4B242EA032356
:10E6C80023439BB2038110BC704700BF70B4068916
:10E6D800048B058C24F4407424F0030425F02205EF
:10E6E80026F0070624042D0442EA03133604240CFA
:10E6F8002D0C360C44F480741D43314344F001045E
:10E70800ADB201810483058470BC7047838829B940
:10E7180023F080031B041B0C838070479BB243F0DB
:10E7280080038380704700BFA0F85010704700BF77
:10E73800044B054900221A605A609A60DA605961F0
:10E74800704700BF003C0140FFFF7F00837933B36F
:10E758001C4B0279417970B404681E68E5432E4069
:10E768001E605E6802F1804202F59E3235405D60AF
:10E7780015682C43146002689C68D04304409C6070
:10E78800DC68102900EA0400D86013D001F1804346
:10E7980003F59E3370BC19680A431A607047037901
:10E7A800016803F1804303F59E331A6822EA0102E7
:10E7B8001A607047996811439960D9680A43DA600A
:10E7C80070BC7047003C014000230C22427103607A
:10E7D80003718371704700BF024A136918431061BF
:10E7E800704700BF003C0140014B5861704700BFB3
:10E7F800003C0140034B5B69034214BF0120002029
:10E80800704700BF003C0140FFF7F4BF014B58615F
:10E81800704700BF003C014008B53A4B984221D0F0
:10E82800394B984228D0394B984231D0384B9842CE
:10E838003AD0384B984243D0374B98424CD0374B5C
:10E84800984253D0364B984200D008BD01214FF072
:10E858000040FEF769F800214FF00040BDE808408D
:10E86800FEF762B801211020FEF76AF80021102097
:10E87800BDE80840FEF764B801214FF40030FEF708
:10E8880053F800214FF40030BDE80840FEF74CB8BB
:10E8980001214FF48020FEF747F800214FF4802033
:10E8A800BDE80840FEF740B801214FF40020FEF70C
:10E8B8003BF800214FF40020BDE80840FEF734B8CB
:10E8C80001214FF48010FEF72FF800214FF480103B
:10E8D800BDE80840FEF728B801212020FEF730F8EF
:10E8E80000212020BDE80840FEF72AB801214FF09A
:10E8F8008040FEF719F800214FF08040BDE808403D
:10E90800FEF712B8001001400044004000480040E3
:10E91800004C0040005000400014014000780040C6
:10E92800007C0040028AF0B592B20446C8880D46C1
:10E9380022F4405202438989AB882F896E8922824A
:10E94800A28922F4B05222F00C023B431204334352
:10E95800120C9BB21343A381A38A9BB223F4407386
:10E968000B4385B0A3826846FDF77EFE1C4B9C4294
:10E9780028D003F580639C4224D0029AA389A189F8
:10E9880013F4004F2B68174D02EB820214BF5B0093
:10E998009B0002EB8202B2FBF3F0A5FB00325209A6
:10E9A800642303FB120310010A040DD41B01323344
:10E9B800A5FB0323C3F3431343EA000292B2228167
:10E9C80005B0F0BD039AD9E7D9003231A5FB013172
:10E9D800C1F34212024392B2228105B0F0BD00BFDA
:10E9E800001001401F85EB5100234FF416510C22F3
:10E9F800016042818380C38003818381704700BFA7
:10EA080030B40B884D888C88028AC9882B432343ED
:10EA18000B4392B29BB222F470621343038230BC60
:10EA2800704700BF0023038043808380C380704702
:10EA3800838929B923F400531B041B0C8381704775
:10EA48009BB243F400538381704700BF038B03F4E8
:10EA58007F430383038B9BB219430183704700BF35
:10EA6800838919B9C3F30E03838170476FEA43435F
:10EA78006FEA53439BB28381704700BF838A29B9E9
:10EA880023F400631B041B0C838270479BB243F47E
:10EA980000638382704700BFC1F30801818070471B
:10EAA8008088C0F308007047038A23F00F031B0413
:10EAB8001B0C0382038A9BB219430182704700BF73
:10EAC800838929B923F002031B041B0C8381704737
:10EAD8009BB243F002038381704700BF838923F40C
:10EAE80000631B041B0C838183899BB219438181BA
:10EAF800704700BF038A23F020031B041B0C03820A
:10EB0800038A9BB219430182704700BF038A29B95F
:10EB180023F480431B041B0C038270479BB243F40D
:10EB280080430382704700BF83899BB243F001038F
:10EB380083817047838A29B923F008031B041B0CBF
:10EB4800838270479BB243F008038382704700BFFB
:10EB5800038BDBB20383038B9BB243EA012101835E
:10EB6800704700BF838A29B923F020031B041B0CBC
:10EB7800838270479BB243F020038382704700BFB3
:10EB8800838A29B923F010031B041B0C8382704766
:10EB98009BB243F010038382704700BF838A23F03F
:10EBA80004031B041B0C8382838A9BB21943818252
:10EBB800704700BF838A29B923F002031B041B0C8A
:10EBC800838270479BB243F002038382704700BF81
:10EBD800838A9BB21AB923EA0101818270471943DB
:10EBE8008182704710B401F01F04C1F34211012360
:10EBF800012903FA04F30FD002290CBF1030143096
:10EC08002AB9026810BC22EA03030360704702684D
:10EC180010BC1343036070470C30F1E703881942B6
:10EC280014BF012000207047C94389B20180704792
:10EC3800C1F3421210B4012301F01F04012A03FAA0
:10EC480004F315D0022A0CBF028A828A92B21340BA
:10EC5800028892B24BB10123090A03FA01F10A4270
:10EC680014BF1846002010BC7047184610BC7047E7
:10EC7800828992B21340EBE7090A012303FA01F1F2
:10EC8800C94389B201807047014BC0B21870704700
:10EC9800003C0240054A136818B923F480731360D6
:10ECA800704743F480731360704700BF003C024014
:10ECB800054A136818B923F400731360704743F4C6
:10ECC80000731360704700BF003C0240054A136898
:10ECD80018B923F480631360704743F480631360AA
:10ECE800704700BF003C0240024A136843F40063C7
:10ECF80013607047003C0240024A136843F4805393
:10ED080013607047003C0240044B1A69002A03DA7A
:10ED18000349044A59605A60704700BF003C0240EA
:10ED280023016745AB89EFCD024A136943F00043DD
:10ED380013617047003C0240044B5A69D20703D55F
:10ED48000349044A99609A60704700BF003C02403A
:10ED58003B2A19087F6E5D4C024A536943F0010350
:10ED680053617047003C0240034A137803F07F0365
:10ED780018431070704700BF173C0240044B1A78C4
:10ED880002F0EF021A701A7810431870704700BF2B
:10ED9800143C0240044B1A7802F0F3021A701A78F5
:10EDA80010431870704700BF143C0240024B58696A
:10EDB800C0F34710704700BF003C0240014B188861
:10EDC80080B27047163C0240014B188880B27047E9
:10EDD8001A3C0240014B188880B27047163C02402A
:10EDE800014B188880B270471A3C0240024B1878D1
:10EDF800AA3818BF01207047153C0240024B18780A
:10EE080000F00C00704700BF143C0240044A13692C
:10EE180019B923EA00001061704718431061704760
:10EE2800003C0240034BDB68034214BF0120002072
:10EE3800704700BF003C0240014BD860704700BFDC
:10EE4800003C02400E4BDA68D20309D4DA68D106D6
:10EE580001D506207047DA68D20503D5022070472D
:10EE680001207047DA6812F0E00F01D007207047E0
:10EE7800DB6813F0020F14BF08200920704700BF99
:10EE8800003C024000B583B009238DF80730FFF736
:10EE9800D9FF8DF807009DF80730012BF7D09DF8B2
:10EEA8000700C0B203B05DF804FB00BF70B50646AA
:10EEB80059B301292FD002290CBF4FF400744FF425
:10EEC8004074FFF7DFFF092824D1144D2B6923F480
:10EED80040732B612969214329612B6923F0F803C9
:10EEE8002B612B6943F002031E432E612B6943F407
:10EEF80080332B61FFF7C6FF2B6923F002032B61D8
:10EF08002B6923F0F8032B6170BD0C46FFF7BAFF9D
:10EF18000928DAD070BD4FF48074F7E7003C02404E
:10EF280038B50446FFF7AEFF3CB1012C08D0022CDF
:10EF38000CBF4FF400744FF44074092804D038BD56
:10EF480009284FF48074FAD10B4D2B6923F44073D0
:10EF58002B612B691C432C612B6943F004032B6143
:10EF68002B6943F480332B61FFF78CFF2B6923F067
:10EF780004032B6138BD00BF003C0240FFF7D0BF3F
:10EF880038B50446FFF77EFF3CB1012C08D0022CAF
:10EF98000CBF4FF400744FF44074092804D038BDF6
:10EFA80009284FF48074FAD10B4D2B6923F4407370
:10EFB8002B612B691C432C612B6943F400432B61A3
:10EFC8002B6943F480332B61FFF75CFF2B6923F433
:10EFD80000432B6138BD00BF003C0240F8B5054630
:10EFE80016461F46FFF74EFF092800D0F8BD0B4C08
:10EFF800236923F440732361236943F44073236135
:10F00800236943F001032361C5E90067FFF73AFF6D
:10F01800236923F001032361F8BD00BF003C0240CF
:10F0280070B505460E46FFF72DFF092800D070BDC4
:10F038000A4C236923F440732361236943F4007362
:10F048002361236943F0010323612E60FFF71AFF50
:10F05800236923F00103236170BD00BF003C024017
:10F0680070B505460E46FFF70DFF092800D070BDA4
:10F078000A4C236923F440732361236943F48073A2
:10F088002361236943F0010323612E80FFF7FAFE11
:10F09800236923F00103236170BD00BF003C0240D7
:10F0A80070B505460E46FFF7EDFE092800D070BD85
:10F0B800094C236923F4407323612369236123697D
:10F0C80043F0010323612E70FFF7DCFE236923F070
:10F0D8000103236170BD00BF003C024038B50446FF
:10F0E8000D46FFF7CFFE092800D038BD2DB9064BD5
:10F0F8001A881443A4B21C8038BD034A13889BB2F3
:10F1080023EA0404148038BD163C024038B504468E
:10F118000D46FFF7B7FE092800D038BD2DB9064BBC
:10F128001A881443A4B21C8038BD034A13889BB2C2
:10F1380023EA0404148038BD1A3C024038B504465A
:10F148000D46FFF79FFE092800D038BD35B9064A9D
:10F1580013889BB223EA0404148038BD024B1A8832
:10F168001443A4B21C8038BD163C024038B504468E
:10F178000D46FFF787FE092800D038BD35B9064A85
:10F1880013889BB223EA0404148038BD024B1A8802
:10F198001443A4B21C8038BD1A3C024010B5044682
:10F1A800FFF770FE092804BF014B1C7010BD00BF9B
:10F1B800153C024008B5FFF765FE092802D1024B4D
:10F1C800FF221A7008BD00BF143C0240034A13789E
:10F1D80043F002031370FFF755BE00BF143C024012
:10F1E80008B501214FF48070FDF7AAFB00214FF408
:10F1F8008070BDE80840FDF7A3BB00BF42680B69FB
:10F20800F0B522F0407291F804E00E68CF688C687F
:10F218000C4D22F4807242EA0E2232434260866824
:10F228004A793B43354023432B4343EA42038360F7
:10F238000A7DC36A013AD2B223F4700343EA025347
:10F24800C362F0BDFDF7FFC0002301220275036011
:10F25800037143718360C360036170470749084ABB
:10F2680070B490E848004D688468C06833432A4009
:10F278001343234303434B6070BC70470023014092
:10F28800E030FCFF0023036043608360C360704785
:10F29800836819B923F001038360704743F00103C1
:10F2A80083607047436823F4400323F400731943D1
:10F2B8004160704741628262704700BF436823F033
:10F2C8001F03194341607047054A536818B923F46E
:10F2D80000035360704743F400035360704700BF56
:10F2E80000230140054A536818B923F4800353608A
:10F2F800704743F480035360704700BF0023014008
:10F30800092970B41CD9A1F10A0404EB4404C568A6
:10F318000726A640A34025EA06042343062AC3601D
:10F328001AD90C2A25D90D3A02EB8202C36A1F2486
:10F338009440914023EA04021143C16270BC7047B3
:10F3480001EB410604690725B540B34024EA0504EA
:10F358002343062A0361E4D8013A02EB8202436B95
:10F368001F249440914023EA04021143416370BC76
:10F378007047073A02EB8202036B1F2494409140C6
:10F3880023EA04021143016370BC7047836843F0A9
:10F3980080438360704700BF8068C0F38070704707
:10F3A800836819B923F480638360704743F48063EA
:10F3B80083607047836819B923F00203836070473C
:10F3C80043F00203836070474B1E416821F460419B
:10F3D80041EA433141607047436819B923F4006337
:10F3E8004360704743F4006343607047C06C80B269
:10F3F800704700BF014B1868704700BF08230140E1
:10F40800836819B923F480738360704743F4807369
:10F4180083607047836819B923F400738360704769
:10F4280043F4007383607047054A536818B923F49E
:10F4380000535360704743F400535360704700BF54
:10F4480000230140092970B41AD801EB4106046968
:10F458000725B540B34024EA050423430361836BC1
:10F468000232C3F30154121BD2B202EB82021F24F0
:10F47800944023EA040391401943816370BC7047A8
:10F48800A1F10A0404EB4404C5680726A640A3407A
:10F4980025EA06042343C360E1E700BF4B1E816BE6
:10F4A80021F4401141EA03518163704782B000237F
:10F4B80001930190019B19440191019B1A6002B0CC
:10F4C800704700BF836823F4702319438160704735
:10F4D800836823F44013194381607047836843F4B9
:10F4E80080038360704700BF8068C0F38050704716
:10F4F800436819B923F480634360704743F4806319
:10F5080043607047436819B923F4805343607047D8
:10F5180043F480534360704782B000230193019005
:10F52800019B283319440191019B186880B202B0ED
:10F53800704700BFC9B201238B4041681AB921EA5C
:10F548000303436070470B434360704703681942E5
:10F5580014BF012000207047C9430160704700BFF5
:10F568004268006810EA112007D00123C9B203FAE3
:10F5780001F1114214BF1846002070476FEA1121AB
:10F588000160704702683549002310B422F0010277
:10F59800212488420260036043608360C360036182
:10F5A800446149D02E4B984234D02E4B984237D0E4
:10F5B8002D4B98423AD02D4B984242D02C4B984232
:10F5C80043D02C4B98421CD02B4B98421DD02B4B30
:10F5D80098423ED02A4B98421CD02A4B98421FD0C2
:10F5E800294B984222D0294B98422AD0284B98423E
:10F5F8002BD0284B984204D0274B984205D010BCFA
:10F608007047264A43F8942CF9E74FF03D5243F8E7
:10F61800AC2CF4E74FF4746243F8202C10BC70470C
:10F628004FF4741243F8382C10BC70474FF07462D2
:10F6380043F8502C10BC7047194B10BC3D229A60FF
:10F648007047184A43F8642CD9E7174A43F87C2CCA
:10F65800D5E73D2243F8082CD1E700BF10600240EF
:10F6680028600240406002405860024070600240DA
:10F6780088600240A0600240B86002401064024006
:10F6880028640240406402405864024070640240AA
:10F6980088640240A0640240B864024000003D2033
:10F6A800006002403D000020400F00200B68CA693E
:10F6B800F0B4CE684D698C690F6A33432B432343FA
:10F6C8004E6A8D6A4C6B13433B4333438A6B07681E
:10F6D8000B4E2B4323433E4013433343CD6A036011
:10F6E80042690B6B0E694C6889682B4322F007024C
:10F6F8001343436146608460C160F0BC704700BF3B
:10F708003F801CF00023036043608360C360036193
:10F7180043618361C361036243628362C3620363BB
:10F7280043638363704700BF036819B923F001037B
:10F738000360704743F0010303607047036819B919
:10F7480023F400430360704743F4004303607047A9
:10F75800036819B923F020030360704743F02003BE
:10F768000360704741607047406880B2704700BFCF
:10F77800036822B923F4002303600161704743F44E
:10F788000023036001617047036819B923F48023DB
:10F798000360704743F48023036070470AB9C1606F
:10F7A80070470161704700BF0068C0F3C0407047F0
:10F7B800006800F001007047406900F038007047A9
:10F7C8000A4B0B4A10B40B4CA04294BF1846104683
:10F7D8008B004CBF4368036810BC21F0F02121F076
:10F7E8008211194214BF01200020704700600240B6
:10F7F800006402400F6402400B060CD54369AAB1AD
:10F8080043F08003802943610FD0036801F01E0193
:10F81800194301607047802907D0002AF5D1036891
:10F8280001F01E0123EA01010160704723F0800303
:10F8380080294361F3D1704730B4114B114D124AFE
:10F8480021F0F02424F0C314A84298BF1A469CB1B2
:10F85800006800EAD12000F01E0388004CBF506801
:10F86800106821F0F02121F08211084002D0181C04
:10F8780018BF012030BC7047436903F08003ECE7F0
:10F88800006002400F6402400064024010B4094B5B
:10F89800094C0A4AA04294BF1846104611F0005F6E
:10F8A80021F0F02121F0821114BFC160816010BCE9
:10F8B800704700BF006002400F64024000640240CD
:10F8C800FFF7E4BF30B40C4B0022072508240120C1
:10F8D80002211D705C7158709970DA701A719A71F2
:10F8E8001A755A759A75DA751A769860D9601A6118
:10F8F800DA611A6230BC704798820020F8B52D4B47
:10F908002D4C4FF4FA60012504214FF48057E62668
:10F91800586083F8365099751F629E824FF47A6753
:10F928004FF47A7632224FF4FA7064250521DA63AF
:10F938009863002248F2DC20A3F8465083F85C1054
:10F948001F604FF49671DF609E609E83C8254FF458
:10F95800803746F2A81618825882DA751A769A768F
:10F968009A84DA7683F8262083F8312083F83220C7
:10F9780083F833209A8683F8372083F85820DD836C
:10F98800A3F84850A3F84010A3F842102046A3F863
:10F998004410A3F85A1083F82F2083F8302083F8F6
:10F9A8005D201F66DE6406F099FD4FF6FF73238322
:10F9B800F8BD00BF308200200482002038B5FFF770
:10F9C800A3F902211020FFF771FA084A08481369C1
:10F9D8009568D46851791B0443EA056343EA042314
:10F9E8001943BDE83840FFF71BBB00BF98820020D1
:10F9F80010800008104B1B685A1E033210B402D83E
:10FA08000E4A12785AB10E4B082201245A7100206E
:10FA180002219C6010BC1861D960FFF7CFBF084A6B
:10FA28001C0EC3F30740C3F30721537194601061A0
:10FA3800D16010BC704700BF108000082C820020E5
:10FA4800988200202DE9F04F012185B0A04CDFF805
:10FA580088B2DFF888A2DFF888920846FCF704FF2E
:10FA680002A800250227FDF73BF9032220460D23B3
:10FA780002A94FF001088DF80C20019202938DF82D
:10FA88000D708DF80F50FDF7D7F843F60203029377
:10FA980020468DF80E508DF80D708DF80F508DF8AA
:10FAA8000C8002A92783FDF7C7F841463846FCF7C2
:10FAB800DBFE02A8FDF714F94FF4805302A958465B
:10FAC800029300938DF80C808DF80E508DF80D7010
:10FAD8008DF80F50FDF7B0F8009BABF8183002A86E
:10FAE80000934FF40056FDF7FBF8584602A98DF82D
:10FAF8000C508DF80D708DF80F500296FDF79CF89C
:10FB080041460420FCF7B0FE02A8FDF7E9F8019A87
:10FB18000292504602A98DF80C204FF4007B8DF814
:10FB28000D708DF80F50FDF787F8504602A9CDF8F3
:10FB380008B08DF80C808DF80E508DF80D708DF88A
:10FB48000F50FDF779F8AAF81AB041460820FCF7DB
:10FB58008BFE4FF4806B4022009B8DF80C804FF495
:10FB6800E2514FF4006A02918DF80E508DF80D7035
:10FB78008DF80F504846A9F81A2002A9A9F81AB01A
:10FB8800A9F81AA0A9F81A30FDF756F84AF2202366
:10FB9800484602A902938DF80C508DF80E508DF846
:10FBA8000D708DF80F50FDF747F841461020FCF70F
:10FBB8005BFE0822102340F61A4102918DF80C8052
:10FBC8008DF80E508DF80D708DF80F50A9F8187437
:10FBD800A9F81824A9F81834D9440DEB02014846AD
:10FBE800A9F818B0A9F818A0FDF726F84FF4607323
:10FBF800484602A902938DF80C508DF80E508DF8E6
:10FC08000D708DF80F50FDF717F841464FF0005072
:10FC1800FCF74EFE204602A902968DF80C808DF85E
:10FC28000E508DF80D708DF80F50FDF705F8204631
:10FC380002A94FF480438DF80D708DF80C508DF8A3
:10FC48000E508DF80F500293FCF7F6FF224630460F
:10FC58002C460A2156834FF47A7300BF013BFCD12E
:10FC6800136910835F0458BF01344FF47A7300BFDF
:10FC7800013BFCD113695B0448BF01350139E9D167
:10FC88000A2C144B1FD000221A700223002402A948
:10FC98004FF4C0420E488DF80C308DF80D300292AA
:10FCA8008DF80E408DF80F40FCF7C6FF22460D2157
:10FCB8000748FDF755F822460E210548FDF750F88C
:10FCC80005B0BDE8F08F0A2DDDD101221A70DCE7FE
:10FCD800000002402C82002000040240000802407C
:10FCE800000C024070B5614C614B94F8365083F8B3
:10FCF800245094E844001A6000225E6111461046C0
:10FD080007F056F8002210460A2107F051F8A37DA3
:10FD1800E27D1B2143EA0242002006F0DDFC0022BE
:10FD28001046172106F0D8FC40F69F7218210020D3
:10FD380006F0D2FC41F619121921002006F0CCFC7D
:10FD480007221A21002006F0C7FC4A4A0A2100208F
:10FD580006F0C2FC4FF010120421002006F0BCFC93
:10FD68004FF080520521002006F0B6FC0022104614
:10FD7800062106F0B1FC404A0721002006F0ACFC41
:10FD8800228A092142F08072002006F0A5FC628ACE
:10FD9800082142F08072002006F09EFC002005F049
:10FDA800EFFBA27E25211203002006F095FC226AB3
:10FDB8002621002006F090FCA28C292112040020A4
:10FDC80006F08AFCB4F84220B4F84010002006F08F
:10FDD8008FFFB4F84620B4F84410002006F098FFCE
:10FDE8000022B4F84810104606F098FFA37D226858
:10FDF800602102FB03F2002006F06EFC62682021FD
:10FE0800002006F069FC4FF4FA425D21002006F05C
:10FE180063FC47F6FF725C21002006F05DFCE26897
:10FE2800A18A002006F08EFD00221046242106F04B
:10FE380053FC002210464A2106F04EFC00221046D0
:10FE48004B2106F049FC00221046212106F044FC13
:10FE58004FF6FF722021002006F03EFC00221046DB
:10FE68004C21BDE8704006F037BC00BF308200204E
:10FE780004820020000100244E014E012DE9F04FBC
:10FE880001219DB04FF48000FCF7EEFC734E744CDA
:10FE9800DFF8D891734F01214FF48070FCF714FDFF
:10FEA80001214FF40070FCF70FFD3046FFF76AFBA5
:10FEB8000DA8FFF727FC4FF4806300254FF48072EC
:10FEC8004FF005080DA930464FF4006B4FF4005A67
:10FED8000E941393012401934FF400331692009269
:10FEE80017930F970D951095129518951A951B95C0
:10FEF800CDF84480CDF850B0CDF854A01994FFF750
:10FF0800D5FB21463046FFF70FFC4846FFF73AFB82
:10FF18000DA8FFF7F7FB019B009A139307F10C0E4E
:10FF28000226514B16920DA94FF4003248464FF065
:10FF38000077CDF83CE017920E930D971095129527
:10FF4800CDF850B0CDF854A0189519941A951B9572
:10FF58001196FFF7ABFB21464846FFF7E5FB07F193
:10FF680078574FF4004303A807F590370593039596
:10FF780004950695FFF772F907A8FFF765F9A9F543
:10FF8800A13907A93846A9F5A07907958DF8204029
:10FF98008DF8214009950A950B958DF83080FFF76B
:10FFA8002DF907A8FFF750F907A9484607958DF8D6
:10FFB80020408DF8214009950A950B958DF8306001
:10FFC800FFF71CF921463846FFF71AFA214648463A
:10FFD800FFF716FA2346224638460321FFF790F921
:10FFE8002346324631463846FFF78AF923462946E2
:08FFF80038460322FFF784F9EB
:020000040801F1
:100000002346384604220A21FFF77EF9234642465A
:1000100038460B21FFF778F9234622464846082147
:10002000FFF772F92346324648460921FFF76CF97B
:1000300021463846FFF7F2F921464846FFF7EEF928
:1000400021463846FFF728F921464846FFF724F9AC
:100050003846FFF79FF94846FFF79CF91DB0BDE809
:10006000F08F00BF106402404C200140D4000020FB
:100070004C21014040640240704700BF014B1022F8
:100080005A83704700100240014B10221A837047B8
:100090000010024010B9024B02225A83704700BF81
:1000A0000010024010B9024B02221A83704700BFB1
:1000B0000010024010B9024B08225A83704700BF5B
:1000C0000010024010B9024B08221A83704700BF8B
:1000D00000100240704700BF704700BF30B90449AC
:1000E000044B4FF48050022208831A83704700BFEC
:1000F000000402400000024060B9074B1B7C4BB972
:1001000003F18043054903F5013302204FF4805287
:1001100048835A83704700BFD4000020000002408B
:1001200050B9064B186910F4805006D0A3F58063CF
:100130001869C0F340007047002070470004024077
:1001400008B9014B19747047D4000020024B4FF4DA
:1001500000621A83704700BF00000240024B4FF458
:1001600000625A83704700BF00000240024A536990
:1001700083F400635361704700000240024B4FF468
:1001800080521A83704700BF00000240024B4FF4B8
:1001900080525A83704700BF00000240704700BF82
:1001A000704700BF704700BF704700BF704700BF77
:1001B00000207047024B4FF400721A83704700BF53
:1001C00000080240024B4FF400725A83704700BF90
:1001D00000080240014B00205B69704700080240A4
:1001E0000D4B10B40D4C19691A69236920692469F3
:1001F0009B00C4F3400403F004032343C1F3401104
:10020000C2F3403243EA011343EAC203C0F3800061
:1002100043EA400010BC7047000C0240000402405A
:1002200004281DD8DFE800F0080D121703000D4B5D
:10023000186900F0010070470B4B1869C0F340309B
:100240007047094B1869C0F340107047054B186997
:10025000C0F340007047034B1869C0F3800070473B
:100260000020704700040240000C024048B90129F8
:100270000AD00ED3022906D1084B186900F00100FC
:100280007047002070477047044B1869C0F3800026
:100290007047024B1869C0F34000704700040240E9
:1002A000032817D8DFE800F0110C07020A4B186981
:1002B000C0F300307047084B1869C0F3C020704786
:1002C000054B1869C0F380207047034B1869C0F3D1
:1002D0008010704700207047000C0240032807D8A8
:1002E000DFE800F0110C0702094B4FF480525A83EB
:1002F0007047074B4FF400625A837047044B4FF42A
:1003000080625A837047024B40225A83704700BF75
:10031000000C0240032807D8DFE800F0110C0702A8
:10032000094B4FF480521A837047074B4FF4006219
:100330001A837047044B4FF480621A837047024B54
:1003400040221A83704700BF000C024000B583B002
:10035000062842D8DFE800F011171D23292F0400DA
:100360001F4A10238DE80C000221012303220020E4
:1003700006F0DEFC03B05DF804FB1A4B988880B2EF
:1003800003B05DF804FB174BD88880B203B05DF86A
:1003900004FB144B188980B203B05DF804FB114BC9
:1003A000188880B203B05DF804FB0E4B588880B209
:1003B00003B05DF804FB00204FF6FF73009301903B
:1003C00001230322022106F0B3FCA0F51040883877
:1003D00020EAE07003B05DF804FB0020CAE700BF2C
:1003E0000000FFFFD4000020704700BF704700BF2F
:1003F000704700BF134B1B7813B370B41249134AF4
:100400004FF4805583B02E464FF4006400200E83D5
:100410004C830190019B934205D8019B01330193CA
:10042000019B9342F9D94D830C830190019B934228
:10043000EDD8019B01330193019B9342F9D9E6E783
:10044000704700BF2C820020000002403F420F0096
:1004500008B5FEF7D7FC40B1FEF772FC0020FEF7AE
:100460009DFCFEF7B7FEFEF77BFCFBF7EBFE62B6EA
:1004700008BD00BF034B10B9034ADA607047034A56
:10048000DA60704700ED00E00100FA050400FA05AB
:10049000684620F007018D4619B5124A124C1278B1
:1004A00023789A4218D86368104A0133636013684E
:1004B0003BB11368013B1360136813B90C4B012265
:1004C0001A7000F001FF00232370A3680133A360BA
:1004D000BDE819408546704723780133DBB22370AD
:1004E000F3E700BF34000020E8000020D0830020A4
:1004F000CC83002030B4084B084C41F26F70F025DB
:100500005860002184F82350072299606FF004009E
:100510001A6030BCFBF7B0BF10E000E000ED00E077
:10052000014B5868704700BFE8000020014B9868F5
:10053000704700BFE80000202DE9F04F8BB0044663
:1005400003A888461746FCF735FD601E072809D822
:10055000DFE810F0650168016A016C0161010800C3
:10056000540163010C2301210022ADF80C308DF8F9
:1005700010308DF811108DF80F20AD4BAD4D184691
:100580002B60FCF705FC01214FF00060FCF794F9AB
:1005900001210220FCF76CF900240223182201A992
:1005A000A5488DF808308DF8093001928DF80A4081
:1005B0008DF80B40FCF744FB0B2204219E48FCF70E
:1005C000D3FB0B2203219C48FCF7CEFB4FF0010A22
:1005D00003A928688DF80E408DF812408DF814405C
:1005E0008DF815408DF813A08DF816A08DF817A082
:1005F000FCF7FEFBB8F5006F80F2AE801FFA88F6BC
:100600000DF118094FF6FF737201494628688DF8FD
:1006100022408DF823408DF824A0ADF81A40ADF8A3
:1006200020408DF825A0ADF81820ADF81C30ADF8AD
:100630001E30FCF751FC1FB1B7F5006FC0F2C2804D
:10064000002301224FF6FF74494628688DF82220C6
:100650008DF82420ADF820208DF82330ADF8183027
:10066000ADF81A308DF82530ADF81C40ADF81E40BD
:10067000FCF732FCF6004FF0000B022301244FF68A
:10068000FF7A46F004064FEA683849462868ADF814
:100690001A60ADF818808DF822308DF823B0ADF8CF
:1006A00020B08DF824408DF82540ADF81CA0ADF8A1
:1006B0001EA0FCF711FC5F456BDDFB0043F004035B
:1006C0007F130322494628688DF823B08DF8244013
:1006D000ADF81CA0ADF81EA0ADF820408DF8254067
:1006E000ADF81A30ADF818708DF82220FCF7F4FB45
:1006F00001240727002668464B238DF800308DF82B
:1007000001708DF802608DF80340FBF769FE6846C2
:100710004C238DF800308DF801708DF802608DF853
:100720000340FBF75DFE4A2368468DF800308DF8E4
:1007300001708DF802608DF80340FBF751FE2246F0
:1007400028680221FCF720FE224628681021FCF7C9
:100750001BFE0BB0BDE8F08F0DF118094FF6FF73CB
:10076000494628688DF822408DF823408DF824A052
:10077000ADF81840ADF81A40ADF820408DF825408E
:10078000ADF81C30ADF81E301FFA88F6FCF7A4FB5C
:1007900051E703220423494628688DF823B08DF8D9
:1007A0002440ADF818B0ADF81CA0ADF81EA0ADF80F
:1007B00020408DF825B08DF82220ADF81A30FCF7D6
:1007C0008BFB95E7002101234FF6FF747A018DF82A
:1007D0002310ADF81A1028688DF8223049468DF89C
:1007E0002430ADF820308DF82530ADF81820ADF864
:1007F0001C40ADF81E40FCF76FFB3BE706200C21C8
:1008000001220023ADF80C008DF810108DF8112096
:100810008DF80F30B1E61820F1E70320EFE74FF431
:100820009670ECE79620EAE73C20E8E71E20E6E732
:10083000006C00403800002000040240F0B543780E
:1008400087B004463BB3042342688DF80C30002384
:1008500002920193A378DBB102238DF80D30234679
:100860000DF10F0213F8081B8DF80E1004F11000A3
:1008700013F8011B02F8011B8342F9D1184E01A99C
:100880003068FCF7FDFB04280BD0012007B0F0BD59
:100890008DF80D30E3E742688DF80C300293019239
:1008A000D8E7104F104B3D681B680135082D08BF75
:1008B00000259D4211D094E80F00D7F800E00B4CC2
:1008C00004EB0E1484E80F00012230683D601146ED
:1008D000FCF75AFD012007B0F0BD002007B0F0BDC5
:1008E00038000020C0820020C48200204C830020F9
:1008F00070B40F4B0F4C22681B689A4214D02268C8
:100900000D4B511C216003EB021305460FCB2668EB
:10091000082E85E80F0002D0012070BC704700232C
:100920002360012070BC7047002070BC704700BF7E
:1009300048830020BC820020C8820020684620F046
:1009400007018D4671B52A4C2A4B26681B68013673
:10095000082E08BF00269E4287B0274B35D0186866
:10096000264D01AA0021FCF71DFC9DF80C30042B3C
:10097000236833D005EB03130021019A59702368D3
:1009800005EB03135A609DF80D30022B236805EB2D
:1009900003130CBF012200229A7023689DF80E20D9
:1009A0001B010DF10F01EA540022236811F8010B1D
:1009B00005EB031313440132082A1872F5D126609F
:1009C00007B0BDE871408546704700211868FCF704
:1009D00037FC07B0BDE871408546704705EB03134F
:1009E0000121029A5970236805EB03135A60CAE784
:1009F00048830020BC82002038000020C8820020EC
:100A0000684620F007018D4671B52A4C2A4B2668AE
:100A10001B680136082E08BF00269E4287B0274B70
:100A200035D01868264D01AA0121FCF7BBFB9DF8C3
:100A30000C30042B236833D005EB03130021019AFB
:100A40005970236805EB03135A609DF80D30022B93
:100A5000236805EB03130CBF012200229A70236860
:100A60009DF80E201B010DF10F01EA5400222368AE
:100A700011F8010B05EB031313440132082A187215
:100A8000F5D1266007B0BDE8714085467047012169
:100A90001868FCF7D5FB07B0BDE871408546704784
:100AA00005EB03130121029A5970236805EB031328
:100AB0005A60CAE748830020BC820020380000202A
:100AC000C8820020684620F007018D4611B52E49E6
:100AD0002E4B0A681B689A4287B04DD00B682C4C8D
:100AE00004EB03135B7803F0FF02002B36D10B6895
:100AF0008DF80C2004EB031302925B6801930B68E2
:100B000004EB03139B7803F0FF02002B31D0022388
:100B10008DF80D300B681B010DF10F00E35C8DF8B3
:100B20000E3000220B6804EB0313134401321B7ACE
:100B300000F8013B082AF5D10B6801330B600B6804
:100B4000082B04BF00230B60124B01A91868FCF7A7
:100B500097FA07B0BDE81140854670470B6804EB73
:100B6000031304225B68029300238DF80C20019389
:100B7000C5E78DF80D20CDE7064B0022186801214E
:100B8000FCF702FCE5E700BFC4820020C082002021
:100B90004C83002038000020704700BF70B5064627
:100BA0000D46FFF76BFA0D4C02212046FCF7DAFEEA
:100BB0000028F9D0094831460446FCF799FE012186
:100BC0002046FCF7CFFE0028F9D00DB1FFF75CFA04
:100BD0000248FCF789FEC0B270BD00BF003401407E
:100BE00010B5002104460320FFF7D8FFC4F3072007
:100BF0000021FFF7D3FFE0B20021FFF7CFFF012173
:100C00000020BDE81040FFF7C9BF00BF38B504465B
:100C10000D4606200121FFF7C1FF00210520FFF747
:100C2000BDFF01210020FFF7B9FF8207F5D50021A4
:100C30000220FFF7B3FF0021C4F30720FFF7AEFF48
:100C40000021E0B2FFF7AAFF28460121FFF7A6FF27
:100C500000210520FFF7A2FF01210020FFF79EFFE2
:100C6000C307F5D438BD00BF38B54FF40065012186
:100C70000620FFF793FF00210520FFF78FFF0121DA
:100C80000020FFF78BFF8207F5D500210220FFF738
:100C900085FF0021C5F30720FFF780FF0021E8B2A0
:100CA000FFF77CFF0024A4F13F01B1FA81F149096B
:100CB00000200134FFF772FF402CF4D10021052001
:100CC000FFF76CFF01210020FFF768FFC307F5D491
:100CD0004035B5F5804FCAD138BD00BFF0B5C0EB87
:100CE000C00083B000F500640D4603200021FFF72B
:100CF00055FFC4F307200021FFF750FFE0B20021A9
:100D0000FFF74CFF00210846FFF748FF0021064689
:100D10000846FFF743FF002104460846FFF73EFF61
:100D2000002107460846FFF739FF00218DF804002F
:100D30000846FFF733FF00218DF805000846FFF74E
:100D40002DFF01218DF806000020FFF727FF8DF809
:100D500000608DF80140BDF800202B888DF8070059
:100D60009A4202D0002003B0F0BDAB78BB42F9D16B
:100D70006B680198C01AB0FA80F04009F3E700BF31
:100D800038B50D46C0EBC00404F500600978FFF7E4
:100D90003DFF697804F60100FFF738FFA97804F6F3
:100DA0000200FFF733FF297904F60300FFF72EFF57
:100DB000697904F60400FFF729FFA97904F6050014
:100DC000FFF724FFE97904F60600BDE83840FFF795
:100DD0001DBF00BFC0EBC00038B50C4600F5006574
:100DE00000210320FFF7DAFE0021C5F30720FFF7FB
:100DF000D5FE0021E8B2FFF7D1FE00210846FFF73B
:100E0000CDFE002120700846FFF7C8FE002160706B
:100E10000846FFF7C3FE0021A0700846FFF7BEFE9C
:100E2000002120710846FFF7B9FE002160710846D5
:100E3000FFF7B4FE0121A0710020FFF7AFFEE071C3
:100E400038BD00BF2DE9F04105460E4606200121C0
:100E50001746FFF7A3FE00210520FFF79FFE0121A3
:100E60000020FFF79BFE8207F5D500210220FFF747
:100E700095FE0021C5F30720FFF790FE0021E8B2A0
:100E8000FFF78CFE002F40D0013E002407F1FF3811
:100E900009E0A8EB0401B1FA81F14909FFF77EFEF0
:100EA0000134A74231D00135AB0616F8010FF0D15D
:100EB0000121FFF773FEA045F2D900210520FFF7BD
:100EC0006DFE01210020FFF769FEC107F5D4012165
:100ED0000620FFF763FE00210520FFF75FFE0121DA
:100EE0000020FFF75BFE8207F5D500210220FFF707
:100EF00055FE0021C5F30720FFF750FE0134002105
:100F0000E8B2FFF74BFEA742CDD100210520FFF745
:100F100045FE01210020FFF741FEC307F5D4BDE8DF
:100F2000F08100BFF8B504460D46032000211646A7
:100F3000FFF734FE0021C4F30720FFF72FFEE0B2D5
:100F40000021FFF72BFE76B1013D771E0024391BEF
:100F5000B1FA81F149090020FFF720FE0134A642D1
:100F600005F8010FF3D1F8BD10B540F2FF70FFF79F
:100F700037FE062802D1164B1B78ABB1002140F298
:100F8000FF70FFF743FEFFF76FFE24221149002098
:100F9000FFF758FF104940206422FFF753FF062156
:100FA00040F2FF70FFF732FE0A4C24222146002057
:100FB000FFF7B8FF607806F001F840206422064988
:100FC000FFF7B0FF6078BDE8104006F003B800BF3F
:100FD0002C8200209882002030820020F0B55E4BE9
:100FE0005E4C89B0074618462360FDF719FC0121C5
:100FF0002020FBF76DFC01210420FBF739FC0226C1
:101000000025402302A9564802938DF80C608DF804
:101010000D608DF80E508DF80F50FBF711FE8023F8
:1010200002A94F4802938DF80C608DF80E508DF890
:101030000D608DF80F50FBF703FE0822062148488B
:10104000FBF792FE464808220721FBF78DFE04A815
:10105000FDF7CEFC0B2F07D8DFE807F006585C60E1
:1010600064686C7074787B554FF41653049304A92C
:101070002068FDF75BFC002505230126472201A817
:101080008DF805308DF804208DF806508DF8076036
:10109000FBF7A6F9206840F2FF31FDF7C9FD2A46AB
:1010A00020682821FDF7A2FD3246206840F2277112
:1010B000FDF79CFD3246206840F22661FDF796FD63
:1010C0003246206840F22551FDF790FD2A462068FF
:1010D00040F22441FDF78AFD2A46206840F6460189
:1010E000FDF784FD2A46206840F66A11FDF77EFD73
:1010F0002A4620686021FDF779FD31462068FDF71A
:101100009BFC09B0F0BD174B0493B0E74FF461535B
:101110000493ACE74FF496430493A8E74FF4E143FC
:101120000493A4E74FF416430493A0E74FF46143FC
:1011300004939CE74FF49633049398E74FF4E1331C
:10114000049394E74FF46133049390E7064B0493C0
:101150008DE7064B04938AE7001401403C00002011
:101160000008024040420F0090D0030020A1070079
:10117000684620F007018D4631B5294D286803885F
:10118000990627D403881A0611D5264C226B636B67
:101190009A423BD0FFF70EF8636B28685A1C234431
:1011A000626393F838308380636B202B35D00388DB
:1011B0005B0603D4BDE831408546704740F22661A6
:1011C000FDF75EFD174B5A6B1B6B9A42F2D1FEF78F
:1011D000F9FFEFE7FEF7FEFFA8B9124A2868136887
:1011E00051680133202B08BF00238B4205D01168C2
:1011F00084881144E4B20C7213600B4B0A2119600D
:10120000936AD362BEE728688388BBE7002240F276
:101210002771FDF7EBFC2868C9E700236363C6E785
:101220003C000020F4000020D083002010B40C4CBF
:10123000236B626B0133202B08BF002393420DD038
:10124000226B22440146074882F838100068236365
:10125000012240F2277110BCFDF7C8BC10BC7047DA
:10126000F40000203C0000200A4B59681A689142A3
:101270000ED05A68511C1A445960117A5A6801708C
:10128000202A01D00120704700225A6001207047B7
:1012900000207047F4000020014B9862704700BFA7
:1012A000F4000020044A137803F0FF0013B1002378
:1012B00013700120704700BFCC830020014BD86A17
:1012C000704700BFF4000020034BDA6A12B1DA6AFB
:1012D000013ADA62704700BFF400002010B4054BF9
:1012E00005491C684C604A78887810BC052101F0DB
:1012F0006DB900BF3C840020DC830020094B9A7844
:1013000042B95B78142B09D80749084A096842F8A2
:1013100023107047064B04221A707047044B0322B7
:101320001A707047DC8300203C840020E883002092
:10133000B0840020034A044B12685A60092002F06E
:101340006DBC00BF3C840020DC830020054B0649B7
:101350005A7801208242087002D1044A5B68136007
:10136000704700BFDC830020A2840020708400202E
:10137000014B02221A707047A2840020F0B4084F7B
:10138000084E094D094C0A480A490B4A00233B7094
:1013900033602B60237003600B601360F0BC7047F8
:1013A000A284002070840020A8840020D88300201C
:1013B0003C840020BC840020E4830020014B0022F8
:1013C0001A707047A284002028494B78032B32D82A
:1013D000DFE803F026110602254B0A225A60704707
:1013E0002449254B00220A6003F1280143F8042B0D
:1013F0008B42FBD1704770B41E4E306870B11E4AEC
:101400004D681368AB421ED01146002303E051F82B
:10141000044FAC4218D001338342F8D170BC7047FE
:10142000144A1368092B0AD81348496840F8231056
:101430000133136070470E4B03221A7070470C4B38
:1014400009221A7070470023411E8B420BD200F113
:101450008040013802EB800002EB83035A6843F8B6
:10146000042B8342FAD13160D8E700BFDC8300202F
:10147000B0840020A4840020748400202B4A537878
:10148000092B50D8DFE803F010161C232A33393F0C
:101490004505274953680B60264A002B3ED0136848
:1014A00023F0080313607047214953680A68134406
:1014B0000B60F1E71E4952680B689B1A0B60EBE763
:1014C0001B4952680B6803FB02F30B60E4E7184901
:1014D00052680B6893FBF2F30B60DDE71449526826
:1014E000086890FBF2F302FB13030B60D4E710498A
:1014F00053680A6813400B60CEE70D4953680A68C9
:1015000013430B60C8E70A4953680A6853400B60ED
:10151000C2E7074A1368DB431360BDE7136843F073
:10152000080313607047024B1B68B5E7DC8300209B
:101530003C840020E4830020354B5B780A2B63D881
:10154000DFE803F0141B222A323C434A51580600BC
:101550003049314A086813680B6010602F4A002B2D
:101560004DD0136823F0080313607047294A2A4BB3
:1015700011681B680B441360F0E7264A264B11687C
:101580001B68CB1A1360E9E7224A234913680968EC
:1015900001FB03F31360E1E71E4A1F4B11681B6850
:1015A00091FBF3F31360D9E71A4A1B4913680968E2
:1015B00093FBF1F001FB10331360CFE7154A164B94
:1015C00011681B680B401360C8E7124A124B116880
:1015D0001B680B431360C1E70E4A0F4B11681B6871
:1015E0004B401360BAE70C490A4B0A681B68D243A8
:1015F0000A60B3E7074B084A1B681360AEE713683D
:1016000043F0080313607047024B1B68A6E700BF56
:10161000DC8300203C840020BC840020E483002084
:10162000164B5B78052B09D8DFE803F0090F151B73
:101630002103134A136823F4807313607047104A20
:10164000136803F00F03136070470D4A136823F00B
:101650001003136070470A4A136823F020031360D5
:101660007047074A136823F0400313607047044A29
:10167000136823F080031360704700BFDC830020F1
:10168000E4830020104A114B11685B68104A8B42BA
:10169000136809DA23F0030343F00403136079B1FC
:1016A00023F00803136070470BBF23F0060323F0F9
:1016B000050343F0010343F0020313600029EFD157
:1016C00043F00803136070473C840020DC83002053
:1016D000E4830020830703D5054B08221A70704766
:1016E0000449054A4968054B116004221A70704785
:1016F000B0840020DC830020D4830020A28400205A
:10170000014B00221A707047A284002008B50C4BD0
:10171000196821F07F4121F0FF0121B95A6840F298
:10172000D2439A4200D008BD40F2FF70FFF76EFA34
:10173000FFF79AFA0120BDE80840FEF79BBE00BF04
:10174000DC830020104B5B78032B07D8DFE803F025
:10175000190C07020D4A0E4B12685A6070470D4A69
:101760000B4B12685A6070470B4B1A680B48084BBA
:101770000B49007809781A71120A5A71D871997157
:101780007047084BF1E700BFDC830020BC840020D9
:10179000B08400203C84002070840020A2840020BB
:1017A000D8830020D4830020014B02221A70704796
:1017B00040840020024A034B52681A60704700BF01
:1017C000DC83002070840020284A53780C2B0CD82E
:1017D000DFE803F0071E141923282E33383D424753
:1017E0000C00234B1B68180704D47047204B1B6860
:1017F000DB05FAD51F4B52681A6070471C4B1B68FB
:10180000DB07F7D470471A4B1B68D807F2D570472F
:10181000174B1B681907EDD57047154B1B68590707
:10182000E8D47047124B1B6813F0050FE2D17047E4
:101830000F4B1B689B07DDD470470D4B1B68980747
:10184000D8D170470A4B1B68D906D3D47047084BD0
:101850001B689B06CED47047054B1B685806C9D43D
:101860007047034B1B681906C4D47047DC83002003
:10187000E483002070840020084A1368072B0BD8EB
:1018800030B40749074C0D6844F8235030BC064873
:101890000133406808601360704700BFA8840020CF
:1018A0007084002050840020DC830020F0B5204BA1
:1018B000204A5B68204D0124B3F5006F83B014709B
:1018C000287001DC0C400AD01C4B0021DA1D03F803
:1018D000011B9342FBD12B782B7203B0F0BD18464D
:1018E0006946FFF777FA9DF801309DF805009DF8ED
:1018F00000209DF802E09DF807709DF80660AB702F
:101900009DF80430A871EB716A70214685F803E0F8
:101910002F716E71AB1C05F1080001E013F8012B6B
:101920001144C9B283422972F8D103B0F0BD00BF9F
:10193000DC83002040840020448400204584002073
:10194000054A136833B1013B0448054950F82300A8
:1019500013600860704700BFA884002050840020F6
:101960007084002030B5134D6C7883B084B1012CA5
:1019700004D0114B03221A7003B030BDAB782A2B70
:10198000F7D1291D042240F2FB70FFF75BFAF3E761
:1019900004220DEB020140F2FB70FFF7C3FA6A6804
:1019A000019B9A42044B06BF01225A605C6003B05F
:1019B00030BD00BFDC830020B0840020014B00223A
:1019C0001A707047A284002070B5114E114D306816
:1019D000114C2A786B686270B0F5006F636005D9AE
:1019E0000E4A002107231170237070BD2946FFF7AE
:1019F000C7F929463068FFF771F928B133686522C5
:101A000001332270336070BD0723237070BD00BFA7
:101A1000D4830020DC830020B0840020A284002036
:101A200070B52A4E2A4C33786BB963685A1C2BD098
:101A300003EB8303274A5B001360FEF771FD264A20
:101A4000012310603370657885B1012D0DD1A07828
:101A500000F000F910F4804530D11E4C2368DBB94A
:101A60001E4A1368013B136070BD70BDFEF758FD40
:101A7000194B184A1B681268C01A0028B8BF4042A8
:101A80009042EDD9357070BD154B124A1B6803EBBF
:101A900083035B001360D0E7FEF742FD0E4B226824
:101AA0001B68C31A002BB8BF5B429342D8D90D4ABA
:101AB0003570136843F01003136070BD094A136852
:101AC000002123F010033170136070BDD883002013
:101AD000DC830020C08800209C84002070840020CB
:101AE0003C840020E4830020094B9A783AB95A7864
:101AF000142A08D807495B6841F822307047064B22
:101B000004221A707047044B03221A70704700BFFA
:101B1000DC830020E8830020B0840020144B9A78F6
:101B20005AB95A78142A19D81249134B51F822205D
:101B30005A60124A12783AB970470F4B04221A7051
:101B40000E4A1278002AF7D00D4A5B6813600D4ADE
:101B500043B1136823F0080313607047064B032258
:101B60001A70EDE7136843F008031360704700BF75
:101B7000DC830020E8830020B0840020A1840020C2
:101B80003C840020E48300200A4B987838B910B5D3
:101B90005C78142C07D9084B03221A7010BD064B31
:101BA00004221A70704703F0EBF9044B43F8240049
:101BB00010BD00BFDC830020B0840020E88300203B
:101BC000034A52F82030194342F82010704700BFF2
:101BD000C4880020024A136818431060704700BF91
:101BE000C4880020034A52F8203023EA010142F859
:101BF00020107047C4880020024A136823EA0000BE
:101C000010607047C48800203AB9074A52F8203063
:101C100023EA010142F820107047034A52F82030AD
:101C2000194342F820107047C4880020034B53F832
:101C300020300B4214BF012000207047C4880020D0
:101C4000034A52F8203023F0610342F820307047F5
:101C5000C48800200246054B53F8200053F8221098
:101C600021F0610143F82210704700BFC4880020B2
:101C70000246064B53F8200053F8221021F0610170
:101C800000F06B0043F82210704700BFC4880020AA
:101C90002DE9F041454C2378656882B00022013B74
:101CA0000192042B7FD8DFE803F01E432640030097
:101CB00001AAE9B2280E00F0B7FB01982569217D41
:101CC000E268237A2840C8409042CCBF0124002417
:101CD0008CBF01210021062B63D8DFE803F05A53A3
:101CE0004C4740392E0001ABEAB2280E062100F025
:101CF0006DFC0198E2E72E0EC5F307273946304602
:101D000004F0CCFCC5F3074280463946304604F067
:101D1000E7FCE9B2304604F0C1FC42460190394686
:101D2000304604F0DDFC0198C8E7FEF7F9FBC5E793
:101D3000E9B2280E04F0B2FCC0E71D4B9A788A4243
:101D400001D002221A705C70997002B0BDE8F08177
:101D5000174B9D78002DF6D09042F2D9F3E7144B43
:101D60009D78002DEFD19042EBD8ECE7104B5A78DC
:101D7000A242E6D1E7E70E4B5D78002DE3D090421A
:101D8000DFDDE0E70A4B5D78002DDCD19042DADD43
:101D9000D7E7074B02221A705C70997002B0BDE859
:101DA000F081034BCFE7002088E700BFE8880020E0
:101DB0004C010020024B1B78012B00D0704767E7D5
:101DC0004C0100202DE9F04F3F4CE37885B04BB13A
:101DD0002378012B27D03D4E63683268013393424C
:101DE000636002D205B0BDE8F08F23780027022B94
:101DF0006760F7D1364D05F120092B781BB90835FE
:101E0000A945FAD1EEE7D4F80880039708F101025A
:101E1000013BA260D5F804A0042B53D8DFE803F0FF
:101E2000473F1F1B0600FFF733FFD4E703AA5FFA03
:101E30008AF14FEA1A6000F0F7FAA2680398736813
:101E400004EB88089342C8F80C00D8D8032200237A
:101E50002270E370C6E7FEF763FBA268EFE74FEA84
:101E60001A6BCAF3072319465846019304F016FC6F
:101E7000019B00901946CAF30742584604F030FC13
:101E80005FFA8AF1584604F009FC019B009A03901E
:101E90001946584604F024FCA2680398CFE75FFA7D
:101EA0008AF14FEA1A6004F0F9FBA268C7E75FFA0B
:101EB0008AF203AB4FEA1A60062100F087FBA268A2
:101EC0000398BCE70020BAE74C0100204000002046
:101ED000C88800201348144903460022F0B403F8D0
:101EE000082BC27043F8042F8B42FBD10F49104BD3
:101EF000104C114F826001264FF400554FF0FF3017
:101F00000A75C7F84429266065601A705A601A720B
:101F1000DA601A745A611A76DA610A704A600861E6
:101F2000F0BC70474C01002054810020E88800205C
:101F3000C88800204000002014780020034BB0F532
:101F4000005F28BF4FF400505860704740000020E9
:101F5000014B1860704700BF4000002005280FD8D3
:101F60000B4B1B7863B930B40A4A12F8334002EBCA
:101F7000C3053CB10133042BF7D1002030BC7047BE
:101F80000020704702F833006960012030BC7047C0
:101F90004C010020C88800200528034607D8054AC0
:101FA000127822B9044A0120137051607047002052
:101FB000704700BF4C010020E8880020014B1861E9
:101FC00019757047E888002006281AD82DE9F043D3
:101FD000354D2B7883B083B9344C237800B193B15D
:101FE0000022013B2072E16001926668042B58D800
:101FF000DFE803F0293238530D00002003B0BDE8BC
:10200000F08300207047184603B0BDE8F083F1B2BA
:1020100001AA300E00F008FAE16801982269237DD8
:102020001040D8408842C8BF01224FF00100D8BFFD
:1020300000228CBF012300236A70AB702870E87007
:1020400003B0BDE8F083062101ABF2B2300E00F020
:10205000BDFAE1680198E1E7F1B2300E04F01EFB31
:10206000E168DBE7370EC6F307284146384604F03F
:1020700015FBC6F3074281464146384604F030FB63
:10208000F1B2384604F00AFB414601904A46384610
:1020900004F026FBE1680198C0E7FEF741FAE16829
:1020A000BCE70020BAE700BF4C010020E888002010
:1020B000014B1878704700BF4C010020054B9A680F
:1020C000824205D903EB80030120DB680B60704777
:1020D000002070474C01002003280ED8DFE800F0F4
:1020E000020A070404207047054B9868704742F2C3
:1020F000107070474FF4005070474FF0FF3070473A
:102100004C010020FF2809D0032805D8064B13F8FE
:1021100030300B700120704700207047034B1B7854
:102120000B700120704700BFC8880020E88800209D
:10213000FF280AD0032806D8064B03EBC003012072
:102140005B680B60704700207047034B5B680B6057
:1021500001207047C8880020E8880020F0B50121E0
:1021600089B0254E254F4FF40050FAF7B1FB0024FB
:10217000642302250121102001938DF808508DF869
:1021800009508DF80A408DF80B40FAF771FB304684
:1021900001A9FAF755FD294630460522FAF7E4FD74
:1021A000052230461146FAF7DFFD304605220621AA
:1021B000FAF7DAFD01264FF4827E4FF400722023F5
:1021C000384603A9ADF80EE0ADF81620ADF818308A
:1021D000ADF81250ADF80C40ADF81040ADF81A4013
:1021E000ADF81C40ADF81460FBF738FA31463846BC
:1021F000FBF7F2FA09B0F0BD0010024000340140D4
:10220000F8B50E4615460746FDF744FF0D4C022172
:102210002046FBF7A7FB0028F9D00A4831460446C0
:10222000FBF766FB01212046FBF79CFB0028F9D059
:102230000448FBF759FBC4B215B13846FDF732FF2D
:102240002046F8BD00340140704700BFF8B50E4687
:1022500015460746FDF72EFF0D4C02212046FBF7E1
:1022600081FB0028F9D00A4831460446FBF740FBC1
:1022700001212046FBF776FB0028F9D00448FBF744
:1022800033FBC4B215B13846FDF71CFF2046F8BD3C
:102290000034014010B50020FDF72EFF1A4B00243A
:1022A000204683F8584004F013F872B64FF0FF321E
:1022B0002046830003F1604303F5614301300828A1
:1022C000C3F88020C3F88021F3D100230F481946BA
:1022D000C2180133F02B82F80013F9D10C4B0D48D2
:1022E00019600021FDF724FA0A48FDF74FF9FCF7C1
:1022F0007BFFFCF721FA0848FBF75CFB0020BDE8F8
:102300001040FEF7B7B800BF3082002000E100E0C7
:1023100010E000E01064024000000140FFF770BFD1
:10232000FFF794BF10B5144604F0B8F9206010BD53
:1023300004F0D6B910B5144604F01CFD206010BDA1
:1023400004F03ABDF8B51649164E174D174C18480B
:10235000184B00220A7032602A602260026003F586
:10236000806143F8042F8B42FBD1134F3B7E73B93E
:10237000124E40F21A7440F2FA75A4F21A71042255
:10238000204631441444FEF7CDFDAC42F5D17B7DAF
:1023900013B90B4A1370F8BD094B01221A70F8BD2E
:1023A000D8830020708400203C840020BC8400205E
:1023B000E4830020BC84002098820020C084002098
:1023C000A2840020024B59689878494202F0B4BFB9
:1023D000DC830020024B5968987802F0ADBF00BF43
:1023E000DC830020024B0021987802F0A5BF00BFDB
:1023F000DC8300200A4B9A7832B95A7862B1012AFC
:1024000006D1596802F0ECBF064B04221A707047DF
:10241000044B03221A707047596802F0B1BF00BF25
:10242000DC830020B084002030B5044683B015461C
:10243000392900F2C780DFE801F0C1BCB7B3ADA60F
:10244000A09B968E888172C5C5C5C5C5C5C5C5C5C5
:10245000C5C5C5C5C5C5C5C5C5C5C5C5C5C5C5C52C
:10246000C5C5C5C5C5C5C5C5C5C5C5C56C664D4BC6
:1024700049472B1D18226F21204604F031F92046D0
:102480006E2104F00BF964232860184603B030BDB8
:102490000621204604F06EF920224E21204604F049
:1024A0001FF92A684D21204604F01AF921224E21F5
:1024B000204604F015F9204601224D2104F010F9C0
:1024C0006423184603B030BD1522D4E70521E0E7A8
:1024D0001622D0E7042104F04DF920224E21204697
:1024E00004F0FEF82A684D21204604F0F9F8212274
:1024F0004E21204604F0F4F820460A224D2104F033
:10250000EFF86423C1E7242104F0C8F864232860AD
:10251000BBE71268242104F0E3F86423B5E702A9BD
:10252000002341F8043DFFF703FE019B2B600028C8
:1025300014BF64230923184603B030BD02A9002349
:1025400041F8043DFFF7DEFDEFE71068FFF7C4FD3B
:102550006423286099E702A9002341F8043D10682C
:10256000FFF7ACFDE1E7FFF7A3FD642328608CE7EC
:102570001168FFF729FD642387E701461068FFF71C
:102580001DFD642381E71168FFF706FD002897D140
:1025900009237AE71168FFF7E1FC002890D1F7E7FB
:1025A0001068FFF7D5FC8BE71368002B88D0042355
:1025B0006BE71068FFF7C2FC642366E7FFF78AFC4D
:1025C000642362E7032360E7704700BF30B51C4611
:1025D00083B0002840F00581FF2A00F23486DFE84E
:1025E00012F03001DF03DA03D003BD030104EF036F
:1025F00032063206320613047E034F033D032B03DB
:10260000190310030703FE023206F00240043206EB
:10261000320632062E0432063206320632069E0496
:10262000250473036A033206320632063206320686
:10263000320681046103B403A2038C0490033206C2
:102640003206320632066B0447047604A802D2052D
:10265000C805150632063206320632063206320642
:102660003206320632063206320632063206B50528
:10267000E804D604C404B2043F05350528062B053A
:10268000E002CC02F8053206320632063206320685
:10269000320632063206BA027C056905560549053E
:1026A0003206320632063206320602068F05A205CF
:1026B000A90419050705E505FA049B0279026702DA
:1026C000320632063206320632063206320632064A
:1026D000320632063206320632063206320632063A
:1026E000320632063206320632063206320632062A
:1026F000320632063206320632065502CD01BB01E1
:102700003206B2013206320632063206320632068E
:1027100032063206320632063206AA013206320686
:1027200032063206320632063206320632063206E9
:1027300032063206320632063206320632063206D9
:1027400032063206320632063206320632063206C9
:1027500032063206320632063206320632063206B9
:1027600032063206320632063206320632063206A9
:102770003206320632063206320632063206320699
:10278000320632060802F6011A0212013B02360234
:1027900032063206320632063206A3019C013206A8
:1027A00032063206320632063206320632064D0252
:1027B000DF01EE01320632063206320632063206FA
:1027C000320693018A0166017801540181015D019D
:1027D0006F014B01420132063206320632063206E2
:1027E0003701042306290BD1C04A127842B122686E
:1027F000BF490A60FAB1BF490A6822F008020A60BC
:10280000184603B030BD06291ED1BB4D95F82F30B8
:1028100013F0020001F07C8101210020FDF726FD6C
:10282000012800F009810022B04B22601B785BB1C7
:10283000AF4964230A60AF490A6842F008020A609F
:10284000DEE7062900F0BF876423184603B030BDD9
:10285000052900F050850629F6D10020FDF760FC1F
:1028600020606423C0E7052900F0C1870629EBD169
:1028700004F0DAFB2060F4E7052900F0D087062990
:10288000E2D104F0C5FB2060EBE7052900F0BB872F
:102890000629D9D104F08CFB2060E2E7052900F07D
:1028A000CA870629D0D104F09BFB2060D9E705290F
:1028B00000F0A3870629C7D104F062FB2060D0E7AF
:1028C000052900F0B2870629BED104F095FB2060EF
:1028D000C7E7052900F09D870629B5D104F05CFB08
:1028E0002060BEE7052900F0AC870629ACD104F0D2
:1028F0006BFB2060B5E7052900F047870629A3D1C7
:1029000004F032FB2060ACE7052900F06A87062955
:102910009AD104F01DFB2060A3E7062994D102F0B0
:102920002FFA642320605FE706298DD102F022FA96
:102930006423206058E7062986D10020FFF78AF932
:102940006423206050E706297FF47EAF002003F067
:1029500019FD6423206047E7052900F080860629D9
:1029600000F00386072901F0158008297FF46CAF79
:10297000012262499C20FEF7D5FA65E7052900F09F
:102980006486062900F0CD85072901F05A800829C0
:102990007FF45AAF02225A499A20FEF7C3FA53E74E
:1029A00006297FF451AF1821002003F077FE83B28F
:1029B0000133544A92FBF3F26423226014E70629A0
:1029C0007FF442AF04F0B0FA642320600CE70529DD
:1029D00000F07C84062900F0FF85072901F084803F
:1029E00008297FF431AF012247496F20FEF79AFA98
:1029F0002AE7052900F08884062900F0D7850729F1
:102A000001F0B78008297FF41FAF01223F497020F1
:102A1000FEF788FA18E706297FF416AF364D95F8C9
:102A20002F3013F0010101F0668000210846FDF708
:102A30001DFC01287FF4F7AE01222C4B22601B788D
:102A4000002B3FF401AF2A4964230A60D3E605292D
:102A500000F0BD846423C5E606297FF4F5AE264D5B
:102A600095F82F3013F0040001F0008002210020BF
:102A7000FDF7FCFB01287FF4D6AEDDE706297FF4E5
:102A8000E3AE04F0F5F964232060ADE6052900F01B
:102A9000F985062900F05085072900F0828708296A
:102AA0007FF4D2AE01221A499820FEF73BFACBE61A
:102AB000052900F02386062900F05285072900F039
:102AC000838708297FF4C0AE042212498C20FEF7C8
:102AD00029FAB9E606297FF4B7AE7621002003F083
:102AE000DDFD00F00700206064237DE6A184002066
:102AF0003C840020E4830020308200208C8200206F
:102B00008A82002000E1F5055F82002060820020BB
:102B1000888200207C820020052900F06D8406292F
:102B20007FF492AED74B93F83730C3F38003236022
:102B300097E6052900F0DA84062900F07285072956
:102B400000F0BD8708297FF47FAE0422CE497C20A7
:102B5000FEF7E8F978E6052900F0C183062900F0C0
:102B60006487072900F0378708297FF46DAE0122BA
:102B7000C6497120FEF7D6F966E606297FF464AEF1
:102B80004FF0FF3300200093019002236D226C214F
:102B900004F0CEF8BB4A6423927D90FBF2F22260EF
:102BA00022E606297FF450AE4FF0FF330020009359
:102BB000019001236D226C2104F0BAF86423206097
:102BC00012E606297FF440AE002002F0D7FC05464D
:102BD000002002F0C7FC2B1A1BB2236041E6062935
:102BE0007FF432AE002002F0C3FC64232060FBE5DA
:102BF00006297FF429AE002002F0C0FC6423206087
:102C0000F2E506297FF420AE002002F0ABFC64233D
:102C10002060E9E5052900F08185062900F04A8653
:102C2000072900F0338608297FF40EAE0122984967
:102C30005820FEF777F907E6052900F038850629C0
:102C400000F05F86072900F0418608297FF4FCAD7B
:102C5000012290495720FEF765F9F5E5052900F0B6
:102C60006585062900F02C86072900F0368608299C
:102C70007FF4EAAD012288499D20FEF753F9E3E590
:102C8000052900F03D84062900F07584072900F02D
:102C9000858708297FF4D8AD042280494820FEF7B3
:102CA00041F9D1E506297FF4CFAD002002F0C0F84C
:102CB0006423206098E506297FF4C6AD002002F069
:102CC00083F8642320608FE5052900F064850629D8
:102CD0007FF4BAAD002002F07DF82060C1E505293F
:102CE00000F09883062900F01986072900F00F8666
:102CF00008297FF4A9AD042269494C20FEF712F996
:102D0000A2E5052900F0CB84062900F01B840729E1
:102D100000F06F8608297FF497AD01226149762083
:102D2000FEF700F990E5052900F0E084062900F09F
:102D30001284072900F0648608297FF485AD0422F7
:102D400050494020FEF7EEF87EE506297FF47CAD81
:102D5000002002F073F86423206045E506297FF423
:102D600073AD1221002003F099FC001400F5F94323
:102D70007F334FF6FE12934288BF00202060642309
:102D800032E506297FF460AD1321002003F086FCB4
:102D900000B2206065E506297FF456AD1221F4E704
:102DA00006297FF451AD00221046032103F098FC60
:102DB0000221002003F072FC000C2060642313E564
:102DC000052900F0F884062900F06E85072900F037
:102DD000648508297FF438AD022233495220FEF77A
:102DE000A1F831E5052900F0DE84062900F03685DA
:102DF000072900F02C8508297FF426AD02222B49F3
:102E00005020FEF78FF81FE5052900F00F830629F3
:102E100000F0BA85072900F0FA8508297FF414AD7F
:102E2000012223495620FEF77DF80DE506297FF49F
:102E30000BAD002001F0C2FF64232060D4E405291B
:102E400000F04584062900F05685072900F04C85DE
:102E500008297FF4F9AC012216495920FEF762F8DF
:102E6000F2E406297FF4F0AC002002F081FBAEE62C
:102E700006297FF4E9AC002002F060F864232060AA
:102E8000B2E400BF308200206C820020618200200A
:102E900048820020478200208D8200203882002056
:102EA0003C82002066820020428200204082002076
:102EB0004682002049820020052900F03F8406292F
:102EC0007FF4C2AC002002F01BF82060C9E40529A1
:102ED00000F0058406297FF4B7AC002002F050F81A
:102EE0002060BEE4052900F0EA8306297FF4ACAC3B
:102EF000002001F097FF2060B3E4052900F0AE81C7
:102F0000062900F01483072900F0888508297FF43A
:102F10009BAC0422DB494420FEF704F894E4052925
:102F200000F0138406297FF48FAC002001F078FFB5
:102F3000206096E406297FF487ACD34B93F82630C3
:102F40002360642350E4052900F00E82062900F076
:102F50001D83072900F01B8608297FF475AC022227
:102F6000CA498820FDF7DEFF6EE4052900F069827A
:102F7000062900F03F83072900F0ED8508297FF43A
:102F800063AC0222C2498620FDF7CCFF5CE4052930
:102F900000F06982062900F03383072900F0E285FA
:102FA00008297FF451AC0222BA498420FDF7BAFF08
:102FB0004AE4052900F08882062900F02C830729BD
:102FC00000F06F8508297FF43FAC0222B2498220CD
:102FD000FDF7A8FF38E4052900F0AB8106297FF44E
:102FE00033ACA94B93F8373003F00103236038E486
:102FF000052900F0AC81062900F0DE82072900F0E7
:10300000BF8508297FF420AC0222A4495E20FDF789
:1030100089FF19E4052900F02B81062900F0D782E9
:10302000072900F0308508297FF40EAC02229C4964
:103030005C20FDF777FF07E406297FF405AC002349
:103040004FF0FF32019318460092B3E506297FF452
:10305000FBAB4FF0FF330020009301900523A9E55F
:1030600006297FF4F1AB4FF0FF330020009301906D
:1030700004239FE506297FF4E7AB7621002003F0C7
:103080000DFBC0F3022020606423FFF7ADBB0529D0
:1030900000F0EF82062900F03E82072900F0D88474
:1030A00008297FF4D1AB02227E497420FDF73AFF54
:1030B000FFF7CABB052900F0E881062900F0488423
:1030C000072900F0CC8408297FF4BEAB01227649A1
:1030D0007320FDF727FFFFF7B7BB052900F01D811F
:1030E000062900F06584072900F07C8408297FF414
:1030F000ABAB01226D497120FDF714FFFFF7A4BBB4
:10310000052900F02A83062900F0B583072900F07D
:10311000AB8308297FF498AB012265495A20FDF75B
:1031200001FFFFF791BB052900F09080062900F010
:103130004982072900F0088508297FF485AB012220
:103140005C495B20FDF7EEFEFFF77EBB052900F032
:10315000A981062900F01482072900F0BE840829FD
:103160007FF472AB022254498020FDF7DBFEFFF7AB
:103170006BBB06297FF468AB002002F07DFA642364
:103180002060FFF731BB052900F02C81062900F0F3
:103190003D82072900F08C8408297FF455AB042276
:1031A00046497820FDF7BEFEFFF74EBB052900F02B
:1031B000FB80062900F0F081072900F087840829A8
:1031C0007FF442AB02223E496420FDF7ABFEFFF7DD
:1031D0003BBB06297FF438AB4FF0FF330020009350
:1031E00001900323E6E4052900F0CF80062900F0D2
:1031F000BB83072900F0C18308297FF425AB042293
:1032000030496020FDF78EFEFFF71EBB052900F058
:10321000D580062900F0C581072900F03B840829E4
:103220007FF412AB04222849A020FDF77BFEFFF7B4
:103230000BBB06297FF408AB00204FF0FF320B4692
:1032400001900092A2E40323FFF7CCBA2268022A7D
:103250000BD80D496423CA76FFF7D2BA2168002043
:1032600001F01AFE00287FF4EFAA0423FFF7C8BA82
:10327000226842F210739A42F7D8034964238A8382
:10328000FFF7BEBA3482002030820020788200200E
:103290007682002074820020728200204E820020FC
:1032A0004C82002064820020638200206282002021
:1032B0004A8200204B820020708200206882002019
:1032C0005482002050820020908200202268072A29
:1032D000CBD8C449642381F82F20FFF791BA236823
:1032E000012BC2D8BF4A002082F8313002F04CF9DD
:1032F0006423FFF785BA2068002840F09781FCF727
:10330000FBFE6423FFF77CBA2368B64A03F0070389
:1033100082F830306423FFF773BA2368012BA4D8F6
:10332000B04A002082F8323002F02EF96423FFF711
:1033300067BA2368002B40F0F883AA4A92F8373026
:1033400023F0010382F837306423FFF759BA22686B
:10335000A54902F5433303F5A0738B4285D8A149F3
:103360006423CA83FFF74CBA2368B3F5004FBFF458
:103370007CAF9C4C9BB200221946A4F84830104602
:1033800003F0D0FC6423FFF73BBA2368B3F1807FDE
:10339000BFF46BAF934C1A4623622621002003F042
:1033A0009FF96423FFF72CBA2268B2F5803FBFF47F
:1033B0005CAF8C4964238A84FFF722BA2268052A0D
:1033C0007FF753AF874964230A66FFF719BA21686C
:1033D00007293FF64AAFC9B20020FDF705F864237C
:1033E000FFF70EBA2268814B9A423FF63EAF7D4905
:1033F00064238A63FFF704BA23687A4A002B00F03B
:103400001B8192F8373043F0040382F8373064238D
:10341000FFF7F6B9216844F2506399423FF625AFB1
:10342000002002F01BF86423FFF7EAB921684B1E65
:10343000FE2B3FF61AAF002002F002F86423FFF7DC
:10344000DFB92368B3F5004FBFF40FAF65489BB2F7
:10345000A0F846301A46B0F84410002003F05CFC97
:103460006423FFF7CDB92368B3F5004FBFF4FDAE79
:103470005C489BB2A0F844301946B0F846200020C2
:1034800003F04AFC6423FFF7BBB92368012B3FF626
:10349000ECAE544A002082F8333002F075F8642311
:1034A000FFF7AEB92368B3F5004FBFF4DEAE4D4869
:1034B0009BB2A0F840301946B0F84220002003F03B
:1034C0001BFC6423FFF79CB92368B3F5004FBFF4DE
:1034D000CCAE44489BB2A0F842301A46B0F8401037
:1034E000002003F009FC6423FFF78AB92268404BEF
:1034F0009A423FF6BAAE3B496423CA63FFF780B9EC
:10350000226844F250639A423FF6AFAE35496423D5
:103510008A60FFF775B9334BB3F934302360FFF796
:10352000A0B9304BB3F85A302360FFF79AB92D4B4E
:103530005B682360FFF795B92A4B93F858302360F6
:10354000FFF78FB9274B93F83630003318BF0123AC
:103550002360FFF786B9234B1B682360FFF781B90F
:10356000204BDB6C2360FFF77CB91E4B93F85C307B
:103570002360FFF776B91B4B9B682360FFF771B997
:10358000184BB3F840302360FFF76BB9154BB3F815
:1035900048302360FFF765B9124B9B8C2360FFF71F
:1035A00060B9104B1B6E2360FFF75BB90D4B93F8AE
:1035B00030302360FFF755B90A4BB3F91E30236052
:1035C000FFF74FB9074BDB7E2360FFF74AB9054B86
:1035D0009B8B2360FFF745B9024B93F82F30236094
:1035E000FFF73FB930820020801A0600400D03002B
:1035F000A0860100CC4BB3F846302360FFF731B909
:10360000C94BB3F844302360FFF72BB9C64B9B6B13
:103610002360FFF726B9C44BB3F842302360FFF7AD
:1036200020B9C14BDB6B2360FFF71BB90020FCF70F
:1036300055FD6423FFF7E4B892F8373023F0040314
:1036400082F837306423FFF7DBB8B74B2268A3F862
:103650005A20002002F03CFE6423FFF7D1B8B24BA1
:10366000226883F85C20002002F032FE6423FFF71A
:10367000C7B8AD4B22689A86002001F085FF64230D
:10368000FFF7BEB82368A84A003318BF012382F8A9
:103690005830002002F01CFE6423FFF7B1B8216807
:1036A000002001F013FC00287FF4CEA8DDE521788E
:1036B000002001F0E9FE00287FF4C6A8D5E52168C6
:1036C000002001F039FE00287FF4BEA8CDE5217866
:1036D000002001F031FF00287FF4B6A8C5E521687D
:1036E000002001F06BFC6423FFF78AB821680020FA
:1036F00001F0B2FB00287FF4A7A8B6E58A4B226848
:10370000DA642368894A92FBF3F29200013A1821A5
:10371000002002F0E5FF6423FFF772B82178002053
:1037200001F0E6FE00287FF48FA89EE521780020B6
:1037300001F0C6FE00287FF487A896E521680020E6
:1037400001F01EFE6423FFF75BB82168002001F042
:103750009FFD00287FF478A887E52368724C00332A
:1037600018BF01232521A376002002F097FFA37E36
:103770001B0303F4805320F480521A4325210020B8
:1037800002F0AEFF6423FFF73BB8206803F0E6FBCE
:103790006423FFF735B82168002001F0A7FD002859
:1037A0007FF452A861E52168002002F055FD002851
:1037B0007FF44AA859E52168002002F06DFD002839
:1037C0007FF442A851E500221046032102F088FF51
:1037D0000221002002F062FF80B220606423FFF724
:1037E00003B8206803F0AEFB6423FFF709B8206834
:1037F00003F014FC6423FFF703B8206803F0BAFB5E
:103800006423FEF7FDBF206803F0CCFB6423FEF7C2
:10381000F7BF206803F0BAFB6423FEF7F1BF20680E
:1038200003F0F0FB6423FEF7EBBF206803F0DEFB40
:103830006423FEF7E5BF206803F0CCFB6423FEF7AA
:10384000DFBF206803F0BAFB6423FEF7D9BF022272
:1038500037495020FDF7F6FAFEF7F6BF002002F0D8
:10386000EFFC2060FEF7FDBF012232495A20FDF730
:10387000E9FAFEF7E9BF2521002002F00FFF2A4BED
:10388000C0F3003098762060FEF7EBBF01222A4992
:103890005820FDF7D7FAFEF7D7BF0222274952205A
:1038A000FDF7D0FAFEF7D0BF002002F0E9FC20605F
:1038B000FEF7D7BF002001F037FE2060FEF7D1BF32
:1038C000002001F00BFE2060FEF7CBBF01221C4957
:1038D0005720FDF7B7FAFEF7B7BF012219499D201F
:1038E000FDF7B0FAFEF7B0BF012217495920FDF7E6
:1038F000A9FAFEF7A9BF002001F02CFE2060FEF718
:10390000B0BF002001F0D0FD2060FEF7AABF042266
:103910000E494C20FDF796FAFEF796BF002001F005
:10392000ABFD2060FEF79DBF3082002040787D0116
:10393000408200204A8200204882002042820020EB
:10394000478200208D820020498200203C82002096
:103950003321002002F0A2FE944BC0F3002083F834
:1039600033002060FEF77DBF2621002002F096FE86
:103970008E4B18622060FEF774BF04228C496020D1
:10398000FDF760FAFEF760BF002001F04DFD2060FA
:10399000FEF767BF022287499C20FDF753FAFEF726
:1039A00053BF012284499820FDF74CFAFEF74CBF23
:1039B0003321002002F072FE7C4BC0F3003083F80C
:1039C00032002060FEF74DBF04227C498C20FDF7B9
:1039D00039FAFEF739BF012279497120FDF732FA31
:1039E000FEF732BF012277497220FDF72BFAFEF76E
:1039F0002BBF012274497620FDF724FAFEF724BF7D
:103A000004226A494020FDF71DFAFEF71DBF01227E
:103A10006E495620FDF716FAFEF716BF04226C49D0
:103A20004420FDF70FFAFEF70FBF3321002002F00C
:103A300035FE5E4B00F0010283F831202260FEF774
:103A400010BF022263499A20FDF7FCF9FEF7FCBE85
:103A5000022261497420FDF7F5F9FEF7F5BE012257
:103A60005E497320FDF7EEF9FEF7EEBE0221FCF78A
:103A7000FDFB00283EF4E0AF95F82F305B077EF5A4
:103A8000D2AEFEF7F3BF022255495C20FDF7DAF90A
:103A9000FEF7DABE04225349A020FDF7D3F9FEF762
:103AA000D3BE022250498220FDF7CCF9FEF7CCBEEE
:103AB00004224E497820FDF7C5F9FEF7C5BE042261
:103AC0004B497C20FDF7BEF9FEF7BEBE02224949F4
:103AD0006420FDF7B7F9FEF7B7BE02224649802001
:103AE000FDF7B0F9FEF7B0BE012244496F20FDF7A3
:103AF000A9F9FEF7A9BE0846FCF7B8FB00283EF47A
:103B00009BAF95F82F30D9073EF58FAFFEF78BBEF0
:103B10000121FCF7ABFB00283EF48EAF95F82F3067
:103B20009A077EF580AEFEF777BE00221046282168
:103B300002F0D6FD1D4A92F8373043F0010382F8B7
:103B400037306423FEF75CBE01222D495B20FDF770
:103B500079F9FEF779BE02222A498620FDF772F92B
:103B6000FEF772BE022228498420FDF76BF9FEF7AA
:103B70006BBE012225497020FDF764F9FEF764BE93
:103B8000022223495E20FDF75DF9FEF75DBE0222A9
:103B900020498820FDF756F9FEF756BE04221E493B
:103BA0004820FDF74FF9FEF74FBE00BF30820020DE
:103BB000508200208C820020888200207C8200209D
:103BC00061820020628200206682002046820020FE
:103BD000348200208A8200206482002063820020D8
:103BE0004C82002090820020728200206882002097
:103BF0006C82002054820020708200205F820020AE
:103C00004B82002076820020748200206082002097
:103C10004E820020788200203882002038B5874C00
:103C2000A378002B40F0C7806378403BBF2B00F2A5
:103C30004482DFE813F00B02750118024202DF0133
:103C4000FA018401B4014202A3014202C2016601E9
:103C50005701420242024202440135011E01420262
:103C60001101420242024202420242024202420266
:103C70004202420242024202420242024202420224
:103C80004202420242024202420242024202420214
:103C90004202420242024202420242024202420204
:103CA00042024202420242024202420242024202F4
:103CB000420242024202290296013102D401EF017E
:103CC00042024202420242024202420242024202D4
:103CD00042024202420242024202420242024202C4
:103CE00042024202420242024202420242024202B4
:103CF00042024202420242024202420242024202A4
:103D00004202420242024202420242024202420293
:103D10004202420242024202420242024202420283
:103D20004202420242024202420242024202420273
:103D30004202420242024202420242024202420263
:103D40004202420242024202420242024202420253
:103D50004202420242024202420242024202420243
:103D60004202420242024202420242024202420233
:103D70004202420242024202420242024202420223
:103D80004202420242024202420242024202420213
:103D9000420242024202FC0042024202420242024B
:103DA00042024202420242024202420242024202F3
:103DB0004202FC003902022B11D0214B04221A705E
:103DC0000A280BD11F4A127842B11F4A5B68136060
:103DD0001E4AEBB1136823F00803136038BD657801
:103DE000372D1AD80A2800F06C8109281AD00B2820
:103DF00000F0D8810C28F1D11549042240F21A7044
:103E000001EB850102FB0500BDE83840FDF78AB8EB
:103E1000136843F00803136038BD0A2800F051818D
:103E20000928DBD10A4B626843F8252038BD0A28EF
:103E3000D4D1084A024B12785A60C3E7DC830020D1
:103E4000B0840020A18400203C840020E483002072
:103E5000C0840020948200200A2800F04A810928AA
:103E6000BCD16368012B40F2B681B74B04221A70B3
:103E700038BD0A2800F078810928AFD1B34D6368B6
:103E80002946042241F8103F1020FCF7DBFFFBF726
:103E900099FD2A69A9686879BDE83840FCF74CBBF0
:103EA0000A2800F02181092898D1A849636841F8BF
:103EB000203F04222020BDE83840FCF7C3BF0A2879
:103EC00000F00D81092889D1A04D21792B7DDA07D9
:103ED00002D5CB0740F1898129751420BDE838400F
:103EE000FCF794BE0A2800F0448109287FF476AFDD
:103EF000964A2379537519461520BDE83840FCF7DA
:103F000085BE0A2800F0168109287FF467AF8F4A22
:103F10002379937019460220BDE83840FCF776BE3D
:103F20000A2800F0308109287FF458AF874A2379A6
:103F3000137019460020BDE83840FCF767BE0A2818
:103F400000F0E68009287FF449AF8049636841F8B2
:103F50000C3F04220C20FCF775FFBDE83840FBF74E
:103F600031BD0A287FF43AAF794A774B1278A2F133
:103F70000402B2FA82F252095A6023E70A2800F0DA
:103F8000D18009287FF42AAF2179002940F01D81D2
:103F90006E4BD9751720BDE83840FCF737BE0A28AC
:103FA00000F0EC8009287FF419AF684D636829465A
:103FB000042241F8083F082067E70A2800F09E80A5
:103FC00009287FF40BAF2379604C19460320E37076
:103FD000FCF71CFEE078BDE83840FDF75DB90A2823
:103FE00000F0DB8009287FF4F9AE574A594B52683C
:103FF0001A6038BD0A2800F0868009287FF4EEAEEA
:104000005249636841F81C3F04221C20BDE8384037
:10401000FCF718BF0A2800F0BB8009287FF4DEAE49
:10402000494A4D4B52681A6038BD0A2800F0878013
:1040300009287FF4D3AE2379444A194605205371E9
:10404000FCF7E4FDBDE83840FBF7BCBC0A2800F0F3
:10405000B58009287FF4C2AE217940F2FF70BDE837
:104060003840FCF7D3BD0A2857D009287FF4B6AEF4
:104070002379364C1846637002F0B8FF617801204E
:10408000BDE83840FCF7C2BD0A287FF4A7AE304A2D
:104090002D4B12785A6095E60A287FF49FAE2F4A7E
:1040A000294B12685A608DE60A2810D009287FF43F
:1040B00095AE2B4B22791A7038BD234B03221A7010
:1040C0007EE6284A204B52F825205A607AE6244A98
:1040D0001D4B1278003218BF01225A6072E61B4A4B
:1040E000194B127D5A606DE6184A174B126A5A60D6
:1040F00068E6164A144B127E5A6063E6134A124B66
:10410000D2785A605EE6114A0F4BD2695A6059E67E
:104110000E4A0D4BD2685A6054E60C4A0A4B52784C
:104120005A604FE6094A084BD27D003218BF01227F
:104130005A6047E6054A044B92785A6042E6034AC1
:10414000014B52795A603DE6B084002098820020ED
:10415000A2840020048900200089002070840020AF
:10416000A0840020C0840020224A234B12695A6098
:1041700028E6204A204B527D5A6023E61D4A1E4BFA
:1041800092685A601EE61B4A1B4B12785A6019E669
:104190001A4A194B12685A6014E6194A164B1268EB
:1041A0005A600FE61749042240F21A7001EB8501AC
:1041B00002FB0500BDE83840FCF744BE40F2FF704A
:1041C000FCF70EFD0C4B5860FCE50A4A0A4B012136
:1041D000D1755960DEE60749237901F8183F0122BD
:1041E0001820BDE83840FCF72DBEFCF73DFD2179D5
:1041F00072E600BF98820020B08400200089002071
:1042000004890020C0840020074B9A78022A04D138
:104210005A6858782AB9FCF761B8044B04221A701E
:104220007047FCF777B800BFDC830020B084002023
:1042300010B51E4CA378012B27D01ED3022B06D01D
:104240001B4B04221A7022780F2A08D010BD607808
:10425000FCF726F82278164B0F2A5860F6D1154A3B
:104260001278002AF2D0144A5B681360134A93B1A3
:10427000136823F00803136010BD6078FF280FD087
:10428000FBF7CEFF0A4B5860DDE76078FCF75EF87D
:10429000074B5860D7E7136843F00803136010BD5D
:1042A000FBF79EFF024B5860CDE700BFDC83002088
:1042B000B0840020A18400203C840020E4830020FE
:1042C00010B4224B5B789BB92149224B0868224AE3
:1042D00022499B7802F8013B0124431E0C700730F1
:1042E00013F8011F02F8011B8342F9D110BC70477B
:1042F000012B0FD0052B15D0062B1DD0072BF5D188
:10430000174B0A240B200C210D22DC719871597176
:104310001A71EBE7124A0621512053719071D17145
:104320001171E3E70E4B142412200B211D22DC71C6
:10433000987159711A71D9E7094B002411200E2187
:104340002622DC71987159711A71CFE7DC83002045
:104350003000002098820020448400204084002007
:10436000B084002070B5054D054C29786E686170E9
:1043700064224B1E82B02270666003E0DC83002062
:10438000B0840020FE2B00F2C181DFE813F0BA01F7
:10439000B501B001AC01A101A101A101A1019D01E3
:1043A0009D019D019D01BF019A019701BF01BF01C0
:1043B000BF01940191018E018B0188018501BF012C
:1043C000BF0182017F01BF017C0179017601730188
:1043D00070016D016A01BF01BF016701BF01BF012B
:1043E000BF01BF01BF01BF01BF01BF01BF01BF01CD
:1043F000BF01BF01BF01BF01BF01BF01BF01BF01BD
:10440000BF01BF01BF01BF01BF01BF010901BF0162
:10441000BF01BF01BF01BF01BF01BF01BF01BF019C
:10442000BF01BF01BF01BF01BF01BF01BF01BF018C
:10443000BF01BF01BF01BF01BF01BF01BF01BF017C
:10444000BF01BF01BF01BF01BF01BF01BF01BF016C
:10445000BF01BF01BF01BF01BF01BF01BF01BF015C
:10446000BF01BF01BF01BF01BF01BF01BF01BF014C
:10447000BF01BF01BF01BF01BF01BF01BF01BF013C
:10448000BF01BF01BF01BF01BF01BF0164016101E5
:104490005E015B0156014C014601430140013D01B3
:1044A000BF01BF013A0137012C01BF01BF01BF01AC
:1044B000FF00BF012101BF01BF01BF01BF01BF015B
:1044C000BF01BF01BF01BF01BF01BF01BF01BF01EC
:1044D000BF01BF01BF01BF01BF01BF01BF01BF01DC
:1044E000BF01BF01BF01BF01BF01BF01BF01BF01CC
:1044F000BF01BF01BF01BF01BF01BF01BF01BF01BC
:10450000BF01BF01BF01BF01BF01BF01BF01BF01AB
:10451000BF01BF01BF01BF01BF01BF01BF01BF019B
:10452000BF01BF01BF01BF01BF01BF01BF01BF018B
:10453000BF01BF01BF01BF01BF01BF01BF01BF017B
:10454000BF01BF01BF01BF01BF01BF01BF01BF016B
:10455000BF01BF01BF01BF01BF01BF01BF01BF015B
:10456000BF01BF01BF01BF01BF01BF01BF01BF014B
:104570001301BF01BF01BF01BF01BF01BF01BF01E7
:10458000BF01BF01BF01BF01BF010B01A878002817
:1045900000F0C480012803D13246697802F00CFC97
:1045A00002B070BD40F2D2439E42F9D15E4B01226F
:1045B0001A70F5E72B685D4A23F07F4323F0FF0371
:1045C0009342EDD15A4B9E42EAD1FDF763FEE7E7F5
:1045D000A878002800F09D800128E1D1697802F0D8
:1045E000C9FB6060DCE702AA697842F8046DA8782C
:1045F000FDF71AFF019B20706360D1E7FCF7E4FE32
:10460000CEE7FDF7AFF9CBE7FDF780F8C8E7FFF796
:1046100057FEC5E7FDF796F8C2E7464B197D987837
:10462000FDF744F9BCE7FDF76BF80020FBF756FDFA
:104630000021084600F02CFEB2E73E4B187DFDF746
:1046400049F8ADE7FCF79AFEAAE7FCF791FEA7E769
:10465000FCF77CFEA4E7FCF7B1FEA1E7FCF74EFEF9
:104660009EE7FCF7DDFF9BE7FCF764FE98E7FCF7AD
:1046700035FE95E7FCF760FF92E7FDF785FA8FE7D7
:10468000FDF74CFA8CE7FDF72FFA89E7FDF796F96D
:1046900086E7FDF7C5F983E7FDF752F980E7FDF7F7
:1046A000EBF87DE7FDF786F87AE7FDF78DF877E719
:1046B000FCF7E8FF74E7FCF7E1FE71E7FFF7B8FDF0
:1046C0006EE7FFF7A1FD6BE70846FFF7A7FA67E77C
:1046D00002AB6A7843F8046DA878FDF777FF019B79
:1046E000207063605CE7A878FDF784FE58E7A8783F
:1046F000002100F021FE53E77142A87800F01CFE73
:104700004EE73146A87800F017FE49E702232370F0
:1047100046E7697801F0C2FF606041E73246697898
:1047200001F0DEFF3CE700BF5C81002000819200C9
:10473000D6C5B4A3988200202DE9F043BE4B1B7868
:1047400089B053B1BD4B1B78063BDBB2192B54D853
:10475000BB4A22FA03F3D9074FD5BA4CBA4D637856
:104760005A1E012A40F2E38004AE032B00F0998028
:10477000042B00F092812278002363702B70002AB2
:1047800044D13046FCF7B4F80646002847D10DF175
:104790000F00FCF769FDAD4D002840F094802B78A8
:1047A0005A1E012A40F27081042B62786ED0082ACA
:1047B00040F2B480FFF7D6FD6378092B1AD12B782D
:1047C000022B00F05581A24B186898B12B78012B71
:1047D00010D1A04BA04A1C6813689C4218BF00234C
:1047E00005D1A2E152F8041F8C4200F09E810133F2
:1047F0009842F7D809B0BDE8F083924C924D2278E8
:10480000002304AE63702B70002ABAD00120FBF79E
:1048100031FE3046FCF76CF806460028B7D002F0AF
:104820002DFB864B9DF810209DF818501D709DF8AB
:1048300019009DF81D5058705D71072A9DF81A10D7
:104840009DF81B709DF81C609DF81E007F4D9970AF
:10485000DF719E7118710CBF0123022363702B78E6
:104860009DF81110A1705A1E012A40F2E080052B1C
:1048700000F0DD80794B01221A700DF10F00FCF77A
:10488000F3FCF8B92B786278042B90D16B4B93F939
:104890000030002B8BDB082A40F2ED80FDF794F806
:1048A000A8E72B78002B00F08480012B7FF463AF06
:1048B0006B4F07F1090817F8010FFCF7B7FC4745E4
:1048C000F9D158E70126FCF7EDFC002861D1E27828
:1048D0009DF80F10531CDBB22244092BE3701171B9
:1048E0005CD1E070019002F0C9FA5E4B22795B78EE
:1048F00001989342C6D15C4BD91D01E013F8012BFE
:1049000010448B42C0B2F9D1237B834200F0108166
:104910002A7804239A426370B8D01A4640F25113A1
:10492000D340DA077FF546AF09B0BDE8F0834D49C3
:104930002A78CE680596012BA0788DF811000CBF5F
:104940000726082600238DF810608DF812304ABB28
:10495000464B89681F785E78D8798DF818108DF8E5
:104960001F2099795A791B798DF819708DF81A6082
:104970008DF81B008DF81C108DF81D208DF81E3051
:1049800004AE3046FBF75AFF00283FF433AF63789C
:10499000EBE601229DF80F30E2702371002E7FF4C8
:1049A00071AFFCE6012A00F0A580022AE8D104AE2E
:1049B000E1E6DFF8B090DFF8B48099F8020099F8EA
:1049C000017098F8002098F801300744174498F8CF
:1049D00007201F4498F80630174498F805201F4414
:1049E00098F8043017441F44FCF720FC99F80100A4
:1049F000FCF71CFC98F80000FCF718FC98F8010084
:104A0000FCF714FC98F80700FCF710FC98F8060077
:104A1000FCF70CFC98F80500FCF708FCFFB298F8CE
:104A20000400FCF703FC3846FCF700FCA3E60B4B44
:104A300000221A7021E700BFA0840020DC83002040
:104A4000110200025C81002040840020A28400202A
:104A5000A48400207084002074840020A18400209D
:104A6000438400209882002061810020B0840020CF
:104A700005232B70A7E640F25113D340DB077FF5E7
:104A80000DAF09B0BDE8F0833C4B1868B0F5006F7E
:104A90003BD900232B70627889E6DFF8FC90384F11
:104AA00099F8020099F80180002301223A707B7086
:104AB0007B608044FCF7BAFB99F80100FCF7B6FB79
:104AC0003878FCF7B3FB7878FCF7B0FBF879FCF7A3
:104AD000ADFBB879FCF7AAFB08F101087879FCF77F
:104AE000A5FB5FFA88F83879FCF7A0FB4046FCF795
:104AF0009DFB40E6234B06AA03F1080013F8011BB7
:104B000002F8011B8342F9D13AE7421C1E491A60A0
:104B1000FCF760F91D4A01210923117063702B789D
:104B2000042B7FF447AE6278B0E605232B7061E674
:104B3000154B6179A279267A19705A70A17AE27AB6
:104B4000E779607ADE7159711A719F709871FBF77D
:104B5000E7FC0F4A2B7810600E4E5A1E00200321EE
:104B6000012A3070617005D9052B03D0074B012253
:104B70001A70D4E7054B00221A70D0E77084002029
:104B8000B084002045840020DC830020A184002024
:104B9000AC840020B884002098820020F0B5024642
:104BA000264B007992F801C092F802E0D678D871CD
:104BB00050799871224C9E700D469179597194E804
:104BC0000300D7791F4A83F800C083B083F801E05F
:104BD0001F71002313708DE80300FFF7C3FB1A4B0E
:104BE0001B786E46B3B1012B05D096E8030084E82C
:104BF000030003B0F0BD154A6B1E073512F8011B08
:104C000003F8011FAB42F9D196E8030084E80300E2
:104C100003B0F0BD2B706B7063782278AA70EB70D4
:104C2000E3792B71A3796B716379AB7196E803001B
:104C30002379EB7184E8030003B0F0BDDC8300202E
:104C4000B0840020A18400204084002045840020FE
:104C500000224FF0FF31930003F1604303F56143FD
:104C60000132082AC3F88010C3F88011F3D1002361
:104C700004481946C2180133F02B82F80013F9D109
:104C8000704700BF00E100E0074A0849136823F0BD
:104C90007F4323F0FF038B4200D070475268044BE0
:104CA0009A42FAD1FDF7F6BADC8300200081920027
:104CB000D6C5B4A3044B5A6840F2D2439A4202D1FB
:104CC000024B01221A707047DC8300205C810020B7
:104CD000F8B5184F184E194D19491A4A1A4B1B4866
:104CE000DFF888E0DFF888C000243C603460184FAB
:104CF000184E2C600C60146017491C60174D184A40
:104D00000460FF233C60337016482B700026002798
:104D10000B708CF80040CEF80040C2E9006702F04A
:104D20006BF8114B20461C804FF48071BDE8F840B1
:104D3000FCF746BF28890020148900200C89002038
:104D400018890020608900206489002030890020B3
:104D500038890020348900201089002068890020CB
:104D600020890020408900206C81002008890020D3
:104D70002C890020014B5868704700BF6C810020CF
:104D8000014B9868704700BF6C81002010B5044645
:104D9000FBF7C6F900B110BD2046FCF769FF0028FB
:104DA000F9D14FF480712046FCF740FF0028F2D182
:104DB0002046BDE81040FBF791B900BF014B53F806
:104DC0002000704708890020014B53F820007047ED
:104DD0000889002010B5114C642101FB00410346F5
:104DE0000A7E012A11D0642202FB034292F85D1070
:104DF00029B1918A1846BDE8104001F025BD18463A
:104E0000918A01F021FD404210BDCA7D012AEAD0FD
:104E1000898ABDE8104001F017BD00BF3082002034
:104E2000FFF7D8BF014B53F8200070470C890020D2
:104E3000014B53F82000704760890020014B53F864
:104E40002000704718890020642303FB00F0014B09
:104E500018587047308200200C4B994201D900202D
:104E6000704770B50A4D0B4E642404FB00F40B46EA
:104E7000291900EB8002897D46F832302B5103FB63
:104E800001F2602101F02CFC012070BD400D0300F7
:104E90003082002004820020094B99420ED830B4A1
:104EA000084B094C642500EB800203EBC20305FBB1
:104EB00000405961416030BC0120704700207047BC
:104EC000A08601000482002030820020012901D93F
:104ED0000020704730B4084B084C642500EB80027A
:104EE00003EBC20305FB0040C9B280F8361083F81B
:104EF0002410012030BC7047048200203082002042
:104F000038B50C4B044653F8200003F029F80A4B3F
:104F1000642202FB04340546206E03F021F80146AA
:104F2000284603F071F84FF05E5103F06DF803F07E
:104F3000BBF938BD648900203082002038B50E4BA3
:104F400000EB800203EBC2030446986803F008F804
:104F50000A4B642202FB04340546206E03F000F87D
:104F60000146284603F050F84FF05E5103F04CF82C
:104F700003F09AF938BD00BF04820020308200207F
:104F800038B50C4B044653F8200002F0E9FF0A4BF9
:104F9000642202FB04340546206E02F0E1FF014664
:104FA000284603F031F84FF05E5103F02DF803F07E
:104FB0007BF938BD308900203082002038B50446A6
:104FC000084602F0CDFF4FF08F4103F01DF8134A61
:104FD000642303FB04230546186E02F0C1FF01465B
:104FE000284603F0C5F803F05FF96B210546024639
:104FF000204601F075FB4FF480412046FCF7F2FD9E
:105000000749084B41F8245004EB840103EBC1032A
:10501000054A9D6042F824505D6038BD3082002012
:10502000308900200482002064890020B1F5007FCF
:1050300010B5044634D025DDB1F5806F12D0B1F53E
:10504000006F3DD1FCF7BCFD20464FF48E41FCF7CC
:10505000C9FD1C4A0123135520461946BDE81040DE
:1050600001F088BBFCF7ACFD20464FF49641FCF7FD
:10507000B9FD144B03221A5520460221BDE8104009
:1050800001F078BBB1F5807F1BD1FCF799FD4FF49F
:105090009C412046FCF7A6FD0A4B00221A5510BD84
:1050A000FCF78EFD20464FF49A41FCF79BFD054A24
:1050B0000223135520461946BDE8104001F05ABBA3
:1050C00010BD10BD2C89002008B5214B1878FBF7C6
:1050D0003DF902F0CDFA1AA3D3E9002302F03EFB1A
:1050E00019A3D3E9002302F063FC02F0E7FD194B9A
:1050F000B0F58C7F586009DA3C280CDD0420FCF701
:105100007BFD0220BDE80840FCF776BD0420BDE829
:105110000840FCF75FBD0220FCF75CFD002108465B
:10512000FBF70EF84FF480710020FFF77FFF00209F
:10513000FAF7E2FF0420BDE80840FCF75DBD00BFC0
:105140000000000000E052400000000000FEAF4000
:10515000250000206C810020F8B5494B1878FBF73A
:10516000F5F8A0F50840B83802F082FA0022454B65
:1051700002F0F4FA34A3D3E9002302F019FC02F0A0
:10518000E5FD02F097FA02460B4604460D4602F092
:1051900033F902460B462EA1D1E9000102F02AF9AB
:1051A0002DA3D3E9002306460F462046294602F0E8
:1051B000FFFB02460B463046394602F0F9FB02F08F
:1051C000C5FD02F077FA00222F4B02F0F1FB03F04D
:1051D000F7FA23A3D3E9002302F0C0FA22A3D3E90C
:1051E000002302F009F902460B4621A1D1E9000192
:1051F00002F0DEFB20A3D3E9002302F0FBF802F06B
:10520000A5FD03F051F8214B7728986002DC642853
:1052100012DDF8BD08210020FCF7D2FC4FF48071AC
:105220000020FFF703FF00210846FAF789FF00205E
:10523000BDE8F840FAF760BF08210020BDE8F8405B
:10524000FCF7D0BCAFF3008000000000E0FFEF40AF
:105250006666666666660A409A99999999990140C8
:10526000C3F5285C8FA272400000000000FEAA4037
:105270009A999999FD6F2F41C3F5285C8F1271405F
:105280002400002000001440000024406C81002015
:10529000134B642202FB0032137E43B1012B1AD060
:1052A00001F58C43503348F6A042934201D90020C7
:1052B000704710B50B4A0C4B42F8201004460022F0
:1052C0004FF4006143F82020FFF7B0FE2046FFF7BF
:1052D0005DFD012010BDD37D012BE1D00020704782
:1052E00030820020288900201489002070B50F4CDE
:1052F000642303FB00431B7E012B06D901F58C437D
:10530000503348F6A044A34201D9002070BD084D97
:10531000084C0B4600264FF4006145F8206044F825
:105320002030FFF783FE012070BD00BF30820020D7
:10533000288900201489002010B50E4C642303FB3B
:1053400000431B7E33B101F543330B4C03F5A073CF
:10535000A34201D9002010BD084A0B4604464FF471
:10536000007142F82030FFF761FE2046FFF70EFD86
:10537000012010BD30820020801A06000C89002018
:10538000F8B5154B642404FB0034237E03B9F8BD43
:105390000546084602F0E4FD4FF08F4102F034FE6E
:1053A0000746206E0D4E02F0DBFD0146384602F046
:1053B000DFFE02F079FF4FF4804146F825002846D1
:1053C000FCF710FC28464FF48061FFF72FFE2846BB
:1053D000BDE8F840FFF7DABC308200206489002085
:1053E0000F4B70B5044653F820000D4602F0B8FD8F
:1053F0000C4A642303FB04230646186E02F0B0FD3A
:105400000146304602F000FE4FF05E5102F0FCFD16
:1054100002F04AFF41192046BDE87040FFF7B0BFD7
:10542000308900203082002010B5044601F022FCB3
:10543000024B642202FB0434A07510BD30820020B0
:1054400010B4054C642303FB0043CAB29A7511469D
:1054500010BC01F015BC00BF30820020054A642357
:1054600003FB002310B40C460A46DC60998A10BC8A
:1054700001F06CBA30820020024A642303FB002052
:10548000C068704730820020032901D9002070478E
:1054900038B5044C642505FB0042D17501F0DAFBF8
:1054A000012038BD3082002010B5044601F0CAFB4F
:1054B000024B642202FB0434E07510BD30820020F0
:1054C000012901D900207047034B642202FB0033FD
:1054D000012083F85D10704730820020034A642366
:1054E00003FB002090F85D00704700BF3082002071
:1054F000042912D80A4AF8B5642505FB00220129BF
:10550000117608D00026074F29463346324647F821
:10551000206001F013F90120F8BD0020704700BFA2
:105520003082002014890020024A642303FB0020FB
:10553000007E704730820020022906D8044B642286
:1055400002FB00330120597670470020704700BFEE
:1055500030820020024A642303FB0020407E704713
:105560003082002008B5232101F098F800B208BD70
:1055700008B5392101F092F800B208BD08B52A211A
:1055800001F08CF8001408BD70B51A4E642303FBBB
:105590000063044693F8315093F83230003518BF59
:1055A00001250BB145F48055642303FB046393F894
:1055B00033300BB145F480753321204601F06EF88D
:1055C000020C12042A432046332101F089F83721C6
:1055D000204601F063F8642303FB046382B2B3F94D
:1055E0003430204642EA03423721BDE8704001F0E2
:1055F00077B800BF30820020054A642303FB0020F7
:1056000090F8373023EA010180F83710704700BF67
:1056100030820020054A642303FB002090F83730D5
:10562000194214BF01200020704700BF30820020C3
:1056300010B50A4B642404FB003494F83730D907C2
:105640000AD50021FFF7BAFC94F837305A0744BF57
:1056500023F0010384F8373010BD00BF30820020F2
:1056600010B52821044601F019F800B910BD2046F4
:10567000BDE81040FFF7DCBF08B5FCF7EBFAC0F35C
:10568000803008BD70B54A4D642303FB00530446C7
:105690001B7E042B1BD8DFE803F0394C5557030061
:1056A000642303FB0053DE7D012E55D001225221DD
:1056B000204601F015F84FF400612046FCF7B6FAD9
:1056C000002814BF01210221204601F053F8642371
:1056D00003FB04535B7E012B11D009D3022B06D1AF
:1056E000204601225121BDE8704000F0F9BF70BD95
:1056F000204600225121BDE8704000F0F1BF204655
:1057000003225121BDE8704000F0EABF00222421AD
:1057100000F0E6FF01222046522100F0E1FF204682
:10572000082101F027F800222121204600F0D8FFAF
:10573000CDE70222522100F0D3FF0121204601F0E3
:1057400019F8C4E70522B2E7642303FB0053DB7DAD
:10575000012B17D00322AAE733460022522100F082
:10576000EDFF00231A4620461C2100F0E7FF3246D9
:105770002046512100F0B4FF32465021204600F06F
:10578000AFFFA4E70022522100F0D8FF00231A4601
:1057900020461C2100F0D2FF20460322512100F0B8
:1057A0009FFF03225021204600F09AFF8FE700BFA1
:1057B00030820020F8B54249424D434E2F5C6422AE
:1057C00002FB0012137E9F424ED0032B044650D0A2
:1057D000642202FB0012527E012A18D04FF0000E04
:1057E000042B3BD0642000FB0410407E022835D0FF
:1057F0002B553255BEF1000F18D12046FFF742FF5E
:1058000020464FF40041BDE8F840FCF7D9B9032F1A
:1058100031D1042B41D1305C022844D0642000FBFC
:1058200004112B550120325581F82D00274B4FF4E0
:1058300000610022204623F81420FCF7F7F9002825
:1058400008BF0221204618BF012100F093FF204627
:105850004FF40041BDE8F840FCF7C4B9042FC7D0AD
:10586000305D0228DAD1C3E7527E345C9442ACD179
:10587000F8BD032F11D0325D012A4FF0640202FB04
:10588000041213D0D07D012894BF4FF0000E4FF0CA
:10589000010E82F826E0527EA2E7642202FB041287
:1058A000527E022A06D02B553255A6E74FF0000E45
:1058B000527E95E7305D0228B0D12B5530559CE7DC
:1058C0003082002034890020108900206C81002063
:1058D0002DE9F0410D46097882B0044616460329A9
:1058E00003D8DFE801F07C45070200232B7002B0EB
:1058F000BDE8F081594F37F81020013292B2632A87
:1059000027F8102072D84FF480481C2120460193BC
:1059100000F0C4FE000C000440EA08021C212046EE
:1059200000F0DEFE37F81420B242E0D3019B002BDA
:105930007BD14B4B642606FB04362046B18A0022FD
:1059400000F056FF0022B18A204600F0DDFF4FF440
:1059500000612046FCF76AF900280CBF02210121F2
:10596000204600F007FF03232B7002B0BDE8F08152
:1059700000230122292100F0E1FE2046012300221C
:10598000522100F0DBFE00231A4620461C2100F0C5
:10599000D5FE2046012100F0EDFE6421204600F0F6
:1059A0007DFE642182B2204600F09AFE2C4E6421D6
:1059B000204600F073FE642101FB0466020CB3680C
:1059C000B08A12041B0293FBF0F39BB21A432046E9
:1059D00000F086FE02232B7002B0BDE8F0811F4B61
:1059E000002223F8102002B0BDE8F081C72A16D9A2
:1059F000B2F5967F16D3B2F5C87F22D3B2F5FA7FFF
:105A000022D3B2F5167F22D3B2F52F7F22D3B2F57F
:105A1000487F4FF2FF7828BF4FF0000875E74BF63C
:105A2000FF7872E74FF400586FE7002227212046E5
:105A300000F056FE0A4B642202FB043200219184DE
:105A400078E74DF6FF7860E74FF480585DE74EF653
:105A5000FF785AE74FF4006857E700BF6C810020D9
:105A600030820020401A00B2704700BF2DE9F0419B
:105A70000D78012D0E46044632D02FD3022D2BD1A6
:105A80005A4B1B5C9A1E012A56D9012B6AD0002260
:105A90003921204600F044FE554FB7F90C3002B2D0
:105AA0009A421BD09BB2C01A05B205EBD57503EB29
:105AB000650301222A2120469DB200F031FEFB89B8
:105AC000C31AEB1A9BB220460122292100F036FEB0
:105AD00000233370BDE8F08100230B70BDE8F08136
:105AE000332100F0DBFD332120F48072204600F0EA
:105AF000F7FD00232A462921204600F01FFE002240
:105B00003921204600F00CFEDFF8E48007462A46E3
:105B10002A212046A8F80C7000F002FE3F1ABFB2FE
:105B20003B462A4620462921A8F80E7000F006FEC2
:105B300002233370BDE8F0812E4D642303FB005334
:105B400093F85D30002B43D02B4B53F82020642377
:105B500003FB04556621AB7D204602FB03F200F0F7
:105B6000BFFD94E7234D642303FB005393F85D309E
:105B70009BB3224B53F820706421204600F08EFD29
:105B8000642101FB045882B23B02B8F8140093FB75
:105B9000F0F3204642EA034200F0A2FD98F85D309F
:105BA00003BB174B53F824707F426421204600F05A
:105BB00075FD642101FB0455020C3B02A88A93FB8E
:105BC000F0F312049BB21A43204600F089FD5EE711
:105BD000094B53F820205242B9E7084B53F8207084
:105BE0007F42C9E7064B53F82470DEE72C8900207A
:105BF0006C810020308200206089002028890020EC
:105C0000148900202DE9F043164D642404FB00F0B4
:105C10002C182F58B4F84800891A1E4680FB0145FD
:105C2000002C4FF00003C7F10002316075F1000154
:105C3000736183B030614FEAE2730EDB200AB8462D
:105C40004FEAE77940EA05602912CDE9008901F0C1
:105C50008DFBB06103B0BDE8F083FF3445F1000572
:105C6000ECE700BF308200202DE9F04F89B0FAF751
:105C700057FCB94E0746FAF759FC3369984203D0EE
:105C80000446FCF79FF834617369FB1A002BB8BF18
:105C90005B42B3F57A7F80F25B81B3699F4200F08B
:105CA000408101F039F90020FFF784FDAB4C6A21F7
:105CB000002000F0F3FC94F85D20A37D90FBF3F04E
:105CC00002B94042237EDFF8B8A2DFF8B882012B88
:105CD00004BFA34B1869CAF80000002000F088FE3A
:105CE00094F85D20A37D90FBF3F0C8F8000012B992
:105CF0004042C8F800006921002000F0CFFCE27D9E
:105D0000012A4FEA104300F03F8147F6FF41CA18CD
:105D100092B24FF6FE15AA4204D8014489B2A942B4
:105D200040F26D8294F8305015F0010300F0FC80D1
:105D300094F82F1011F0010100F0A3810021084612
:105D4000FAF794FA94F83050031C18BF012315F0A9
:105D50000205039340F0ED804FF480610020FBF7D3
:105D600065FF00286BD094F836007E4B002800F0C9
:105D70002A81DFF8EC91069348461B68C9F8043085
:105D800000F0F8FBD9F80810774BD8F80020002075
:105D9000FFF738FFD8F800300493744BD9F8081097
:105DA0001860049B6268A1EB030E8EEAEE73A3EB0E
:105DB000EE7378204FEAE37C82FB000100FB0CF2DB
:105DC00003FB0122A0FB030123680793F3464FEA7C
:105DD000EE7C114400234FF6FF72CDE904BC02F0C3
:105DE00089FA079B83FB0323CDE9002300220023CC
:105DF00000F0D2FA00F0E2FADDE904BCBBF1010FD9
:105E00007CF10002C0F259812268514200F0BCFAD4
:105E100080EAE072A2EBE0725142544BDFF850B1DD
:105E2000186801F093FAD9F8103022684F490860D9
:105E30001844514201F08AFACBF80000CFE0484BF9
:105E40004849D8F800200A609A6018624FF400713F
:105E50000020FBF7EBFE002840F0EE804FF40061DD
:105E60000020FBF7E3FE68B13D4A4149DAF8003013
:105E70000B60D3601361002D40F00D81039B002B5C
:105E800040F015814FF480710020FBF7CFFE002811
:105E900044D1217E012900F03081023902293DD808
:105EA0004FF40041FBF7C2FE002800F01481314B93
:105EB0001B789A1E012A40F27A81012B2ED194F888
:105EC0005D30002B40F098812B4B1D686D426421A2
:105ED000002000F0E3FB82B2A18A2B02002093FB9A
:105EE000F1F3642142EA034200F0FAFB94F85D30DA
:105EF000002B40F06E81214B1D686D426421002013
:105F000000F0CCFB020CA18A12042B0293FBF1F3EC
:105F10009BB21A436421002000F0E2FBFFF7D4F8A3
:105F2000B76109B0BDE8F08F039315F002053FF4A7
:105F300013AF94F82F0010F002004FF0010100F0B1
:105F40009A800020FAF792F9051C18BF012503E793
:105F5000FFF702F97761A0E66C8100203082002013
:105F600004820020648900204089002038890020B4
:105F7000608900202C8900202889002014890020B5
:105F8000188900203089002003F5F9427F3292B24F
:105F90004FF6FE118A423FF6C5AEA18A1BB203FB43
:105FA00001F10029B8BFFF31091294F85D3003B93F
:105FB00049429A4D9A482A6808230093012300F029
:105FC00073FA2860AEE61A4606931168954BD8F826
:105FD0000020DFF854B2FFF715FECBF80000069B57
:105FE000D8F800101B68E26B5B1A002BB8BF5B424D
:105FF000934207DCDAF80030A26B002BB8BF5B429B
:10600000934262DD1DB1DBF80030002B08DB039BFF
:10601000002B3FF41BAFDBF80030002B7FF716AFEF
:1060200000210846FFF7DCF94FF400710020FBF770
:10603000FDFD00283FF412AFDFF8FC91DFF8FC8192
:106040004846D8F80030C9F80C3000F059FA764AC2
:10605000D9F8103013600DB1002B06DB039A002A2B
:106060003FF4FCAE002B7FF7F9AE0023C8F80030F8
:10607000C9F81030F2E6FAF7F9F8B0FA80F56D09D0
:106080006AE60846FAF7F2F8B0FA80F35B09039380
:1060900094F8305049E70020FEF79CFE0028BFF638
:1060A000EDAE6249624A00230B601360EAE600200D
:1060B000FEF790FE0028F4DCE4E6DDE904120A4372
:1060C00040F08A8000210A46A7E64FF48041002074
:1060D000FBF776FD96E794F826302BB1237E032B51
:1060E0003AD0637E012B37D00020FFF7CBFA4FF474
:1060F00000410020FBF764FD10E700F03BFBE37D6F
:10610000012B34D0DFF820B1DBF800500DB1A568C9
:106110002D026421002000F0C1FA020CA38A95FB35
:10612000F3F51204ADB22A436421002000F0D8FA3E
:106130006421002000F0B2FA642182B2002000F055
:10614000CFFA94F85D30DBF8002003B952422121E8
:10615000002000F0C5FAE1E6E07E002845D00228E4
:106160007FF4DCAE33490020FFF780FCD6E694F8DC
:106170005D30A3BB2D4B1D686D426421002000F0F3
:106180008DFA82B2A18A2B02002093FBF1F36421E5
:1061900042EA034200F0A4FA6421002000F07EFAF3
:1061A000020C12046421002000F09AFAB6E694F87A
:1061B0005D30BBB91C4B1B685B42A27D662103FBB3
:1061C00002F2002000F08CFA94F85D30002B3FF4CE
:1061D00092AE174B1D6891E62268404215E6134BBC
:1061E0001D68CAE7104B1B68E7E7A28B11490090B6
:1061F0000123FFF76DFB91E60C4B1D6867E61AB2B1
:10620000237EA18A02FA80F0012B01FB00F14FF4FA
:10621000807291FBF2F17FF4C8AECAE608890020D3
:1062200020890020408900206089002028890020E2
:106230001489002056820020048200200C8900204E
:1062400010B5044600F02CFD024B642202FB04341E
:10625000208210BD30820020B1F5803F01D30020A4
:10626000704738B5054C642505FB00428BB21946D2
:10627000138200F01BFD012038BD00BF30820020DA
:1062800010B5044600F022FD024B642202FB0434E8
:10629000608210BD30820020B1F5803F01D3002024
:1062A000704738B5054C642505FB00428BB2194692
:1062B000538200F011FD012038BD00BF3082002064
:1062C00008B5FAF72DF9014B186008BD9081002040
:1062D00070B5274A642404FB002494F8582032B98E
:1062E0004FF0FF327521BDE8704000F0F9B9054666
:1062F000B4F85A00C0EB003001F0CAF918A3D3E992
:10630000002301F055FB18A3D3E9002301F074F832
:1063100001F0FCFC012283B27521284600F00EFA40
:1063200094F85C30B4F85A00C01AC0EB003001F0A9
:10633000AFF90BA3D3E9002301F03AFB0AA3D3E999
:10634000002301F059F801F0E1FC002283B275212D
:106350002846BDE8704000F0F1B900BFAFF30080FF
:106360000000000000E05240000000000011E24088
:10637000308200200020FFF7ABBF00BFFFF7A8BFAF
:10638000704700BF00207047904203DC8842B8BFCE
:10639000084670471046704730B5DDE90345844232
:1063A00075EB010E07DB904271EB030400DB30BD9F
:1063B0001046194630BD2046294630BD021E37DB47
:1063C000FF2A1FDDB2F5803F36490CDBB2F1807F3A
:1063D0001CDBB2F1805F3ADBB2F1804F5ADB13165F
:1063E000CB5C1B0239E0B2F5805F19DBB2F5804F60
:1063F0003EDB1312CB5C581C00FB00F39A4219DA07
:1064000001387047274B985C00097047B2F5801F30
:1064100011DBB2F5800F41DB1314C85C000110E002
:10642000B2F5806F29DB1311CB5C9B08581CE3E7A6
:106430004FF0FF307047B2F5802F27DA9312C85C17
:106440004000431C92FBF0F003445810D4E7B2F133
:10645000806F17DA9314CB5C5B01581C92FBF3F34B
:1064600018444010431C92FBF0F003445810C3E75B
:106470009311CB5C5B08581CBEE79310CB5CDB0828
:10648000581CB9E71315CB5C9B01E6E71313C85CF6
:106490008000D6E79315CB5CDB01DEE79313C85C85
:1064A000C000CEE7BC8C0108D0B49DF80C40D0E908
:1064B0000067E31A891A9940761847EBE177C4F12F
:1064C000200226FA04F307FA02F2203C43EA020310
:1064D0005CBF47FA04F42343C0E900671846D0BC08
:1064E000704700BF00234FF6FF72028303604360D2
:1064F000C36003614361C361036280F82430704765
:10650000F8B590F82430044633B34369C568184E93
:10651000006986FB03262A1AD917002AC1EBA611A7
:10652000B8BF52428A42B8BF4FF47A73E169B8BF2C
:1065300053430F4A0B4482FB0312DE179211971B41
:106540004FF47A7101FB17338542E3610CDC05DA05
:10655000B21A1044206101E0C068206122685142F3
:10656000FFF712FF2061F8BD38442061F6E700BF55
:10657000D34D621090F8243013B94368836070479C
:106580002DE9F0438268456843690668AD1A85EADB
:10659000E572A2EBE5720446782083FB00014FEA26
:1065A000E27900FB09F302FB0133A0FB020183B097
:1065B000228B1944A6FB0667002301F09BFE0022F4
:1065C0000023CDE90067FFF7E7FEFFF7F7FE002D98
:1065D00053DD22680021FFF7D7FE05466369216974
:1065E0002D4E86FB03266A1AD817002AC0EBA61088
:1065F000B8BF52428242B8BF4FF47A73E069B8BF65
:106600005343254A034482FB0302DE179211971B72
:106610004FF47A7000FB17338D42E36136DD394465
:106620002161208B1C4E3C22002380FB010101F0E4
:1066300061FE226AA368801841EBE2714FF47A721E
:10664000C2FB030180EAE075A5EBE075002871F15B
:10665000000386FB05364FEAE573C3EBA61302FB86
:106660001353B8BF5B4223624FF47A72002301F0E8
:1066700041FEA06003B0BDE8F083AFD02168404286
:1066800049420022FFF780FE0546A7E7C9DAB21AA1
:1066900011442161C5E700BFD34D621038B501F048
:1066A0007F0100220546FBF739FE002211462846ED
:1066B000FBF734FE0022114604022846FBF72EFEAB
:1066C0000022114604432846FBF728FE240201223B
:1066D000044300212846FBF721FE2402204338BD55
:1066E00038B541F08001154604460022FBF716FE3E
:1066F000290E20460022FBF711FEC5F30741204674
:106700000022FBF70BFEC5F3072120460022FBF712
:1067100005FEE9B220460122BDE83840FBF7FEBD88
:1067200010B51446FFF7BAFF2CB1012C01D1000CB3
:1067300010BD002010BD80B210BD00BFF8B51446DA
:106740001F4605460E46FFF7A9FF54B1012C01D1A3
:1067500067F31F40024631462846BDE8F840FFF780
:10676000BFBF67F30F00024631462846BDE8F84038
:10677000FFF7B6BF38B50D4663210446FFF78EFF1D
:1067800020F0FF0045EA000263212046BDE83840C2
:10679000FFF7A6BF70B50D4604460121FFF7EAFFDB
:1067A000ABB2204601226421BDE87040FFF7C6BFAE
:1067B00070B56F210446FFF771FF002206466F2176
:1067C0002046FFF78DFF20466E21FFF767FF324618
:1067D00005466F212046FFF783FF284670BD00BFA6
:1067E00008B56921FFF75AFF001408BD0020704763
:1067F00070B50D46144606460121FFF7BBFF240283
:10680000304694FBF5F301229BB26421BDE8704051
:10681000FFF794BF10B50C46FFF7CAFF00FB04F06A
:106820000028B8BFFF30001210BD00BF10B50C46E5
:106830006921FFF733FF001404FB00F00028B8BF04
:10684000FF30001210BD00BF2DE9F0410D466F2151
:106850000446FFF723FF002280466F212046FFF702
:106860003FFF20466E21FFF719FF012206466F21E8
:106870002046FFF735FF20466E21FFF70FFF424607
:1068800007466F212046FFF72BFFF01905FB00F0AC
:106890000028B8BFFF300012BDE8F08110B50C46EB
:1068A0006921FFF7FBFE03B203EB204004FB00F07D
:1068B0000028B8BFFF30001210BD00BF0020704795
:1068C0008BB200226421FFF739BF00BF70B56F2182
:1068D0000446FFF7E3FE012206466F212046FFF73C
:1068E000FFFE20466E21FFF7D9FE324605466F2196
:1068F0002046FFF7F5FE284670BD00BF08B56921A8
:10690000FFF7CCFE00B208BD1302002293FBF1F3A7
:1069100064219BB2FFF712BF10B50C46FFF7D6FFFC
:1069200000FB04F00028B8BFFF30001210BD00BF0C
:1069300010B50C466921FFF7B1FE00B200FB04F070
:106940000028B8BFFF30001210BD00BF13020022A4
:1069500093FBF1F35E219BB2FFF7F0BE10B50C463E
:106960005E21FFF79BFE80B204FB00F0001210BD19
:1069700038B50D4604460221FFF7FCFE2A462046A4
:106980006621BDE83840FFF7ABBE00BF6621FFF7C8
:1069900085BE00BF6A21FFF781BE00BF002070479F
:1069A00038B50D4604460321FFF7E4FE2A4620468B
:1069B0006821BDE83840FFF793BE00BF38B50446F4
:1069C0000D460321FFF7D6FE20466B21FFF766FE3A
:1069D000682142192046BDE83840FFF781BE00BF5C
:1069E0006821FFF75BBE00BF0A466B21FFF778BE48
:1069F0006B21FFF753BE00BF00207047F8B50D466E
:106A00000978BDF818600446032903D8DFE801F0CF
:106A10005625050200232B70F8BD1988013189B273
:106A200091421980F8D3274E002227212046FFF7F4
:106A300057FE726824212046FFF752FE3389002258
:106A40001C212046FFF77AFE33882046002252217F
:106A5000FFF774FE03232B70F8BD52212046FFF789
:106A60001DFE184F242138802046FFF717FE1C21F9
:106A700078602046FFF712FE002338810122292189
:106A80002046FFF75BFE0123002252212046FFF73C
:106A900055FE0023012224212046FFF74FFE3346F6
:106AA000002224212046FFF749FE00231A462046F3
:106AB0001C21FFF743FE02232B70F8BD00221A8031
:106AC000F8BD00BF94810020401A00B2704700BF9B
:106AD0002DE9F0410C78012C0D4606462DD028D327
:106AE000022C03D000230B70BDE8F0813921FFF7A1
:106AF000D5FD274FB7F90A3002B29A42F4D09BB2C3
:106B0000C01A04B204EBD47403EB64032A213046A8
:106B10009CB2FFF7C3FDBB89C3EB1043E31A9BB2E2
:106B2000304601222921FFF709FE00232B70BDE822
:106B3000F08100231380BDE8F0813321FFF7AEFD23
:106B4000332120F480723046FFF7CAFD002322462D
:106B500029213046FFF7F2FD39213046FFF79EFD2F
:106B6000DFF82C8007462A213046A8F80A70FFF784
:106B700095FDA7EB1047BFB23B4622463046292180
:106B8000A8F80C70FFF7DAFD02232B70BDE8F08146
:106B9000948100202DE9F045124D98462B6983B071
:106BA0008B42BDF828E00B9FBDF830C014468246EA
:106BB00002D00E462AB12E61022C0AD003B0BDE8E5
:106BC000F085CDF800C072463B464146FFF716FF00
:106BD000F1E73A464146504603B0BDE8F045FFF7BD
:106BE00077BF00BF9481002070B4BDF80C60BDF881
:106BF00014400396059470BCFFF7CCBF137813B90B
:106C000010B1022800D0704701230870137070473C
:106C100091420BD038B5522114461D46FFF760FD56
:106C2000032C02D1049B1B780BB138BD704715F0C3
:106C3000FD0FFAD1049A01231370F6E700221A21FE
:106C4000FFF74EBD08B51B21FFF728FDC0F3074035
:106C500008BD00BF38B50D461B210446FFF71EFDD9
:106C600020F47F0040EA05421B212046BDE8384061
:106C7000FFF736BD08B51B21FFF710FDC0B208BDF8
:106C800038B50D461B210446FFF708FD000C000433
:106C900040EA05021B212046BDE83840FFF720BD31
:106CA00008B50921FFF7FAFC80B208BD38B50D46DA
:106CB00009210446FFF7F2FC000C000440EA05023B
:106CC00009212046BDE83840FFF70ABD08B5082174
:106CD000FFF7E4FC80B208BD38B50D460821044634
:106CE000FFF7DCFC000C000440EA05020821204606
:106CF000BDE83840FFF7F4BC38B542EA014422460B
:106D000005465421FFF7ECFC224628465621BDE8F3
:106D10003840FFF7E5BC00BF42EA01425821FFF7C7
:106D2000DFBC00BF42EA01425A21FFF7D9BC00BFD5
:106D30002DE9F047894611469A4616460546089CB5
:106D40009DF82480FFF7AAFC5246074631462846A4
:106D5000FFF7C6FC49462846FFF7A0FC044024FA8A
:106D600008F428463A463146FFF7BAFC2046BDE80B
:106D7000F08700BF38B501F07F0100220546FBF720
:106D8000CFFA002211462846FBF7CAFA0022114624
:106D900004022846FBF7C4FA0022114604432846A1
:106DA000FBF7BEFA24020122044300212846FBF728
:106DB000B7FA2402204338BD38B541F080011546AA
:106DC00004460022FBF7ACFA290E20460022FBF70E
:106DD000A7FAC5F3074120460022FBF7A1FAC5F345
:106DE000072120460022FBF79BFAE9B22046012248
:106DF000BDE83840FBF794BA00230022C0E9022323
:106E00000023036083617047114B1A68811A81EA7D
:106E1000E172A2EBE172B2F57A7F18DBF0B41F6980
:106E20009E691D6A9C6ADF605E61DD615C62F0BC28
:106E300018609868196B58600022986B9A601A6104
:106E40009A611A629A621A63D9629A6358637047A8
:106E5000A8810020024A936801339360704700BF05
:106E6000A8810020014B9868704700BFA8810020CE
:106E7000014B5868704700BFA8810020024A13697F
:106E800001331361704700BFA8810020014BD8680F
:106E9000704700BFA8810020024A936901339361C3
:106EA000704700BFA8810020014B5869704700BFA0
:106EB000A8810020024A136A01331362704700BFA1
:106EC000A8810020014BD869704700BFA88100202D
:106ED000024A936A01339362704700BFA881002081
:106EE000014B586A704700BFA8810020024A136B0B
:106EF00001331363704700BFA8810020014BD86A9B
:106F0000704700BFA8810020024B186B00EB800087
:106F100040007047A8810020024A936B01339363BD
:106F2000704700BFA8810020014B586B704700BF1D
:106F3000A8810020024B986B00EB80004000704756
:106F4000A8810020014B1860704700BF9089002085
:106F5000014B1868704700BF90890020014B1860F2
:106F6000704700BF88890020014B1868704700BF38
:106F700088890020014B1860704700BF8489002079
:106F8000014B1868704700BF84890020014B1860CE
:106F9000704700BF7C890020014B1868704700BF14
:106FA0007C890020014B1860704700BF8C8900204D
:106FB000014B1868704700BF8C890020014B186096
:106FC000704700BF70890020014B1868704700BFF0
:106FD00070890020014B1860704700BF788900203D
:106FE000014B1868704700BF78890020014B18607A
:106FF000704700BF74890020014B1868704700BFBC
:1070000074890020014B1860704700BF8089002000
:10701000014B1868704700BF80890020014B186041
:10702000704700BF6C890020014B1868704700BF93
:107030006C890020054B10B40022012418705C728A
:1070400059601A72DA6010BC704700BFEC810020F2
:10705000024B00225A721A72DA607047EC810020EB
:10706000014B187A704700BFEC810020014B587A21
:10707000704700BFEC810020014BD868704700BF0B
:10708000EC810020064B0068DA6801320021824260
:10709000DA60196102D159721972D960704700BF64
:1070A000EC81002084B0F0B4144D154E2C69376883
:1070B000013405AEBC422C6186E80E0016DB2B7A4B
:1070C000A3B10168EB68994210DD4268059E069CF9
:1070D00007981F010133D6513A440026089FEB6000
:1070E000994254609060D7602E6102D0F0BC04B029
:1070F00070476E722E72EE60F8E700BFEC810020E0
:10710000480000200068704700680001704700BF19
:107110000420704710B404688C420DDD032A02DDA0
:10712000022010BC7047406810BC00EB0111002029
:1071300051F822201A607047012010BC704700BF30
:107140000A2807D8DFE800F00611150A0E0E060619
:1071500006060E00094B00225A617047074B0322B6
:107160005A617047054B58617047044B01225A61C0
:107170007047024B02225A61704700BFEC81002029
:10718000014B5869704700BFEC810020014B18602B
:10719000704700BF48000020014B1868704700BFCF
:1071A0004800002010B5144B1C78062C08D8DFE8E6
:1071B00004F00713171B1F0C04005A68904207DDE8
:1071C00001221A7200225A7210BD5A688242F7DCFC
:1071D0001A7A002AF6D110BD59689142F8DDEFE71E
:1071E00059688A42ECDCF3E75A688A42E8DCEFE748
:1071F0005A689142E4DCEBE7EC810020B0F5803F77
:107200001CDBB0F1807F31DBB0F1805F39DAB0F1A7
:10721000806F394A4DDB0315D35C9B015A1C90FBF0
:10722000F3F31A445210531C90FBF2F213445B1018
:1072300003FB03F2904217DA581E7047FF2805DC63
:10724000002856DB2C4B185C00097047B0F5805FB6
:10725000294A26DBB0F5804F2FDB0312D35C0133C4
:1072600003FB03F29042E7DB18467047B0F5801F3E
:10727000214A0FDBB0F5800F32DB0314D25C120120
:10728000D1E7B0F1804F22DB1C4B98422CDD4FF64A
:10729000FF707047B0F5802F1EDB0313D25C9200A5
:1072A000C1E7B0F5806F0DDB0311D35C9B080133A0
:1072B000D6E78314D35C5B01B0E78311D35C5B0832
:1072C0000133CDE78310D35CDB080133C8E70A4AFA
:1072D0008315D35CDB01A1E78312D25C5200A2E7E5
:1072E0008313D25CD2009EE7034A0316D35C1B02D1
:1072F00094E74FF0FF307047BC8D01080080FE7F9F
:10730000B0F5806F14D2B0F5007F08D2FF2895BF8A
:107310000A4B0B4BC018181A90F800017047B0F5D3
:10732000407F07D3074B181A90F80001404270477E
:1073300000207047044BC05C40427047BC8D010880
:10734000BB8F0108BB910108BC8C0108904203DC93
:107350008842B8BF0846704710467047904203D82D
:10736000884238BF084670471046704730B5DDE99F
:107370000345844275EB010E07DB904271EB030479
:1073800000DB30BD1046194630BD2046294630BDD1
:1073900070B514460E4600F0E3FD0546204600F0A9
:1073A000DBFD04460146284600F0E2FE0146284681
:1073B00000F020FD0546304600F0D2FD214600F0E9
:1073C000D7FE0146284600F017FD00F06DFF70BDA6
:1073D00030B4029C0568E31A8A1A02FA03F32B44BC
:1073E000036043FA04F030BC704700BF81F00041F5
:1073F00002E000BF83F0004330B54FEA41044FEA9A
:10740000430594EA050F08BF90EA020F1FBF54EA34
:10741000000C55EA020C7FEA645C7FEA655C00F0D0
:10742000E2804FEA5454D4EB5555B8BF6D420CDDA1
:107430002C4480EA020281EA030382EA000083EA24
:10744000010180EA020281EA0303362D88BF30BDC4
:1074500011F0004F4FEA01314FF4801C4CEA11311A
:1074600002D0404261EB410113F0004F4FEA033379
:107470004CEA133302D0524263EB430394EA050F04
:1074800000F0A780A4F10104D5F1200E0DDB02FA73
:107490000EFC22FA05F2801841F1000103FA0EF207
:1074A000801843FA05F359410EE0A5F120050EF1CD
:1074B000200E012A03FA0EFC28BF4CF0020C43FAFE
:1074C00005F3C01851EBE37101F0004507D54FF00B
:1074D000000EDCF1000C7EEB00006EEB0101B1F55B
:1074E000801F1BD3B1F5001F0CD349085FEA3000A1
:1074F0004FEA3C0C04F101044FEA445212F5800FAC
:1075000080F09A80BCF1004F08BF5FEA500C50F148
:10751000000041EB045141EA050130BD5FEA4C0C2B
:10752000404141EB010111F4801FA4F10104E9D1B4
:1075300091F0000F04BF01460020B1FA81F308BFAB
:107540002033A3F10B03B3F120020CDA0C3208DD77
:1075500002F1140CC2F10C0201FA0CF021FA02F152
:107560000CE002F11402D8BFC2F1200C01FA02F1C2
:1075700020FA0CFCDCBF41EA0C019040E41AA2BFE7
:1075800001EB0451294330BD6FEA04041F3C1CDAAF
:107590000C340EDC04F11404C4F1200220FA04F0CF
:1075A00001FA02F340EA030021FA04F345EA030179
:1075B00030BDC4F10C04C4F1200220FA02F001FA3B
:1075C00004F340EA0300294630BD21FA04F02946BD
:1075D00030BD94F0000F83F4801306BF81F4801156
:1075E0000134013D4EE77FEA645C18BF7FEA655CC9
:1075F00029D094EA050F08BF90EA020F05D054EA9B
:10760000000C04BF1946104630BD91EA030F1EBF9F
:107610000021002030BD5FEA545C05D140004941A3
:1076200028BF41F0004130BD14F580043CBF01F596
:10763000801130BD01F0004545F0FE4141F470017C
:107640004FF0000030BD7FEA645C1ABF1946104657
:107650007FEA655C1CBF0B46024650EA013406BF58
:1076600052EA033591EA030F41F4002130BD00BF17
:1076700090F0000F04BF0021704730B54FF48064D4
:1076800004F132044FF000054FF0000150E700BF55
:1076900090F0000F04BF0021704730B54FF48064B4
:1076A00004F1320410F0004548BF40424FF00001A1
:1076B0003EE700BF42004FEAE2014FEA31014FEAE4
:1076C00002701FBF12F07F4393F07F4F81F0605133
:1076D000704792F0000F14BF93F07F4F704730B5A2
:1076E0004FF4607401F0004521F0004120E700BF35
:1076F00050EA010208BF704730B54FF000050AE0BC
:1077000050EA010208BF704730B511F0004502D5BC
:10771000404261EB41014FF4806404F132045FEABE
:10772000915C3FF4DCAE4FF003025FEADC0C18BF63
:1077300003325FEADC0C18BF033202EBDC02C2F159
:10774000200300FA03FC20FA02F001FA03FE40EAEB
:107750000E0021FA02F11444C1E600BF70B54FF0EB
:10776000FF0C4CF4E06C1CEA11541DBF1CEA1355CD
:1077700094EA0C0F95EA0C0F00F0DEF82C4481EA35
:10778000030621EA4C5123EA4C5350EA013518BF55
:1077900052EA033541F4801143F4801338D0A0FB42
:1077A00002CE4FF00005E1FB02E506F00042E0FBEF
:1077B00003E54FF00006E1FB03569CF0000F18BFF5
:1077C0004EF0010EA4F1FF04B6F5007F64F540749D
:1077D00004D25FEA4E0E6D4146EB060642EAC62130
:1077E00041EA55514FEAC52040EA5E504FEACE2E9D
:1077F000B4F1FD0C88BFBCF5E06F1ED8BEF1004FA0
:1078000008BF5FEA500E50F1000041EB045170BD1B
:1078100006F0004646EA010140EA020081EA03015F
:10782000B4EB5C04C2BFD4EB0C0541EA045170BD5B
:1078300041F480114FF0000E013C00F3AB8014F1D5
:10784000360FDEBF002001F0004170BDC4F100041E
:10785000203C35DA0C341BDC04F11404C4F120059F
:1078600000FA05F320FA04F001FA05F240EA0200FA
:1078700001F0004221F0004110EBD37021FA04F630
:1078800042EB06015EEA430E08BF20EAD37070BDEA
:10789000C4F10C04C4F1200500FA04F320FA05F049
:1078A00001FA04F240EA020001F0004110EBD3704B
:1078B00041F100015EEA430E08BF20EAD37070BDBB
:1078C000C4F1200500FA05F24EEA020E20FA04F394
:1078D00001FA05F243EA020321FA04F001F0004143
:1078E00021FA04F220EA020000EBD3705EEA430EB4
:1078F00008BF20EAD37070BD94F0000F0FD101F0E3
:107900000046400041EB010111F4801F08BF013C1B
:10791000F7D041EA060195F0000F18BF704703F059
:107920000046520043EB030313F4801F08BF013DE0
:10793000F7D043EA0603704794EA0C0F0CEA13559C
:1079400018BF95EA0C0F0CD050EA410618BF52EA56
:107950004306D1D181EA030101F000414FF000005C
:1079600070BD50EA410606BF1046194652EA43066A
:1079700019D094EA0C0F02D150EA013613D195EADE
:107980000C0F05D152EA03361CBF104619460AD126
:1079900081EA030101F0004141F0FE4141F4700130
:1079A0004FF0000070BD41F0FE4141F4780170BD20
:1079B00070B54FF0FF0C4CF4E06C1CEA11541DBF85
:1079C0001CEA135594EA0C0F95EA0C0F00F0A7F887
:1079D000A4EB050481EA030E52EA03354FEA0131B4
:1079E00000F088804FEA03334FF0805545EA1313C7
:1079F00043EA12634FEA022245EA111545EA10658F
:107A00004FEA00260EF000419D4208BF964244F125
:107A1000FD0404F5407402D25B084FEA3202B61A44
:107A200065EB03055B084FEA32024FF480104FF418
:107A3000002CB6EB020E75EB030E22BFB61A75468C
:107A400040EA0C005B084FEA3202B6EB020E75EB1F
:107A5000030E22BFB61A754640EA5C005B084FEA87
:107A60003202B6EB020E75EB030E22BFB61A754654
:107A700040EA9C005B084FEA3202B6EB020E75EB5F
:107A8000030E22BFB61A754640EADC0055EA060E20
:107A900018D04FEA051545EA16754FEA06164FEA63
:107AA000C30343EA52734FEAC2025FEA1C1CC0D10F
:107AB00011F4801F0BD141EA00014FF000004FF09C
:107AC000004CB6E711F4801F04BF01430020B4F15D
:107AD000FD0C88BFBCF5E06F3FF6AFAEB5EB030C15
:107AE00004BFB6EB020C5FEA500C50F1000041EB12
:107AF000045170BD0EF0004E4EEA113114EB5C04DF
:107B0000C2BFD4EB0C0541EA045170BD41F48011B1
:107B10004FF0000E013C90E645EA060E8DE60CEAB9
:107B2000135594EA0C0F08BF95EA0C0F3FF43BAFD6
:107B300094EA0C0F0AD150EA01347FF434AF95EA8D
:107B40000C0F7FF425AF104619462CE795EA0C0F71
:107B500006D152EA03353FF4FDAE1046194622E73E
:107B600050EA410618BF52EA43067FF4C5AE50EA18
:107B700041047FF40DAF52EA43057FF4EBAE12E708
:107B80004FF0FF3C06E000BF4FF0010C02E000BFE9
:107B90004FF0010C4DF804CD4FEA410C7FEA6C5CCC
:107BA0004FEA430C18BF7FEA6C5C1BD001B050EA6F
:107BB000410C0CBF52EA430C91EA030F02BF90EA5A
:107BC000020F0020704710F1000F91EA030F58BF19
:107BD000994208BF90422CBFD8176FEAE37040F07B
:107BE000010070474FEA410C7FEA6C5C02D150EA19
:107BF000013C07D14FEA430C7FEA6C5CD6D152EAD4
:107C0000033CD3D05DF8040B704700BF8446104698
:107C100062468C461946634600E000BF01B5FFF797
:107C2000B7FF002848BF10F1000F01BD4DF808ED67
:107C3000FFF7F4FF0CBF012000205DF808FB00BF38
:107C40004DF808EDFFF7EAFF34BF012000205DF892
:107C500008FB00BF4DF808EDFFF7E0FF94BF0120DF
:107C600000205DF808FB00BF4DF808EDFFF7CEFFE0
:107C700094BF012000205DF808FB00BF4DF808ED1F
:107C8000FFF7C4FF34BF012000205DF808FB00BFF0
:107C90004FEA410C7FEA6C5C02D150EA013C0AD108
:107CA0004FEA430C7FEA6C5C02D152EA033C02D1FA
:107CB0004FF0000070474FF0010070474FEA41025B
:107CC00012F5001215D211D56FF47873B3EB62522E
:107CD00012D94FEAC12343F0004343EA505311F055
:107CE000004F23FA02F018BF404270474FF00000E7
:107CF000704750EA013005D111F0004008BF6FF025
:107D0000004070474FF00000704700BF4A0011D29A
:107D100012F5001211D20DD56FF47873B3EB6252E5
:107D20000ED44FEAC12343F0004343EA505323FAF1
:107D300002F070474FF00000704750EA013002D166
:107D40004FF0FF3070474FF0000070474FEA41029C
:107D5000B2F1E04324BFB3F5001CDCF1FE5C0DD9A9
:107D600001F0004C4FEAC0024CEA5070B2F1004FF3
:107D700040EB830008BF20F00100704711F0804FF6
:107D800021D113F13872BCBF01F00040704741F4BB
:107D900080114FEA5252C2F11802C2F1200C10FABF
:107DA0000CF320FA02F018BF40F001004FEAC123A3
:107DB0004FEAD32303FA0CFC40EA0C0023FA02F347
:107DC0004FEA4303CCE77FEA625307D150EA01331D
:107DD0001EBF4FF0FE4040F44000704701F00040ED
:107DE00040F0FE4040F40000704700BF80F00040CB
:107DF00002E000BF81F0004142001FBF5FEA410383
:107E000092EA030F7FEA226C7FEA236C6AD04FEA82
:107E10001262D2EB1363C1BFD218414048404140C7
:107E2000B8BF5B42192B88BF704710F0004F40F479
:107E3000000020F07F4018BF404211F0004F41F495
:107E4000000121F07F4118BF494292EA030F3FD061
:107E5000A2F1010241FA03FC10EB0C00C3F1200374
:107E600001FA03F100F0004302D5494260EB400003
:107E7000B0F5000F13D3B0F1807F06D340084FEA6E
:107E8000310102F10102FE2A51D2B1F1004F40EB63
:107E9000C25008BF20F0010040EA030070474900CB
:107EA00040EB000010F4000FA2F10102EDD1B0FA96
:107EB00080FCACF1080CB2EB0C0200FA0CF0AABF8B
:107EC00000EBC25052421843BCBFD0401843704729
:107ED00092F0000F81F4000106BF80F4000001322F
:107EE000013BB5E74FEA41037FEA226C18BF7FEA06
:107EF000236C21D092EA030F04D092F0000F08BF48
:107F00000846704790EA010F1CBF0020704712F02E
:107F10007F4F04D1400028BF40F00040704712F16D
:107F200000723CBF00F50000704700F0004343F0D2
:107F3000FE4040F4000070477FEA226216BF084608
:107F40007FEA23630146420206BF5FEA412390EACB
:107F5000010F40F4800070474FF0000304E000BFC1
:107F600010F0004348BF40425FEA000C08BF704772
:107F700043F0964301464FF000001CE050EA010236
:107F800008BF70474FF000030AE000BF50EA01024B
:107F900008BF704711F0004302D5404261EB410138
:107FA0005FEA010C02BF84460146002043F0B6435D
:107FB00008BFA3F18053A3F50003BCFA8CF2083A82
:107FC000A3EBC25310DB01FA02FC634400FA02FC8B
:107FD000C2F12002BCF1004F20FA02F243EB020092
:107FE00008BF20F00100704702F1200201FA02FCF4
:107FF000C2F1200250EA4C0021FA02F243EB0200E7
:1080000008BF20EADC7070474FF0FF0C1CEAD0522A
:108010001EBF1CEAD15392EA0C0F93EA0C0F6FD0EB
:108020001A4480EA010C400218BF5FEA41211ED0C9
:108030004FF0006343EA501043EA5111A0FB0131B5
:108040000CF00040B1F5000F3EBF490041EAD3718A
:108050005B0040EA010062F17F02FD2A1DD8B3F106
:10806000004F40EBC25008BF20F00100704790F075
:10807000000F0CF0004C08BF49024CEA502040EAC7
:1080800051207F3AC2BFD2F1FF0340EAC25070478D
:1080900040F400004FF00003013A5DDC12F1190FCB
:1080A000DCBF00F000407047C2F10002410021FA3D
:1080B00002F1C2F1200200FA02FC5FEA310040F155
:1080C000000053EA4C0308BF20EADC70704792F0CE
:1080D000000F00F0004C02BF400010F4000F013A06
:1080E000F9D040EA0C0093F0000F01F0004C02BF01
:1080F000490011F4000F013BF9D041EA0C018FE770
:108100000CEAD15392EA0C0F18BF93EA0C0F0AD075
:1081100030F0004C18BF31F0004CD8D180EA01009B
:1081200000F00040704790F0000F17BF90F0004F34
:10813000084691F0000F91F0004F14D092EA0C0F16
:1081400001D142020FD193EA0C0F03D14B0218BFA9
:10815000084608D180EA010000F0004040F0FE40EF
:1081600040F40000704740F0FE4040F4400070478B
:108170004FF0FF0C1CEAD0521EBF1CEAD15392EA0A
:108180000C0F93EA0C0F69D0A2EB030280EA010CFA
:1081900049024FEA402037D04FF0805343EA111193
:1081A00043EA10130CF000408B4238BF5B0042F1F1
:1081B0007D024FF4000C8B4224BF5B1A40EA0C0096
:1081C000B3EB510F24BFA3EB510340EA5C00B3EBC8
:1081D000910F24BFA3EB910340EA9C00B3EBD10FB6
:1081E00024BFA3EBD10340EADC001B0118BF5FEA08
:1081F0001C1CE0D1FD2A3FF650AF8B4240EBC25031
:1082000008BF20F0010070470CF0004C4CEA5020F1
:108210007F32C2BFD2F1FF0340EAC250704740F440
:1082200000004FF00003013A37E792F0000F00F032
:10823000004C02BF400010F4000F013AF9D040EAB0
:108240000C0093F0000F01F0004C02BF490011F444
:10825000000F013BF9D041EA0C0195E70CEAD1533C
:1082600092EA0C0F08D142027FF47DAF93EA0C0F23
:108270007FF470AF084676E793EA0C0F04D14B0207
:108280003FF44CAF08466EE730F0004C18BF31F0B9
:10829000004CCAD130F000427FF45CAF31F00043B3
:1082A0007FF43CAF5FE700BF4FEA4002B2F1FE4F00
:1082B0000FD34FF09E03B3EB12620DD94FEA0023A8
:1082C00043F0004310F0004F23FA02F018BF404281
:1082D00070474FF00000704712F1610F01D1420268
:1082E00005D110F0004008BF6FF0004070474FF01C
:1082F000000070477BB972B90029BEBF00204FF063
:10830000004106E008BF00281CBF6FF000414FF09D
:10831000FF3000F0ADB9ADF1080C6DE904CE0029D5
:1083200009DB002B1ADB00F035F8DDF804E0DDE9AD
:10833000022304B07047404261EB4101002B1BDB7C
:1083400000F028F8DDF804E0DDE9022304B0404243
:1083500061EB4101524263EB43037047524263EBCE
:10836000430300F017F8DDF804E0DDE9022304B070
:10837000404261EB41017047524263EB430300F01E
:1083800009F8DDF804E0DDE9022304B0524263EBB2
:10839000430370472DE9F0478C460D460446089E7E
:1083A000002B51D18A4217466DD9B2FA82FEBEF136
:1083B000000F0BD0CEF1200C01FA0EF520FA0CFCC8
:1083C00002FA0EF74CEA050C00FA0EF44FEA174ACF
:1083D000250CBCFBFAF81FFA87F90AFB18CC45EA12
:1083E0000C4508FB09F3AB420AD9ED1908F1FF323D
:1083F00080F02381AB4240F22081A8F102083D4485
:10840000ED1AA4B2B5FBFAF00AFB105544EA054494
:1084100000FB09F9A14509D9E41900F1FF3380F007
:108420000A81A14540F2078102383C44A4EB0904CB
:1084300040EA08400021002E61D024FA0EF4002307
:1084400034607360BDE8F0878B4207D9002E54D0AA
:10845000002186E821000846BDE8F087B3FA83F1E1
:10846000002940F08E80AB4202D3824200F2FA80B3
:10847000841A65EB03050120AC46002E3FD086E848
:108480001010BDE8F08712B90127B7FBF2F7B7FA71
:1084900087FEBEF1000F34D1EB1B3A0C1FFA87FCAC
:1084A0000121B3FBF2F8250C02FB183345EA034522
:1084B0000CFB08F3AB4207D9ED1908F1FF3002D2EB
:1084C000AB4200F2D1808046ED1AA3B2B5FBF2F0C8
:1084D00002FB105543EA05440CFB00FCA44507D9F8
:1084E000E41900F1FF3302D2A44500F2B880184627
:1084F000A4EB0C0440EA08409DE731463046BDE855
:10850000F087CEF1200405FA0EF307FA0EF720FAF1
:1085100004F83A0C25FA04F448EA0308B4FBF2F133
:108520004FEA184502FB11441FFA87FC45EA04454F
:1085300001FB0CF3AB4200FA0EF409D9ED1901F17D
:10854000FF3080F08A80AB4240F2878002393D44A0
:10855000EB1A1FFA88F5B3FBF2F002FB103345EA81
:10856000034500FB0CF3AB4207D9ED1900F1FF38CE
:108570006FD2AB426DD902383D44EB1A40EA01415B
:108580008FE7C1F1200722FA07F88B4005FA01F4C2
:1085900048EA030320FA07FE4FEA134CFD404EEA77
:1085A000040EB5FBFCF94FEA1E440CFB19551FFAEB
:1085B00083F844EA054509FB08F4AC4202FA01F2EB
:1085C00000FA01FA08D9ED1809F1FF3043D2AC42A4
:1085D00041D9A9F102091D442D1B1FFA8EFEB5FBDE
:1085E000FCF00CFB10554EEA054400FB08F8A045D2
:1085F00007D9E41800F1FF3529D2A04527D9023860
:108600001C4440EA0940A4EB0804A0FB02894C4545
:10861000C6464D4615D312D056B1BAEB0E0364EBE5
:10862000050404FA07F7CB401F43CC403760746061
:108630000021BDE8F0871846F8E69046E0E6C2451E
:10864000EAD2B8EB020E69EB03050138E4E72846ED
:10865000D7E7404691E78146BEE7014678E7023812
:108660003C4445E7084608E7A8F102083D442BE7EB
:10867000704700BFDFF834D0002103E00C4B5B589B
:10868000435004310B480C4B42189A42F6D30B4A24
:1086900002E0002342F8043B094B9A42F9D3F3F776
:1086A000D1FD00F069F800F00FF8874600000220C5
:1086B000F48F010800000020B4000020B800002062
:1086C00094890020FEE70000294D2A4C08B5F7F7F1
:1086D000BFFEF7F7FBF8F7F715F9F7F7B7F9F7F774
:1086E000D1FBF7F707FFF9F739FDF9F7ADFDF8F71B
:1086F00053FAF8F739FCF7F781F9F7F77BFE28789A
:10870000F8F76CFCE878F8F7C7FD2A69A96868797A
:10871000F7F712FF0026F9F715FE0125FCF7D8FA46
:10872000FDF728FEF7F7E2FA09E0F7F72FFD2571CC
:10873000F7F7F6FE2060F7F7F3FEFEF765FBFEF7AE
:1087400089FBFBF7F9FFFDF78FFAFDF7B9FDF7F7A6
:10875000E7FE2368C01A0028B8BF4042B0F57A7F10
:10876000E9DD2379002BE0D0F7F708FD2671DFE77C
:10877000988200208881002070B50D4E0D4CA41BFE
:10878000A4100025A54209D10B4E0C4C00F01EFC94
:10879000A41BA4100025A54205D170BD56F82530B4
:1087A00098470135EEE756F8253098470135F2E74E
:1087B000EC8F0108EC8F0108EC8F0108F08F0108A5
:1087C0002DE970438AB004460D4600F075F8354B2C
:1087D00093F90060731C804689460DD022462B46D3
:1087E00020462946FFF754FA30B9002200232046DC
:1087F0002946FFF743FA20B1404649460AB0BDE892
:108800007083294B0890CDE90245CDE904450193D9
:1088100020462946CEB9254D4FF060440022002362
:10882000CDE90645FFF702FA002833D00223009372
:10883000684600F035FAA8B1089BC3B9DDE906899E
:10884000404649460AB0BDE87083194D0024002215
:108850000023CDE90645FFF7E9F968B102239E42FE
:108860000093E5D100F024FA22230360E4E700F04E
:108870001FFA089B0360E1E70123022E00930BD14E
:1088800000F016FA212303600A4800F00BFACDE944
:108890000601D1E701230093684600F001FA0028A1
:1088A000F2D1EDE7B0000020C88F0108FFFFEFC74D
:1088B0000000F0FFC48F01082DE9F04FB1F5801FD3
:1088C00085B006460F460B465ADA024621F00044B0
:1088D000224300F0F8800029C0F27A810022D64BB2
:1088E000FEF73CFFD54A0B46934206460F466FF013
:1088F000350C4ADCC3F3130505F5152E0EF6647E20
:108900000EF4801E8EF07F5282F440121C1542EA53
:108910000507A4F2FF3464440022C94B30463946AF
:1089200004EB1E54FEF766FDAB1CC3F31303022BCE
:1089300082468B464FF0000230DC0023FFF776F9C9
:10894000002800F0C980002C00F04B812046FEF783
:108950009FFEA5A3D3E9002306460F46FEF7FEFEC1
:10896000A3A3D3E9002304460D4630463946FEF75B
:10897000F5FE02460B4620462946FEF73DFD0AE07D
:10898000AE4A93424FF0000CB4DD32463B463046CF
:108990003946FEF731FD05B0BDE8F08F4FF080435A
:1089A000FEF72AFD02460B4650465946FFF700F8EF
:1089B000064620460F46FEF76BFE3246CDE9000123
:1089C0003B4630463946CDE90267FEF7C7FE024610
:1089D0000B4680468946FEF7C1FE87A3D3E90023F4
:1089E00006460F46FEF7BAFE85A3D3E90023FEF73D
:1089F00003FD32463B46FEF7B1FE83A3D3E90023D5
:108A0000FEF7FAFC32463B46FEF7A8FE80A3D3E908
:108A10000023FEF7F1FC42464B46FEF79FFE7EA385
:108A2000D3E900238046894630463946FEF796FE54
:108A30007BA3D3E90023FEF7DFFC32463B46FEF77B
:108A40008DFE79A3D3E90023FEF7D6FC32463B46E0
:108A5000FEF784FE0B46024649464046FEF7CCFC34
:108A6000A5F5C223C5F5D725A3F27A4351351D4399
:108A7000002D8046894656DD0022724B50465946ED
:108A8000FEF76CFE52465B46FEF768FE06460F4652
:108A9000002C68D132463B4640464946FEF7ACFCC6
:108AA000DDE90223FEF75AFE02460B463046394600
:108AB000FEF7A0FC02460B4650465946FEF79AFCCC
:108AC00005B0BDE8F08F0022002300205E49FEF7CC
:108AD0006FFF05B0BDE8F08F55A3D3E900235046E2
:108AE0005946FEF73BFE02460B4600205549FEF76D
:108AF00081FC524606460F465B4650465946FEF7F5
:108B00002DFE02460B4630463946FEF727FE064646
:108B10000F46002C40F09A8002460B4650465946BC
:108B2000FEF768FC37E7002C00F0A4802EA3D3E901
:108B30000023DDE90001FEF711FE42464B460446E4
:108B40000D4650465946FEF755FCDDE90223FEF777
:108B500005FE27A3D3E9002306460F46DDE9000101
:108B6000FEF7FCFD21E020A3D3E90023DDE90001AD
:108B7000FEF7F4FD32463B4604460D464046494664
:108B8000FEF73AFCDDE90223FEF7E8FD18A3D3E97E
:108B9000002380468946DDE90001FEF7DFFD02463D
:108BA0000B4640464946FEF727FC02460B46304638
:108BB0003946FEF71FFC52465B46FEF71BFC024699
:108BC0000B4620462946FEF715FC05B0BDE8F08FA0
:108BD00002460B46FEF70EFC00220023FEF7E8FEDD
:108BE000D9E600200021D6E60000E0FE422EE63F56
:108BF000763C7935EF39EA3D44523EDF12F1C23F0F
:108C0000DE03CB966446C73F599322942449D23F52
:108C1000935555555555E53F9FC678D0099AC33FA2
:108C2000AF788E1DC571CC3F04FA97999999D93FB9
:108C3000555555555555D53F00005043FFFFEF7F23
:108C40000000F03F0000E03F000050C32046FEF768
:108C50001FFD0FA3D3E9002380468946FEF77EFD62
:108C60000DA3D3E9002304460D4640464946FEF7CE
:108C700075FD9AE702460B4650465946FEF7BAFB89
:108C8000DDE90223FEF76AFD14E700BFAFF30080C1
:108C90000000E0FE422EE63F763C7935EF39EA3DB2
:108CA0000020704700200149704700BF0000F87F96
:108CB000014B1868704700BF4C0000200010161BC5
:108CC0002023272A2D30323537393B3D404143455B
:108CD00047494B4C4E505153545657595A5B5D5E61
:108CE00060616263656667686A6B6C6D6E707172F5
:108CF000737475767778797A7B7C7D7E80808182CB
:108D0000838485868788898A8B8C8D8E8F909091BD
:108D10009293949596969798999A9B9B9C9D9E9FCB
:108D2000A0A0A1A2A3A3A4A5A6A7A7A8A9AAAAABED
:108D3000ACADADAEAFB0B0B1B2B2B3B4B5B5B6B71D
:108D4000B7B8B9B9BABBBBBCBDBDBEBFC0C0C1C15D
:108D5000C2C3C3C4C5C5C6C7C7C8C9C9CACBCBCCA3
:108D6000CCCDCECECFD0D0D1D1D2D3D3D4D4D5D6F2
:108D7000D6D7D7D8D9D9DADADBDBDCDDDDDEDEDF4A
:108D8000E0E0E1E1E2E2E3E3E4E5E5E6E6E7E7E8A7
:108D9000E8E9EAEAEBEBECECEDEDEEEEEFF0F0F10A
:108DA000F1F2F2F3F3F4F4F5F5F6F6F7F7F8F8F973
:108DB000F9FAFAFBFBFCFCFDFDFEFEFF0010161BA2
:108DC0002023272A2D30323537393B3D404143455A
:108DD00047494B4C4E505153545657595A5B5D5E60
:108DE00060616263656667686A6B6C6D6E707172F4
:108DF000737475767778797A7B7C7D7E80808182CA
:108E0000838485868788898A8B8C8D8E8F909091BC
:108E10009293949596969798999A9B9B9C9D9E9FCA
:108E2000A0A0A1A2A3A3A4A5A6A7A7A8A9AAAAABEC
:108E3000ACADADAEAFB0B0B1B2B2B3B4B5B5B6B71C
:108E4000B7B8B9B9BABBBBBCBDBDBEBFC0C0C1C15C
:108E5000C2C3C3C4C5C5C6C7C7C8C9C9CACBCBCCA2
:108E6000CCCDCECECFD0D0D1D1D2D3D3D4D4D5D6F1
:108E7000D6D7D7D8D9D9DADADBDBDCDDDDDEDEDF49
:108E8000E0E0E1E1E2E2E3E3E4E5E5E6E6E7E7E8A6
:108E9000E8E9EAEAEBEBECECEDEDEEEEEFF0F0F109
:108EA000F1F2F2F3F3F4F4F5F5F6F6F7F7F8F8F972
:108EB000F9FAFAFBFBFCFCFDFDFEFEFF00020305D8
:108EC0000608090B0D0E101113141617191B1C1E82
:108ED0001F2122242527292A2C2D2F3032333536E5
:108EE00038393B3C3E3F4143444647494A4C4D4F4D
:108EF000505153545657595A5C5D5F6062636466C3
:108F000067696A6C6D6E707173747577787A7B7C43
:108F10007E7F808283848687888A8B8C8E8F9092D6
:108F20009394959798999A9C9D9E9FA1A2A3A4A57E
:108F3000A7A8A9AAABACAEAFB0B1B2B3B4B5B7B83D
:108F4000B9BABBBCBDBEBFC0C1C2C3C4C5C6C7C819
:108F5000C9CACBCCCDCECFD0D0D1D2D3D4D5D6D711
:108F6000D7D8D9DADBDCDCDDDEDFDFE0E1E2E2E32B
:108F7000E4E4E5E6E7E7E8E8E9EAEAEBECECEDED66
:108F8000EEEEEFF0F0F1F1F2F2F3F3F4F4F4F5F5C4
:108F9000F6F6F7F7F7F8F8F8F9F9F9FAFAFAFBFB49
:108FA000FBFCFCFCFCFCFDFDFDFDFDFEFEFEFEFEF3
:108FB000FEFEFFFFFFFFFFFFFFFFFFFF31363137F0
:108FC00056313036000000006C6F6700F8B500BF06
:108FD000F8BC08BC9E467047F8B500BFF8BC08BC9A
:048FE0009E467047F2
:088FE400B0F3FF7F0100000063
:048FEC00FDC10008BB
:048FF000D9C10008DB
:108FF4000000000000000000010203040607080945
:1090040000D8B805000000000102030401020304B3
:109014000607080906050403C0000000100000004C
:10902400BC8F010801000000006C004000480040B3
:10903400010000000020000001000000500000209A
:10904400000000000000000000000000000000001C
:10905400000000000000000000000000000000000C
:1090640000000000000000000000000000000000FC
:1090740000000000000000000000000000000000EC
:1090840000000000000000000000000000000000DC
:1090940000000000000000000000000000000000CC
:0490A40001000000C7
:0400000508018675F3
:00000001FF
